:100000000C9473110C9477140C94A2140C94CD14CA
:100010000C94F8140C9423150C944E150C9479152B
:100020000C94A4150C94A3110C94A3110C94A3117B
:100030000C94A3110C94A3110C94A3110C94A31170
:100040000C94A3110C9436350C94A3110C94A311A9
:100050000C94A3110C94A3110C9472290C94A51167
:100060000C94A3110C94A11A0C944D1B0C94A31185
:100070000C94A3110C94A3110C94A3110C94A31130
:100080000C94A3110C94A3110C94A3110C94A31120
:100090000C94A3110C94A3110C94A3110C94A31110
:1000A0000C94A3110C94A3110C94A3110C94A31100
:1000B0000C94A3110C94A3110C94A3110C94A311F0
:1000C0000C94A3110C94A3110C94A3110C94A311E0
:1000D0000C94A3110C94A3110C94A3110C94A311D0
:1000E0000C94A311ED12F212F71201130B138413E7
:1000F00015131D1325132F133913431352135C13B8
:100100008413661370137A13A813AB139A139E13F8
:10011000A413E213AF13B313B913BD13C113C71361
:10012000CB13CF13E213D513D913DD13DD17DB1770
:10013000FF17FC17FA1731182E182C188A185818A0
:1001400055185318D41ADA1AEB1AF61AFE1A131B9A
:10015000021B131B061B0A1B131B101B084AD73B51
:100160003BCE016E84BCBFFDC12F3D6C74319ABD86
:1001700056833DDA3D00C77F11BED9E4BB4C3E91AA
:100180006BAAAABE000000803F05A84CCDB2D44E99
:10019000B93836A9020C50B9918688083CA6AAAA9B
:1001A0002ABE000000803F004E414E494E4954593E
:1001B000494E46CDCCCC3D0AD7233C17B7D1387732
:1001C000CC2B329595E6241FB14F0A000020410048
:1001D00000C84200401C4620BCBE4CCA1B0E5AAE92
:1001E000C59D7400000A0B02090C0D0E08070304DC
:1001F00001000000000000000000000000000000FE
:1002000000000000000000000000000000000012DC
:1002100011100000000000000000000000000000BD
:10022000000000000000000000010210202008086B
:100230001020401020408002010201080402010148
:100240000204081020408080402010080402018031
:100250000402018040201008040201080402010188
:10026000020408102040800102040810204080058C
:10027000050505070508080808020202020A0A081F
:100280000804040404010101010101010103030345
:100290000303030303040707070C0C0C0C0C0C0CE2
:1002A0000C0202020206060606060606060B0B0BE9
:1002B0000B0B0B0B0B000020002300260029002C49
:1002C000002F0032000001000003010601090100B7
:1002D000002200250028002B002E003100340002EF
:1002E000010000050108010B010000210024002786
:1002F000002A002D00300033000101000004010736
:10030000010A014F4646004F4E006563686F3A0090
:100310004572726F723A004572726F72207772691D
:1003200074696E6720746F20454550524F4D210A05
:100330000063616E63656C00706F7765726F6666EF
:10034000002F2F616374696F6E3A0020573A0020C6
:10035000573A00202F002042403A0020403A0054F3
:100360006865726D616C2052756E617761790048C5
:100370006F74656E6420544845524D414C2052556F
:100380004E415741590042454420544845524D4141
:100390004C2052554E4157415900202D20496E7630
:1003A000616C6964206578747275646572206E751D
:1003B0006D62657220210A0048656174696E67206C
:1003C0006661696C65640042656420686561746992
:1003D0006E67206661696C656400546865726D6162
:1003E0006C2052756E617761790042454420544813
:1003F00045524D414C2052554E4157415900486598
:100400006174696E67206661696C656400486F7429
:10041000656E642048656174696E67206661696C09
:10042000656400546865726D616C2052756E617709
:10043000617900486F74656E6420544845524D419F
:100440004C2052554E41574159004D494E54454D4F
:10045000502074726967676572656400486F7465DF
:100460006E64204572723A204D494E54454D5000FD
:100470004572723A204D494E54454D5020424544F4
:10048000004D415854454D5020747269676765723C
:10049000656400486F74656E64204572723A204D41
:1004A000415854454D50004572723A204D415854C0
:1004B000454D502042454400626564002C2073790C
:1004C0007374656D2073746F707065642120486566
:1004D000617465725F49443A200023646566696E01
:1004E000652044454641554C545F004B6420004B09
:1004F0006920004B70200000626564005049442070
:100500004175746F74756E652066696E6973686590
:1005100064212050757420746865206C61737420A8
:100520004B702C204B6920616E64204B6420636FFC
:100530006E7374616E74732066726F6D2062656C89
:100540006F7720696E746F20436F6E66696775728E
:100550006174696F6E2E680A0050494420417574B9
:100560006F74756E65206661696C656421207469BD
:100570006D656F75740A00546865726D616C205208
:10058000756E6177617900486F74656E64205448B8
:1005900045524D414C2052554E415741590042451C
:1005A0004420544845524D414C2052554E415741EC
:1005B000590048656174696E67206661696C65649D
:1005C00000486F74656E642048656174696E6720C9
:1005D0006661696C65640042656420686561746980
:1005E0006E67206661696C656400504944204175FE
:1005F000746F74756E65206661696C656421205442
:10060000656D706572617475726520746F6F2068B6
:100610006967680A00204B643A2000204B693A2041
:1006200000204B703A20000A20436C6173736963A9
:1006300020504944200A002054753A2000204B7570
:100640003A2000206D61783A2000206D696E3A20D2
:100650000020643A200020626961733A200050490A
:1006600044204175746F74756E6520737461727483
:100670000A00504944204175746F74756E65206698
:1006800061696C6564212054656D70657261747573
:10069000726520746F6F20686967680A001000AD8A
:1006A0000330016A0150022B0170030A019004F526
:1006B00000B005E500D006D800F007CE001009C54F
:1006C00000300ABE00500BB700700CB100900DABAB
:1006D00000B00EA600D00FA200F0109D00101299DD
:1006E00000301395005014920070158E0090168BF8
:1006F00000B0178700D0188400F0198100101B7E0D
:1007000000301C7B00501D7900701E7600901F7316
:1007100000B0207000D0216E00F0226B0010246920
:100720000030256600502663007027610090285E27
:1007300000B0295C00D02A5900F02B5600102D542F
:1007400000302E5100502F4E0070304B0090314839
:1007500000B0324500D0334200F0343E0010363B4A
:1007600000303737005038330070392E00903A2966
:1007700000B03B2300D03C1B00F03D1100103F01B6
:1007800000F03F00001000C90210012C01400122BE
:100790000170011801B0010E01F00104015002FACC
:1007A00000B002F0003003E600D003DC009004D279
:1007B000007005C800A006BE000008B400B009AA79
:1007C00000D00BA000600E960060118C0000158216
:1007D0000020197800C01D6E00A0226400B0275AC6
:1007E00000902C500000314600E0343C00103832BC
:1007F00000903A2800603C1E00A03D1400803E0A94
:1008000000203F00006F70656E0054524947474515
:10081000524544003A20007A5F6D6178007A5F6D3E
:10082000696E00795F6D617800795F6D696E00783F
:100830005F6D617800785F6D696E005265706F72F0
:1008400074696E6720656E6473746F702073746171
:100850007475730A00205A3A0020593A0020583A19
:1008600000656E6473746F7073206869743A200059
:10087000486F6D696E67206661696C656400496EDA
:1008800076616C69642065787472756465720A00BB
:1008900045303A20005A3A2000593A20004D533151
:1008A0002C4D53322C4D53332050696E730A583AF5
:1008B00020004D6963726F737465707320756E618B
:1008C0007661696C61626C650A00205A3A002059B1
:1008D0003A0020436F756E7420583A00C231000010
:1008E0001C260000F4190000D80F0000EB080000DF
:1008F000C0040000750200004001000024F4D43060
:1009000050C38E20C2A24017828B7011127A910DB3
:10091000816CD90AA861E108C7586607615143068E
:100920001E4B5D05C145A7041A411104093D9803FA
:10093000713931034036DB0265339102D430540201
:10094000802E1D02632CEE01752AC501B028A0017E
:10095000102781018F2564012B244B01E0223401F3
:10096000AC211F018D200D01801FFC00841EED00B5
:10097000971DDF00B81CD200E61BC600201BBC0080
:10098000641AB200B219A8000A19A0006A189900E6
:10099000D117910040178B00B516840031167E00E8
:1009A000B31579003A157300C7146F0058146A0024
:1009B000EE1366008813630025135E00C7125B0008
:1009C0006C12570015125400C111510070114F00E4
:1009D00021114B00D61049008D10470046104400ED
:1009E00002104200C00F4000800F3E00420F3C004A
:1009F000060F3B00CB0E3800930E37005C0E35001F
:100A0000270E3400F30D3200C10D3100900D30007F
:100A1000600D2E00320D2D00050D2C00D90C2B0081
:100A2000AE0C2900850C29005C0C2700350C270032
:100A30000E0C2600E80B2400C40B2400A00B23009E
:100A40007D0B23005A0B2100390B2100180B2000CD
:100A5000F80A1F00D90A1E00BB0A1E009D0A1D00CD
:100A6000800A1D00630A1C00470A1B002C0A1B0099
:100A7000110A1A00F7091A00DD091900C409190042
:100A8000AB091900920917007B09180063091700C8
:100A90004C09160036091600200916000A0915002F
:100AA000F5081500E0081400CC081400B80814007C
:100AB000A4081400900813007D0812006B081300AE
:100AC00058081200460812003408110023081100CB
:100AD0001208110001081100F0071000E0071000D3
:100AE000D0071000C0071000B0070F00A1071000CA
:100AF00091070E0083070F0074070F0065070E00B3
:100B000057070E0049070E003B070D002E070E0089
:100B100020070D0013070D0006070D00F9060C0055
:100B2000ED060D00E0060C00D4060C00C8060C0013
:100B3000BC060C00B0060C00A4060B0099060C00C5
:100B40008D060B0082060B0077060B006C060B006F
:100B500061060A0057060B004C060A0042060A000E
:100B600038060A002E060A0024060A001A060A00A1
:100B70001006090007060A00FD050900F405090032
:100B8000EB050900E2050900D9050900D0050900B7
:100B9000C7050900BE050900B5050800AD05080038
:100BA000A50509009C050800940508008C050800AF
:100BB000840508007C050800740508006C05070022
:100BC000650508005D050700560508004E0507008D
:100BD00047050700400508003805070031050700F4
:100BE0002A050700230507001C0506001605070057
:100BF0000F0507000805060002050700FB040600B4
:100C0000F5040700EE040600E8040600E20407000D
:100C1000DB040600D5040600CF040600C904060064
:100C2000C3040600BD040600B7040600B1040500B5
:100C3000AC040600A6040600A00405009B04060000
:100C400095040500900406008A040500850405004B
:100C5000800406007A040500750405007004050090
:100C60006B04050066040500610405005C040500D2
:100C700057040500520405004D0405004804050012
:100C8000430405003E0404003A0405003504050051
:100C9000300404002C04050027040400230405008C
:100CA0001E0404001A0404001604050011040400C4
:100CB0000D040400090405000404040000040400F9
:100CC000FC030400F8030400F4030400F003040030
:100CD000EC030400E8030400E4030400E003040060
:100CE000DC030400D8030400D4030400D003040090
:100CF000CC030400C8030300C503030024F404D993
:100D0000201BC40C5C0E9804C4095F0265077101C6
:100D1000F405F900FB04B30048048700C10369002F
:100D20005803550003034500BE023A008402310017
:100D300053022A002902250004022000E4011C00BD
:100D4000C8011900AF0117009801140084011300B5
:100D5000710110006101100051010E0043010D00EE
:100D600036010B002B010B0020010B0015010900BF
:100D70000C01090003010800FB000800F300080053
:100D8000EB000700E4000600DE000600D8000600C5
:100D9000D2000600CC000500C7000500C200050017
:100DA000BD000400B9000400B5000400B100040057
:100DB000AD000400A9000400A5000300A200030088
:100DC0009F0004009B0003009800030095000200B0
:100DD00093000300900003008D0002008B000300CD
:100DE00088000200860002008400030081000200E7
:100DF0007F0002007D0002007B00020079000200FB
:100E00007700010076000200740002007200010009
:100E1000710002006F0002006D0001006C00020012
:100E20006A0001006900020067000100660001001D
:100E30006500010064000200620001006100010021
:100E4000600001005F0002005D0001005C00010025
:100E50005B0001005A000100590001005800010028
:100E60005700010056000100550001005400010028
:100E70005300000053000100520001005100010026
:100E8000500001004F0001004E0000004E00010024
:100E90004D0001004C0001004B0000004B00010020
:100EA0004A0001004900010048000000480001001C
:100EB0004700010046000000460001004500000018
:100EC0004500010044000100430000004300010010
:100ED000420000004200010041000000410001000A
:100EE000400001003F0000003F0001003E00000004
:100EF0003E0001003D0000003D0001003C000000FC
:100F00003C0000003C0001003B0000003B000100F1
:100F10003A0000003A0001003900000039000100E9
:100F200038000000380000003800010037000000E1
:100F300037000100360000003600000036000100D6
:100F400035000000350000003500010034000000CD
:100F500034000000340001003300000033000000C2
:100F600033000100320000003200000032000100B6
:100F700031000000310000003100010030000000AD
:100F800030000000300001002F0000002F000000A2
:100F90002F0000002F0001002E0000002E00000096
:100FA0002E0001002D0000002D0000002D0000008B
:100FB0002D0001002C0000002C0000002C0000007F
:100FC0002C0001002B0000002B0000002B00000073
:100FD0002B0001002A0000002A0000002A00000067
:100FE0002A0001002900000029000000290000005B
:100FF000290000002900010028000000280000004E
:101000002800000028000000280001002700000040
:101010002700000027000000270000002700010033
:101020002600000026000000260000002600000028
:10103000260001002500000025000000250000001A
:10104000250000002500000025000100240000000C
:1010500024000000240000002400000024000100FF
:1010600023000000230000002300000023000000F4
:1010700023000000230000002300010022000000E4
:1010800022000000220000002200000022000000D8
:1010900022000100210000002100000021000000CA
:1010A00021000000210000002100000021000100BB
:1010B00020000000200000002000000020000000B0
:1010C000200000002000000020000000200001009F
:1010D0001F0000001F0000001F0000001F00000094
:1010E0001F0000001F0000001F0001001E00000084
:1010F0001E0000001E0000001E0000003A0A002032
:10110000286D6D2900205300205A002059002058D6
:101110000020204D3432352046004261636B6C6103
:10112000736820636F6D70656E736174696F6E3A7A
:101130000A00204500205A0020204D393037205821
:101140000053746570706572206D6F746F722063E8
:10115000757272656E74733A0A0020204D39303012
:10116000204B004C696E65617220416476616E634C
:10117000653A0A0020204D383531205A005A2D504A
:10118000726F6265204F66667365740020440020AC
:10119000490020204D3330342050002044002049A5
:1011A0000020204D333031205000504944207365D9
:1011B0007474696E67733A0A0020204D343230200F
:1011C00053004175746F20426564204C6576656CF0
:1011D000696E673A0A00204500205A002059002015
:1011E000580020540020530020204D32303520423A
:1011F0000020453C6D61785F655F6A65726B3E00FB
:1012000020583C6D61785F785F6A65726B3E20594B
:101210003C6D61785F795F6A65726B3E205A3C6D08
:1012200061785F7A5F6A65726B3E00416476616ED9
:101230006365643A20423C6D696E5F7365676D65F6
:101240006E745F74696D655F75733E20533C6D69A4
:101250006E5F66656564726174653E20543C6D69BD
:101260006E5F74726176656C5F66656564726174E9
:10127000653E0020540020520020204D32303420A2
:101280005000416363656C65726174696F6E2028FC
:10129000756E6974732F7332293A20503C707269ED
:1012A0006E745F616363656C3E20523C726574725C
:1012B0006163745F616363656C3E20543C7472616A
:1012C00076656C5F616363656C3E0A0020450020B3
:1012D0005A0020590020204D3230312058004D61F5
:1012E00078696D756D20416363656C6572617469C1
:1012F0006F6E2028756E6974732F7332293A0A0055
:10130000204500205A0020590020204D3230332043
:1013100058004D6178696D756D2066656564726110
:101320007465732028756E6974732F73293A0A00E7
:1013300053746570732070657220756E69743A0A13
:10134000002020473231202020203B20556E697438
:101350007320696E206D6D0048617264636F64650F
:10136000642044656661756C742053657474696E9D
:101370006773204C6F616465640A002823000028AD
:1013800023000064000000E8030000000096430012
:1013900000964300000041000020420000C94200C6
:1013A00000C9420000C8440000D243454550524F96
:1013B0004D20496E697469616C697A65640A002917
:1013C0000A002062797465733B20637263200020F9
:1013D00073746F7265642073657474696E677320CB
:1013E00072657472696576656420280020286361DF
:1013F0006C63756C6174656429210A0020213D20AD
:1014000000454550524F4D20435243206D69736D46
:1014100061746368202D202873746F7265642920BD
:10142000002053697A653A2000496E6465783A2055
:1014300000204D61726C696E3D563637290A0045B1
:101440004550524F4D2076657273696F6E206D69FD
:10145000736D617463682028454550524F4D3D00BF
:10146000290A002062797465733B2063726320004F
:1014700053657474696E67732053746F726564206A
:101480002800454550524F4D206461746173697A5C
:1014900065206572726F722E0A004175746F6C65FB
:1014A00076656C206661696C65640A005761726ECE
:1014B000696E673A20486F6D696E672042756D707E
:1014C0002044697669736F72203C20310A00020261
:1014D000042066697273740A00486F6D65200020ED
:1014E000746F6F206C6F6E672065787472757369A6
:1014F0006F6E2070726576656E7465640A00206395
:101500006F6C6420657874727573696F6E20707289
:101510006576656E7465640A0020453A00205A3A83
:101520000020593A00583A000000F0410000F04114
:1015300000000041FF01010000A0400000A04000A9
:101540000000400000254300004543000021430007
:101550000040C0CDCC364300001F4300002243CDE5
:10156000CC364300001F43000040C0333363C1004A
:101570000000C020746F6F206C6F6E6720657874F8
:10158000727573696F6E2070726576656E746564CE
:101590000A0020636F6C6420657874727573696FDC
:1015A0006E2070726576656E7465640A006275738C
:1015B000793A2070617573656420666F7220696E78
:1015C0007075740A00627573793A2070617573657D
:1015D0006420666F7220757365720A006275737994
:1015E0003A2070726F63657373696E670A004D31DC
:1015F00031372050726F6265207375636365737352
:1016000066756C0A0020496E76616C6964206578A5
:101610007472756465722000205A3A200020593A8D
:10162000200042656420583A200050726F626520A5
:101630005A204F66667365743A20003F5A206F75D2
:1016400074206F662072616E676520282D322074C9
:101650006F2035290A00220A00556E6B6E6F776E77
:1016600020636F6D6D616E643A20220045455052D3
:101670004F4D204F4B0A004543484F00494E464FBF
:10168000004552524F52530044525952554E004356
:101690004F4D4D554E49434154494F4E006F66667C
:1016A0000077167C16811688168F164445425547DA
:1016B0003A00205A00205900580020204D61783A05
:1016C0002000205A00205900580020204D696E3A11
:1016D0002000536F667420656E6473746F70733A84
:1016E00020002569730025696D202569730025692F
:1016F000682025696D2025697300256964202569A6
:10170000682025696D202569730025697920256980
:1017100064202569682025696D2025697300507251
:10172000696E742074696D653A20004D3131332043
:1017300053002F2F20004361703A004348414D422F
:1017400045525F54454D5045524154555245004D08
:101750004F54494F4E5F4D4F4445530054484552F6
:101760004D414C5F50524F54454354494F4E0041F8
:1017700055544F5245504F52545F53445F53544158
:101780005455530050524F4D50545F535550504F85
:10179000525400454D455247454E43595F504152C2
:1017A00053455200434153455F4C494748545F42BB
:1017B00052494748544E45535300544F47474C45B0
:1017C0005F4C494748545300534F46545741524584
:1017D0005F504F574552004255494C445F50455267
:1017E00043454E54004C4556454C494E475F444195
:1017F0005441005A5F50524F4245004155544F4C9E
:101800004556454C005052494E545F4A4F42005095
:10181000524F4752455353004155544F5245504F34
:1018200052545F54454D5000564F4C554D455452FF
:10183000494300454550524F4D0042494E4152598F
:101840005F46494C455F5452414E53464552005302
:10185000455249414C5F584F4E5F584F46460046EF
:1018600049524D574152455F4E414D453A4D617287
:101870006C696E20204649524D574152455F56458E
:101880005253494F4E3A322E302E302E31333520BE
:1018900045585452554445525F545950453A53693E
:1018A0006E676C6545787472756465724165726FB8
:1018B000563220534F555243455F434F44455F5581
:1018C000524C3A68747470733A2F2F636F64652EAC
:1018D000616C6570686F626A656374732E636F6DA7
:1018E0002F646966667573696F6E2F4D41524C495E
:1018F0004E2050524F544F434F4C5F564552534920
:101900004F4E3A312E30204D414348494E455F54A9
:101910005950453A4C756C7A426F74204D696E6926
:101920002045585452554445525F434F554E543A02
:101930003120555549443A33353134383762362DE4
:10194000636139612D346331612D383736352D644B
:1019500036363862316461363538350A0020284E13
:101960006F7420796574206D656173757265642983
:1019700000202041766572616765206D6561737531
:10198000726564206261636B6C61736820286D6DA1
:10199000293A002020536D6F6F7468696E672028A4
:1019A0006D6D293A2020202020202020202020207A
:1019B0002020202020530020204261636B6C617343
:1019C000682044697374616E636520286D6D293ADF
:1019D000202020202020202000202846312E3020CA
:1019E0003D2066756C6C2C2046302E30203D206EDC
:1019F0006F6E65290A002020436F727265637469F7
:101A00006F6E20416D6F756E742F466164652D6F2A
:101A100075743A2020202020460061637469766541
:101A20003A0A00696E004261636B6C61736820431F
:101A30006F7272656374696F6E2000205A002050C7
:101A40006F736974696F6E616C204572726F723A60
:101A50000A004E6F7A7A6C6520546970204F757455
:101A600065722044696D656E73696F6E733A0A0022
:101A70002020546F703A2000202046726F6E743A16
:101A8000200020204C6566743A20004261636B6C34
:101A90006173683A0A00205A0043656E7465723AB1
:101AA0000A00202046726F6E743A200020204C6598
:101AB00066743A20002020546F703A200053696405
:101AC00065733A0A00426564204C6576656C696E00
:101AD0006720004661696C656420746F20656E61E3
:101AE000626C6520426564204C6576656C696E6742
:101AF0000A00426564204C6576656C20436F727203
:101B0000656374696F6E204D61747269783A000A7A
:101B10000A426564204C6576656C20436F7272657D
:101B20006374696F6E204D61747269783A00202B7E
:101B3000000A436F727265637465642042656420B5
:101B40004865696768742076732E20426564205466
:101B50006F706F6C6F67793A0A00202B000A42653C
:101B6000642048656967687420546F706F6772619C
:101B70007068793A0A2020202B2D2D2D20424143D8
:101B80004B202D2D2B0A2020207C202020202020BF
:101B900020202020207C0A204C207C20202020286F
:101BA0002B29202020207C20520A2045207C202028
:101BB0002020202020202020207C20490A20462090
:101BC0007C20282D29204E20282B29207C20470AE4
:101BD0002054207C20202020202020202020207C19
:101BE00020480A2020207C20202020282D29202069
:101BF00020207C20540A2020207C2020202020200F
:101C000020202020207C0A2020204F2D2D204652ED
:101C10004F4E54202D2D2B0A2028302C30290A001D
:101C20003474682070726F626520706F696E742CF6
:101C30002064697374616E63652066726F6D2070D5
:101C40006C616E653A2000202844525952554E2945
:101C500000473239204175746F20426564204C651D
:101C600076656C696E67003F20284C2C522C462C00
:101C70004229206F7574206F6620626F756E6473E1
:101C80002E0A003F50726F626520706F696E747328
:101C90002028592920697320696D706C61757369FA
:101CA000626C652028322D32292E0A003F50726F57
:101CB000626520706F696E747320285829206973DB
:101CC00020696D706C61757369626C652028322DB6
:101CD00032292E0A003F2856296572626F736520EB
:101CE0006C6576656C20697320696D706C617573C5
:101CF00069626C652028302D34292E0A00416476F3
:101D0000616E6365204B3D003F4B2076616C7565CD
:101D1000206F7574206F662072616E6765202830B1
:101D20002D3130292E0A004D31313720486F742073
:101D3000456E642048656174696E672E2E2E0A4DCB
:101D400031303420533137302054300A4732382074
:101D50004F310A473120593235205A31302046352B
:101D60003030300A4D313137205265776970696EF5
:101D700067206E6F7A7A6C650A54300A47312058B2
:101D800031313520593137322046353030300A4D27
:101D900031303920523137302054300A4731205AFF
:101DA000310A4731205831313520593137322046F8
:101DB000343030300A4731205834352059313732E9
:101DC0002046343030300A473120583131352059DF
:101DD0003137322046343030300A473120583435DC
:101DE00020593137322046343030300A47312058BC
:101DF00031313520593137322046343030300A47BE
:101E00003120583435205931373220463430303083
:101E10000A47312058313135205931373220463484
:101E20003030300A4731205834352059313732208C
:101E300046343030300A473120583131352059315D
:101E400037322046343030300A473120583435207C
:101E5000593137322046343030300A47312058313A
:101E6000313520593137322046343030300A47314D
:101E70002058343520593137322046343030300A3A
:101E80004731205A31350A4D3130362053323535FD
:101E9000200A47302058302059300A4D313039203F
:101EA000523136302054300A4D3130370A00204646
:101EB0006C6F773A200020643A0020693A00207065
:101EC0003A00204500205A00205900204D39322088
:101ED000580043290A0061626C656420286D696EB0
:101EE0002074656D70200064697300656E00436F37
:101EF0006C64206578747275646573206172652006
:101F000000205400205200416363656C6572617467
:101F1000696F6E3A205000496E76616C6964206585
:101F2000787472756465720A0020643A0020693A18
:101F30000020703A0047322F4733206261642070DE
:101F40006172616D65746572730A005072696E74B6
:101F500065722073746F7070656420647565207499
:101F60006F206572726F72732E20466978207468D4
:101F700065206572726F7220616E642075736520D2
:101F80004D39393920746F20726573746172742E03
:101F9000202854656D70657261747572652069736F
:101FA0002072657365742E205365742069742061F6
:101FB000667465722072657374617274696E6729E4
:101FC0000A004E6F20436865636B73756D207769F7
:101FD0007468206C696E65206E756D6265722C2068
:101FE0004C617374204C696E653A200063686563C8
:101FF0006B73756D206D69736D617463682C204C13
:10200000617374204C696E653A20004C696E6520DE
:102010004E756D626572206973206E6F74204C611D
:102020007374204C696E65204E756D6265722B313C
:102030002C204C617374204C696E653A20004D3140
:10204000313000526573656E643A200020420020F2
:1020500050006F6B00220A00656E717565756569C9
:102060006E67202200504944204175746F74756E6C
:1020700065206661696C6564212042616420657831
:10208000747275646572206E756D6265720A006F98
:102090006B002020506C616E6E65724275666665DD
:1020A0007242797465733A20002046726565204D4E
:1020B000656D6F72793A2000436F6D70696C65646D
:1020C0003A204A756E20313920323031390A0020E9
:1020D0007C20417574686F723A2028416C65706885
:1020E000204F626A6563747320496E632E2C204C06
:1020F000756C7A426F7420476974205265706F73F3
:1021000069746F7279290A0000204C61737420553C
:102110007064617465643A2000322E302E302E31A6
:1021200033350A004D61726C696E0020536F66741E
:10213000776172652052657365740A002057617477
:102140006368646F672052657365740A0020427289
:102150006F776E206F75742052657365740A002066
:1021600045787465726E616C2052657365740A00FF
:10217000506F77657255700A0073746172740A004B
:102180005072696E7465722068616C7465642E208B
:102190006B696C6C28292063616C6C6564210A0092
:1021A0004B494C4C206361757365642062792074DF
:1021B0006F6F206D75636820696E61637469766501
:1021C0002074696D65202D2063757272656E7420B0
:1021D000636F6D6D616E643A20004D3132310A4794
:1021E00030205A31300A4732382058302059300ACE
:1021F0004731320A4D31303920523136300A4D31B3
:1022000031372050726F62696E67206265640070BA
:10221000726F62655F726577697065004175746F92
:102220006C6576656C206661696C6564004D313162
:102230003720426564206C6576656C696E67206640
:1022400061696C65642E0A4730205A31300A473084
:102250002045300A4D333030205032352053383845
:10226000300A4D333030205035302053300A4D3352
:1022700030302050323520533838300A4D3330302A
:10228000205035302053300A4D3330302050323515
:1022900020533838300A47342053310070726F624F
:1022A000655F6661696C65640050726F7465637424
:1022B00065642050696E0A0025301D0C1E282924F3
:1022C000311C0B184527232F1B0A174443222B1AB6
:1022D0004142043803FF3604080606000100D11D00
:1022E000E132586E849411241FBECFEFD1E2DEBFDD
:1022F000CDBF00E00CBF13E0A0E0B2E0EAE7F4E7F6
:1023000001E00BBF02C007900D92AE39B107D9F7BB
:102310002EE0AEE9B3E001C01D92A93EB207E1F79D
:1023200011E1C3E7D1E100E006C021970109802F48
:10233000FE010E94D2B2CF36D10780E00807A9F78C
:1023400071D40C943BBA0C9400001F920F920FB6FC
:102350000F9211242F933F938F939F93AF93BF932B
:1023600080919F039091A003A091A103B091A2033B
:1023700030919E0323E0230F2D3720F40196A11DF9
:10238000B11D05C026E8230F0296A11DB11D2093A3
:102390009E0380939F039093A003A093A103B09307
:1023A000A2038091A3039091A403A091A503B091EF
:1023B000A6030196A11DB11D8093A3039093A403CE
:1023C000A093A503B093A603BF91AF919F918F9166
:1023D0003F912F910F900FBE0F901F9018952FB720
:1023E000F89460919F037091A0038091A103909154
:1023F000A2032FBF08953FB7F8948091A303909153
:10240000A403A091A503B091A60326B5A89B05C07F
:102410002F3F19F00196A11DB11D3FBFBA2FA92F63
:10242000982F8827820F911DA11DB11DBC01CD01E0
:1024300042E0660F771F881F991F4A95D1F70895CC
:102440008F929F92AF92BF92CF92DF92EF92FF92C4
:102450006B017C01D0DF4B015C01C114D104E104AC
:10246000F104F1F09CD3C7DFDC01CB018819990995
:10247000AA09BB09883E9340A105B10570F321E08C
:10248000C21AD108E108F10888EE880E83E0981E90
:10249000A11CB11CC114D104E104F10421F7DDCF6A
:1024A000FF90EF90DF90CF90BF90AF909F908F9074
:1024B00008958230910538F0880F991F880F991F71
:1024C00005970197F1F70895789484B5826084BDEB
:1024D00084B5816084BD85B5826085BD85B5816028
:1024E00085BDEEE6F0E0808181608083E1E8F0E088
:1024F0001082808182608083808181608083E0E8B7
:10250000F0E0808181608083E1EBF0E08081846095
:102510008083E0EBF0E0808181608083E1E9F0E09E
:10252000808182608083808181608083E0E9F0E047
:10253000808181608083E1EAF0E080818260808335
:10254000808181608083E0EAF0E080818160808327
:10255000E1E2F1E08081826080838081816080831C
:10256000E0E2F1E0808181608083EAE7F0E0808151
:1025700084608083808182608083808181608083A9
:102580008081806880831092C10008951F93CF934B
:10259000DF93182FEB0161E016D1209711F460E072
:1025A00004C0CF3FD10531F461E0812FDF91CF919D
:1025B0001F9145C1E12FF0E0ED51FE4FE4914E2F08
:1025C00050E0FA013197E231F10508F09DC088270B
:1025D000EE58FF4F8F4F0C94D2B284B5806884BD03
:1025E000C7BD97C084B5806284BDC8BD92C08091CC
:1025F0008000806880938000D0938900C093880019
:1026000088C080918000806280938000D0938B008E
:10261000C0938A007EC08091800088608093800093
:10262000D0938D00C0938C0074C08091B0008068FE
:102630008093B000C093B3006CC08091B000806202
:102640008093B000C093B40064C080919000806813
:1026500080939000D0939900C09398005AC08091C5
:102660009000806280939000D0939B00C0939A006A
:1026700050C080919000886080939000D0939D001E
:10268000C0939C0046C08091A00080688093A00009
:102690008091A0008F7B8093A000D093A900C0936D
:1026A000A80037C08091A00080628093A000D093E2
:1026B000AB00C093AA002DC08091A00088608093D9
:1026C000A000D093AD00C093AC0023C08091200146
:1026D000806880932001D0932901C093280119C0FC
:1026E00080912001806280932001D0932B01C093C0
:1026F0002A010FC080912001886080932001D0932F
:102700002D01C0932C0105C0C038D1050CF04CCF71
:1027100046CFDF91CF911F91089590E0FC01319752
:10272000E231F10508F04EC08827EC57FF4F8F4F7C
:102730000C94D2B2809180008F7703C0809180008A
:102740008F7D80938000089580918000877FF9CFEE
:1027500084B58F7702C084B58F7D84BD0895809144
:10276000B0008F7703C08091B0008F7D8093B00060
:102770000895809190008F7707C0809190008F7DA1
:1027800003C080919000877F80939000089580918E
:10279000A0008F7707C08091A0008F7D03C080913B
:1027A000A000877F8093A0000895809120018F77FB
:1027B00007C0809120018F7D03C080912001877F19
:1027C000809320010895CF93DF9390E0FC01E75DB3
:1027D000FD4F2491FC01E159FD4F8491882361F163
:1027E00090E0880F991FFC01E751FD4FC591D491EE
:1027F000FC01E153FD4FA591B491611109C09FB750
:10280000F8948881209582238883EC912E230BC035
:10281000623061F49FB7F8943881822F80958323CA
:102820008883EC912E2B2C939FBF06C08FB7F89412
:10283000E8812E2B28838FBFDF91CF9108951F93BE
:10284000CF93DF93282F30E0F901ED51FE4F8491B3
:10285000F901E75DFD4FD491F901E159FD4FC491B4
:10286000CC23C1F0162F811158DFEC2FF0E0EE0FD2
:10287000FF1FE153FD4FA591B4918FB7F89411114B
:1028800005C09C91ED2FE095E92302C0EC91ED2B62
:10289000EC938FBFDF91CF911F910895CF93DF937A
:1028A000282F30E0F901ED51FE4F8491F901E75DE9
:1028B000FD4FD491F901E159FD4FC491CC2389F02A
:1028C00081112BDFEC2FF0E0EE0FFF1FEB54FD4FDB
:1028D000A591B491EC91ED2381E090E021F480E0AA
:1028E00002C080E090E0DF91CF91089508951F929B
:1028F0000F920FB60F9211240BB60F922F933F93A6
:102900004F935F936F937F938F939F93AF93BF93F7
:10291000EF93FF93E0910402F09105021995FF9166
:10292000EF91BF91AF919F918F917F916F915F9147
:102930004F913F912F910F900BBE0F900FBE0F90B4
:102940001F9018951F920F920FB60F9211240BB67D
:102950000F922F933F934F935F936F937F938F9338
:102960009F93AF93BF93EF93FF93E0910602F09193
:1029700007021995FF91EF91BF91AF919F918F91B0
:102980007F916F915F914F913F912F910F900BBE6F
:102990000F900FBE0F901F9018951F920F920FB6B9
:1029A0000F9211240BB60F922F933F934F935F9387
:1029B0006F937F938F939F93AF93BF93EF93FF9307
:1029C000E0910802F09109021995FF91EF91BF91F2
:1029D000AF919F918F917F916F915F914F913F91B7
:1029E0002F910F900BBE0F900FBE0F901F90189558
:1029F0001F920F920FB60F9211240BB60F922F93C6
:102A00003F934F935F936F937F938F939F93AF9376
:102A1000BF93EF93FF93E0910A02F0910B02199597
:102A2000FF91EF91BF91AF919F918F917F916F91A6
:102A30005F914F913F912F910F900BBE0F900FBE62
:102A40000F901F9018951F920F920FB60F9211249E
:102A50000BB60F922F933F934F935F936F937F9398
:102A60008F939F93AF93BF93EF93FF93E0910002F7
:102A7000F09101021995FF91EF91BF91AF919F9154
:102A80008F917F916F915F914F913F912F910F9017
:102A90000BBE0F900FBE0F901F9018951F920F92B4
:102AA0000FB60F9211240BB60F922F933F934F93B3
:102AB0005F936F937F938F939F93AF93BF93EF93A6
:102AC000FF93E0910202F09103021995FF91EF91BB
:102AD000BF91AF919F918F917F916F915F914F9136
:102AE0003F912F910F900BBE0F900FBE0F901F9034
:102AF00018951F920F920FB60F9211240BB60F92DA
:102B00002F933F934F935F936F937F938F939F93F5
:102B1000AF93BF93EF93FF93E0910C02F0910D02FE
:102B20001995FF91EF91BF91AF919F918F917F91F7
:102B30006F915F914F913F912F910F900BBE0F902E
:102B40000FBE0F901F9018951F920F920FB60F9205
:102B500011240BB60F922F933F934F935F936F9374
:102B60007F938F939F93AF93BF93EF93FF93E091E6
:102B70000E02F0910F021995FF91EF91BF91AF9165
:102B80009F918F917F916F915F914F913F912F9185
:102B90000F900BBE0F900FBE0F901F9018950895C9
:102BA0004F925F926F927F92AF92BF92CF92DF92DD
:102BB000EF92FF920F931F93CF93DF93CDB7DEB7C2
:102BC00029013A019B01AC0124193509460957092D
:102BD0008A899B89AC89BD89BC01CD016A197B09B1
:102BE0008C099D090E945EB2A8019701241935093C
:102BF000460957090E94B6B2CA01B9016A0D7B1D88
:102C00008C1D9D1DDF91CF911F910F91FF90EF9033
:102C1000DF90CF90BF90AF907F906F905F904F907C
:102C20000895089551DCFDDF0E94F1ADC0E0D0E0D1
:102C30000E9470AE2097E1F30E940000F9CFCF937D
:102C4000C82F0E944333CC2349F024982C9A65E086
:102C500070E080E090E0F4DB149A03C0249A2C9892
:102C60001498CF91089580E0EACFCF92DF92EF924F
:102C7000FF926B017C0183E3C816D104E104F104E7
:102C800068F082E3C81AD108E108F10862E370E055
:102C900080E090E0D5DB0E949727EDCFC701B60119
:102CA000CFDBFF90EF90DF90CF900C949727DC0163
:102CB000FB01460F571FE417F507C1F081912D91D5
:102CC0003C911197382798E0B901660F771F37FFBD
:102CD00006C09B0181E2282780E1382701C09B01C3
:102CE000915091F711963C932E93E5CF0895CF9391
:102CF000DF93FC018491EF012196882319F061D5BF
:102D0000FE01F8CFDF91CF9108958AE093E0EFCFF5
:102D100080E193E0ECCF0F931F93CF93DF931F924B
:102D20001F92CDB7DEB769837A83E1DF6981062F11
:102D30007A81172FF80181918F01882311F041D5F5
:102D4000F9CF0F900F90DF91CF911F910F910895C0
:102D5000CF93DF93EB01CBDF6AE070E0CE01DF9130
:102D6000CF9122C6CF92DF92EF92FF926A017B0150
:102D7000BEDF4AE050E0C701B601FF90EF90DF9060
:102D8000CF9001C6CF92DF92EF92FF926A017B0152
:102D9000AEDF42E050E0C701B601FF90EF90DF9058
:102DA000CF908DC6CF92DF92EF92FF926A017B01A6
:102DB0009EDF42E050E0C701B601FF90EF90DF9048
:102DC000CF907DC6CF93DF93EB0191DF6AE070E097
:102DD000CE01DF91CF91FDC5CF92DF92EF92FF92AE
:102DE0006A017B0184DF4AE050E0C701B601FF9031
:102DF000EF90DF90CF90E7C5811103C083E093E0AF
:102E000002C087E093E073CFF7DF8AE0DAC4CF93A4
:102E1000DF931F921F92CDB7DEB72091E30E309162
:102E2000E40ECE0101962115310519F4895E9E400C
:102E300002C0821B930B9A83898389819A810F90A8
:102E40000F90DF91CF91089581E0089581E008957A
:102E50008F929F92AF92BF92CF92DF92EF92FF92AA
:102E60000F931F93CF93DF931F921F92CDB7DEB7BF
:102E70006C0159018B017B01E40EF51E0E151F0537
:102E800061F1F60180809180F80161918F01698381
:102E9000C4016A830E9425BA6A81681779F0C40167
:102EA0000E942DBAC4010E9425BA9981891731F078
:102EB0002CDF87E193E01BDF81E010C041E050E0B0
:102EC000BE016F5F7F4FC501F2DEF6014081518187
:102ED0004F5F5F4F51834083D1CF80E00F900F90C1
:102EE000DF91CF911F910F91FF90EF90DF90CF90E6
:102EF000BF90AF909F908F9008958F929F92AF92C6
:102F0000BF92CF92DF92EF92FF920F93CF93DF9316
:102F10001F92CDB7DEB75C016B017A014901F50163
:102F2000808191810E9425BA8983002311F0F601E6
:102F3000808341E050E0BE016F5F7F4FC401B7DE88
:102F4000F501408151814F5F5F4F51834083FFEF17
:102F5000CF1ADF0A81E0E81AF10809F780E00F9044
:102F6000DF91CF910F91FF90EF90DF90CF90BF90C6
:102F7000AF909F908F900895CF93DF93CDB7DEB73A
:102F800060970FB6F894DEBF0FBECDBF9C01E62F51
:102F9000660FFF0BED51FE4FE4918E2F90E0FC0188
:102FA0003797EC30F10508F0B5C08827EA56FF4F97
:102FB0008F4F0C94D2B291E001C090E080E1FE010D
:102FC0003196DF01482F1D924A95E9F740EB50E01A
:102FD0005A83498341EB50E05C834B8343EB50E0E1
:102FE00058874F8344EB50E05A87498742E04F8728
:102FF000988B98C081E001C080E08F5F01C080E0C5
:1030000040E950E0D90111965C934E9341E950E0BC
:1030100013965C934E93129742E950E015965C9399
:103020004E93149748E950E017965C934E93169789
:103030004AE950E019965C934E9318974CE950E09A
:103040001B965C934E931A9746E950E01D965C934D
:103050004E931C9793E058C081E001C080E08F5FE1
:1030600001C080E040EA50E0F9015183408341EA29
:1030700050E05383428342EA50E05583448348EA58
:1030800050E0578346834AEA50E0518740874CEA34
:1030900050E05387428746EA50E05587448794E0E2
:1030A0009687878744C081E001C080E08F5F01C0C0
:1030B00080E040E251E0D90111965C934E9341E2E9
:1030C00051E013965C934E93129742E251E01596AD
:1030D0005C934E93149748E251E017965C934E939D
:1030E00016974AE251E019965C934E9318974CE27A
:1030F00051E01B965C934E931A9746E251E01D9661
:103100005C934E931C9795E01E969C931E971F967A
:103110008C930DC080E1FE013196DF01482F1D9296
:103120004A95E9F7D90101900D928A95E1F7C90115
:1031300060960FB6F894DEBF0FBECDBFDF91CF9182
:1031400008952F923F924F925F926F927F928F924B
:103150009F92AF92BF92CF92DF92EF92FF920F9326
:103160001F93CF93DF93CDB7DEB7AE970FB6F8942A
:10317000DEBF0FBECDBF1B01682FCE014196FCDE26
:103180004B895C895EA34DA35F8D5AA3552309F437
:1031900013C1523021F0CC24CA94DC2C03C0CC24BF
:1031A000CA94D12C2114310409F4DBC09601322FCA
:1031B0002227330F330F330F40E050E060E074E21A
:1031C00084EF90E00E94B6B2C90101969CA38BA344
:1031D00080E1EFE6F2E0DE01119601900D928A9512
:1031E000E1F7FE013196F8A7EFA301E011E019A283
:1031F000AA24AA94B12C412C84E2582E84EF682E84
:10320000712CFAA1F230F1F0033009F49FC00530BF
:1032100009F49CC0EFA1F8A582819381289E9001BA
:10322000299E300D389E300D112440E050E0C3013E
:10323000B2010E94B6B2C901019736952795009751
:1032400029F40AC02FEF30E08FEF90E07C01C81620
:10325000D90628F4760103C0EE24E394F12C21155D
:10326000310531F04901C216D30628F4460103C0E6
:1032700088248394912CEFA1F8A50280F381E02D9E
:10328000FEA7EDA7C70101968E9F90018F9F300D7D
:103290009E9F300D112440E050E0C301B2010E9416
:1032A000B6B229A73AA74BA75CA78DA59EA5880F04
:1032B000991F889D9001899D300D989D300D112496
:1032C00040E050E0C301B2010E94B6B28BA19CA1C4
:1032D0008219930997FF03C091958195910969A57A
:1032E0007AA56219730977FF03C071956195710919
:1032F000F901E219F309F7FF03C0F195E195F1092E
:103300006817790774F4E617F7075CF0FAA1F23052
:10331000A1F449A55AA55CA34BA309A3570113E047
:1033200015C0E817F90794F48AA13CA32BA309A3BD
:103330005401823051F411E009C0E9A5FAA5FCA3BB
:10334000EBA309A357011EE001C01AE00F5F4FA1D4
:1033500058A54E5F5F4F58A74FA3083009F051CFD3
:1033600005C011E019A2AA24AA94B12CE989FA890E
:103370008081912F93708C7F892B8083EDA1FEA19A
:103380002081812F90E0959587959595879543E0CD
:10339000880F991F4A95E1F7122F177E812B8083A2
:1033A0008081887FC9A0C82AC082FAA1F23021F0AA
:1033B000ED8DFE8DB182A082AE960FB6F894DEBF81
:1033C0000FBECDBFDF91CF911F910F91FF90EF9076
:1033D000DF90CF90BF90AF909F908F907F906F9035
:1033E0005F904F903F902F9008954F925F926F9211
:1033F0007F92AF92BF92CF92DF92EF92FF920F93A4
:103400001F93CF93DF93CDB7DEB760970FB6F894D5
:10341000DEBF0FBECDBF6115710511F4622F05C06F
:1034200064177507B9F461E0622760960FB6F894E7
:10343000DEBF0FBECDBFDF91CF911F910F91FF90E7
:10344000EF90DF90CF90BF90AF907F906F905F90A4
:103450004F90F5C9D22E8A017B01682FCE010196CB
:103460008BDD5F85E889552309F44BC0A981BA81BA
:103470004C91F0E083E090E0BC016E1B7F0B660F87
:10348000771F2D2D30E02E5F3F4F062E01C0220FFB
:103490000A94EAF701C0880F6A95EAF780958423B9
:1034A000282B2C93523029F0AD85BE85CD90DC9031
:1034B00003C0CC24CA94D12C3396EE0FFF1F81E0B9
:1034C00090E08C0F9D1FE80FF91FA080B180B7011D
:1034D00080E090E00E94F6AF2B013C01C601B801EC
:1034E0000E946DB280E090E00E94F6AF9B01AC01BB
:1034F000C301B2010E9494B10E94C5AFF50171836E
:10350000608360960FB6F894DEBF0FBECDBFDF912B
:10351000CF911F910F91FF90EF90DF90CF90BF90D0
:10352000AF907F906F905F904F90089598E288E100
:103530000FB6F894A895809360000FBE909360003A
:1035400008951F920F920FB60F9211240BB60F928F
:103550000F931F932F933F934F935F936F937F939B
:103560008F939F93AF93BF93CF93DF93EF93FF938B
:103570000091CD03D091CC0311E01D0F1F77C091B6
:10358000C6009091A803492F092E000C550B660B1D
:10359000770B4C30510508F046C0FA018827EE55EC
:1035A000FF4F8F4F0C94D2B2CD3441F0CE34B9F4EA
:1035B00081E005C0CA3330F0CD3471F582E08093EC
:1035C000A8034AC0C03308F047C0C03209F444C061
:1035D000CD3211F541C0C13329F0C43329F0C032D6
:1035E000D9F43AC083E0EBCF88E0E9CFC03321F0D3
:1035F000C13391F486E0E3CF84E0E1CFC83361F4D6
:1036000085E0DDCFC23341F487E0D9CFC13321F467
:1036100089E0D5CFC03311F08BE0D1CF8AE0CFCF96
:10362000CA30D1F417C0CA30B9F480915704882346
:1036300089F0973049F09A3059F0953059F410924A
:103640006D021092E20E06C081E08093580402C021
:103650000E94C8AC1092A803101731F0ED2FF0E0D3
:10366000E453FC4FC283D12FD093CC03FF91EF9151
:10367000DF91CF91BF91AF919F918F917F916F918A
:103680005F914F913F912F911F910F910F900BBE22
:103690000F900FBE0F901F9018951F920F920FB6AC
:1036A0000F9211240BB60F922F938F939F93EF934A
:1036B000FF938091AB032091AA03281791F0E82F84
:1036C000F0E0E655FC4F92818F5F8F719093C600BA
:1036D0008093AB039091C00090649093C000281336
:1036E00005C08091C1008F7D8093C100FF91EF9153
:1036F0009F918F912F910F900BBE0F900FBE0F9047
:103700001F9018959B01AC011092C000211581EE0D
:10371000380741055105C1F08091C0008260809357
:10372000C00060E079E08DE390E00E94B6B2CA018B
:10373000B901615071098109910922E030E040E04E
:1037400050E00E94B6B202C020E130E03093C500E4
:103750002093C4008091C10080618093C10080915A
:10376000C10088608093C1008091C100806880930F
:10377000C1008091C1008F7D8093C1001092A90388
:1037800008958091CC039091CD03891759F0E92FCA
:10379000F0E0E453FC4F82819F5F9F779093CD03CD
:1037A00090E008958FEF9FEF0895ECECF3E08081B7
:1037B00081830895ECECF3E080819181891B8F7700
:1037C000089591E09093A9039091C10095FD04C0E4
:1037D0009091C00095FD40C02091AA032F5F2F71EA
:1037E0000FB607FC34C09091AB03291322C090910F
:1037F000C00095FF1DC09091AB034091AA034917EB
:1038000091F0E92FF0E0E655FC4F32819F5F9F7108
:103810003093C6009093AB033091C0003064309376
:10382000C000491305C09091C1009F7D9093C100D5
:10383000DACFE091AA03F0E0E655FC4F82832093B3
:10384000AA038091C10080628093C1000895909185
:10385000AB032913EECFFBCF8093C6008091C0004D
:1038600080648093C00008958DE0ABDF8AE0A9CF2B
:10387000CF93DF93EC018991882311F0A2DFFBCF76
:10388000DF91CF91F1CF8F929F92AF92BF92EF9243
:10389000FF921F93CF93DF93CDB7DEB7A0970FB6FC
:1038A000F894DEBF0FBECDBF61157105810591058E
:1038B00079F110E0842E912CA12CB12CEE24E3940C
:1038C000F12CEC0EFD1EE10EF11C17FDFA94A50182
:1038D00094010E9494B2F7016083B901CA011F5F8D
:1038E000611571058105910549F7115010F1E1E06D
:1038F000F0E0EC0FFD1FE10FF11D17FDFA9580813F
:103900008A3010F097E301C090E3890F5ADFEDCFC2
:1039100080E3A0960FB6F894DEBF0FBECDBFDF9157
:10392000CF911F91FF90EF90BF90AF909F908F909D
:1039300048CFA0960FB6F894DEBF0FBECDBFDF9183
:10394000CF911F91FF90EF90BF90AF909F908F907D
:103950000895CF92DF92EF92FF926B017C0197FF67
:103960000AC08DE22EDFF094E094D094C094C11C84
:10397000D11CE11CF11C4AE0C701B601FF90EF9099
:10398000DF90CF9080CF4115510511F4862F19CFCC
:103990004A30510509F4DDCF76CFAB01682F880F8F
:1039A000770B880B990BEFCFAB01BC01990F880BFC
:1039B000990BE9CFAB01BC01990F880B990BE3DFA1
:1039C00053CFE1DF51CF4115510511F4862FF9CEC8
:1039D0005ACFAB01BC0180E090E0F5CF8F929F926F
:1039E000AF92BF92CF92DF92EF92FF92CF936B0193
:1039F0007C01B42E20E030E0A9010E9456AF87FF81
:103A000006C08DE2DEDEF7FAF094F7F8F094C0E03D
:103A100060E070E080E09FE3CB1541F02DEC3CECE2
:103A20004CEC5DE30E9494B1CF5FF6CF9B01AC01FB
:103A3000C701B6010E947DAE6B017C010E94CAAF36
:103A40004B015C014AE01FDFCC2379F1C501B401D1
:103A50000E94F6AF9B01AC01C701B6010E947CAE8B
:103A60006B017C018EE2ADDE20E030E040E251E40B
:103A7000C701B6010E9494B14B015C010E94C5AF21
:103A80006B01770FEE08FF08C701B60162DFC701BF
:103A9000B6010E94F8AF9B01AC01C501B4010E94C0
:103AA0007CAE6B017C01C150F9F6CF91FF90EF9095
:103AB000DF90CF90BF90AF909F908F9008958ECF62
:103AC000CF92DF92EF92FF920F931F930E94EF111C
:103AD00000915204109153042091540430915504E4
:103AE0006B017C01C01AD10AE20AF30AF7FC52C04A
:103AF0008B019C010C53164F2F4F3F4F00935204E4
:103B0000109353042093540430935504079B39C0F9
:103B1000069B37C0059B35C02091DC04211131C0C4
:103B2000049B2FC000914E0410914F04209150042B
:103B300030915104011511052105310571F0DC01A9
:103B4000CB01801B910BA20BB30B80569A4EA1099F
:103B5000B109B7FF02C068E701C060E06093560496
:103B6000809102016111809588708093000170E05E
:103B700086E01F910F91FF90EF90DF90CF900C9413
:103B8000C61260934E0470934F0480935004909338
:103B90005104C8CF1F910F91FF90EF90DF90CF900D
:103BA000089581E080935704089590913006891715
:103BB000D1F00E94C75E80913006882359F04AE513
:103BC00052E066E572E082E592E00E948A5D109222
:103BD000300607C081E08093300682E592E00E94C3
:103BE000F85D0C949B52089580E0DFDF8CE096E056
:103BF0000C9434A82F923F924F925F926F927F92D3
:103C00008F929F92AF92BF92CF92DF92EF92FF92EC
:103C10000F931F93CF93DF93CDB7DEB7A2970FB665
:103C2000F894DEBF0FBECDBF80916504102F18271A
:103C3000DB018D909D90AD90BC9089288A288B28BF
:103C400009F41E7FFA014081518162817381452B05
:103C5000462B472B09F41D7FD9014D915D916D9144
:103C60007C91452B462B472B09F41B7F81278093A2
:103C7000650460917604662309F452C1FC8AEB8ADC
:103C800070E080E090E00E94F6AF20E030E04FE787
:103C900053E40E945DAF69837A838B839C83809118
:103CA000100290911102A0911202B09113028D871F
:103CB0009E87AF87B88BA7E7B4E0BA8BA98BFE824B
:103CC000ED82E9E5F4E0FAA3E9A381E696E09C87BA
:103CD0008B87212C312CC12CD12C7601802F90E0A8
:103CE000A0E0B0E0898F9A8FAB8FBC8F812F90E0DE
:103CF000A0E0B0E08D8F9E8FAF8FB8A389819A81AD
:103D0000AB81BC81B0588F839887A987BA87A9896E
:103D1000BA898D909D90AD90BD90BA8BA98B20E013
:103D200030E0A901C501B4010E9456AF882309F40F
:103D3000E0C0898D9A8DAB8DBC8D022C04C0B695E8
:103D4000A795979587950A94D2F72C013D01E1E05C
:103D50004E225524662477248D8D9E8DAF8DB8A17B
:103D6000022C04C0B695A795979587950A94D2F72B
:103D700080FF3BC0A9A1BAA16D917D918D919C91CD
:103D80000E94F8AF6D8B7E8B8F8B988F41145104FE
:103D90006104710429F0BF81A885E9851A8504C0F2
:103DA000B981AA81EB811C81A50194016B2F7A2F27
:103DB0008E2F912F0E9494B1EB85FC852489358943
:103DC000468957890E9494B19B01AC016D897E8917
:103DD0008F89988D0E947DAE0E94C5AFA9A1BAA11E
:103DE0006D937D938D939C931397E9A1FAA18080A5
:103DF0009180A280B38081149104A104B10409F4DC
:103E000078C020E030E0A9016D857E858F85988996
:103E10000E9456AF882309F447C0D501C401882702
:103E2000B7FD83959927AA27BB274816590609F09D
:103E300060C020E030E0A901C701B6010E9456AF82
:103E400081111EC02D853E854F855889AB89BC895F
:103E50001D966D917D918D919C9150970E945DAFC3
:103E60006B017C0120E030E040E85FE30E9459B143
:103E7000181634F4C12CD12C80E8E82E8FE3F82EEC
:103E8000C501B4010E94F8AF9B01AC01C701B601A6
:103E90000E9494B10E9443AF0E94C5AF61157105A5
:103EA0008105910519F425C0C501B4012B013C0120
:103EB00097FF07C0442455243201461A570A680A5E
:103EC000790AED81FE81058916892789308D400E9A
:103ED000511E621E731E458A568A678A708E861A24
:103EE000970AA80AB90AE9A1FAA180829182A2825E
:103EF000B382FFEF2F1A3F0A8D819E8104969E8325
:103F00008D83A9A1BAA11496BAA3A9A3EB85FC85B8
:103F10003496FC87EB87F3E02F16310409F0F7CED7
:103F2000A2960FB6F894DEBF0FBECDBFDF91CF9142
:103F30001F910F91FF90EF90DF90CF90BF90AF90C7
:103F40009F908F907F906F905F904F903F902F90B9
:103F500008954F925F926F927F928F929F92AF924D
:103F6000BF92CF92DF92EF92FF92CF93DF93CDB7C4
:103F7000DEB728970FB6F894DEBF0FBECDBF809195
:103F800069048F3F09F45FC080905A0290905B02F1
:103F9000A0905C02B0905D02412C512C80E8682E0C
:103FA0008FE3782EC0905A02D0905B02E0905C02C2
:103FB000F0905D0220E030E040E05FE3C501B40135
:103FC0000E947DAE9B01AC01C701B6010E9456AFB5
:103FD00087FF1AC01C9918C049825A826B827C8262
:103FE0002AE037ED43EA5BE3C701B6010E947DAEEC
:103FF0006D837E838F839887BE016F5F7F4FCE0175
:1040000005960E943454CECFA5019401C701B60194
:104010000E947CAE9B01AC016091720470917304AC
:1040200080917404909175040E947DAE6093720437
:104030007093730480937404909375048091690461
:104040008F5F8093690428960FB6F894DEBF0FBE89
:10405000CDBFDF91CF91FF90EF90DF90CF90BF90D9
:10406000AF909F908F907F906F905F904F9008954A
:104070000F931F93CF93DF931F92CDB7DEB78C01C1
:1040800081E493E069830E947716C8010E94771645
:104090006981662339F08AE00F90DF91CF911F91FB
:1040A0000F918FCB0F90DF91CF911F910F910895BA
:1040B00061E088E393E0DCCF61E081E393E0D8CF77
:1040C000EF92FF920F931F93CF93DF931F92CDB781
:1040D000DEB78C017B0180E2498373DB49814F3F6E
:1040E00011F084E501C082E46CDB8AE36ADBF8014D
:1040F000608171818281938142E050E0E0DCF701D0
:10410000408151816281738183E593E00E94C216F0
:1041100062E070E080E090E00F90DF91CF911F911E
:104120000F91FF90EF900C942012FB01DC0112968E
:104130004D915D916D917C911597411551056105EA
:10414000710599F080819181A281B381841B950BC7
:10415000A60BB70B80959095A095B0958827B7FDD5
:1041600083959927AA27BB27089580E00895811198
:1041700009C0CB016F3F710519F010F08FEF90E08F
:104180008093EF04089587FF03C08091DC0407C08B
:1041900097E18902F0011124E051FB4F828590E004
:1041A00008954F925F926F927F928F929F92AF92FB
:1041B000BF92CF92DF92EF92FF92CF93DF9300D026
:1041C0001F92CDB7DEB7E090F804F090F90480902C
:1041D000F4049090F504A090F604B090F70420ED5C
:1041E0003CEC4CE45DE36091030570910405809123
:1041F0000505909106050E9494B12B013C01209188
:10420000B4043091B5044091B6045091B704C5018F
:10421000B4010E947CAE9B01AC01C301B2010E94BB
:1042200094B12B013C0123E333E343E75FE3609167
:10423000B0047091B1048091B2049091B3040E94D3
:1042400094B19B01AC01C301B2010E947DAE6983B0
:104250007A838B839C836093B0047093B1048093C2
:10426000B2049093B3048092B4049092B504A092E7
:10427000B604B092B704E114F104A1F0B701FF0C49
:10428000880B990B0E94F8AFA50194010E947CAEA7
:104290006B017C0120E030E040E251EC0E9456AF1F
:1042A00087FF07C081E08093A704412C512C320185
:1042B000C1C020E030E040E251E4C701B6010E94F5
:1042C00059B1181654F481E08093A704412C512C65
:1042D0002FE7622E23E4722EADC08091A7048823BD
:1042E00051F01092A3041092A4041092A50410920D
:1042F000A6041092A7042091A3043091A404409135
:10430000A5045091A604C701B6010E947DAE4B01E1
:104310005C016093A3047093A4048093A50490931C
:10432000A6042091FB043091FC044091FD045091BF
:10433000FE04C701B6010E9494B12B013C016093B9
:10434000A8047093A9048093AA049093AB042091CD
:10435000FF04309100054091010550910205C5010F
:10436000B4010E9494B19B01AC016093AC047093C2
:10437000AD048093AE049093AF04C301B2010E94D8
:104380007DAE29813A814B815C810E947CAE2B01FC
:104390003C0120E030E04FE753E40E9459B120E0B7
:1043A00030E0A9011816DCF4C701B6010E9459B12A
:1043B0001816B4F5A7019601C501B4010E947CAEA0
:1043C0006093A3047093A4048093A5049093A6041F
:1043D000412C512C9FE7692E93E4792E2BC0C30109
:1043E000B2010E9456AF87FF25C020E030E0A9014E
:1043F000C701B6010E9456AF87FF19C0A7019601F9
:10440000C501B4010E947CAE6093A3047093A40420
:104410008093A5049093A604412C512C32010AC02C
:10442000412C512C8FE7682E83E4782E03C0412C59
:10443000512C3201C301B2010F900F900F900F90D9
:10444000DF91CF91FF90EF90DF90CF90BF90AF9032
:104450009F908F907F906F905F904F9008954F92B4
:104460005F926F927F928F929F92AF92BF92CF9204
:10447000DF92EF92FF92CF93DF93CDB7DEB72C9709
:104480000FB6F894DEBF0FBECDBF8091D6049091D9
:10449000D704A091D804B091D90489839A83AB83BF
:1044A000BC836091DA047091DB04072E000C880B4A
:1044B000990B0E94F8AF29813A814B815C810E945F
:1044C0007CAE6B017C0120919F043091A00440914F
:1044D000A1045091A2040E947DAE4B015C01609347
:1044E0009F047093A0048093A1049093A204209150
:1044F000DD043091DE044091DF045091E004C701F7
:10450000B6010E9494B16D837E838F8398876093F8
:10451000930470939404809395049093960420914F
:10452000E1043091E2044091E3045091E404C501B8
:10453000B4010E9494B169877A878B879C876093C6
:104540009704709398048093990490939A0420EDB3
:104550003CEC4CE45DE36091E5047091E6048091ED
:10456000E7049091E8040E9494B12B013C01209152
:104570008F0430919004409191045091920469818C
:104580007A818B819C810E947CAE9B01AC01C3012E
:10459000B2010E9494B12B013C0123E333E343E7D2
:1045A0005FE360919B0470919C0480919D049091C5
:1045B0009E040E9494B19B01AC01C301B2010E9410
:1045C0007DAE2B013C0160939B0470939C0480930F
:1045D0009D0490939E0489819A81AB81BC818093D4
:1045E0008F0490939004A0939104B0939204298532
:1045F0003A854B855C856D817E818F8198850E948F
:104600007DAEA30192010E947CAE2B013C0120E013
:1046100030E04FE753E40E9459B120E030E0A901B7
:104620001816DCF4C701B6010E9459B11816B4F58A
:10463000A7019601C501B4010E947CAE60939F045E
:104640007093A0048093A1049093A204412C512C58
:104650009FE7692E93E4792E2BC0C301B2010E941B
:1046600056AF87FF25C020E030E0A901C701B601A1
:104670000E9456AF87FF19C0A7019601C501B4017A
:104680000E947CAE60939F047093A0048093A10469
:104690009093A204412C512C32010AC0412C512C80
:1046A0008FE7682E83E4782E03C0412C512C320111
:1046B000C301B2012C960FB6F894DEBF0FBECDBF7A
:1046C000DF91CF91FF90EF90DF90CF90BF90AF90B0
:1046D0009F908F907F906F905F904F9008954F9232
:1046E0005F926F927F928F929F92AF92BF92CF9282
:1046F000DF92EF92FF920F931F93CF93DF933C01D2
:10470000C62F662399F00E9488166AE070E08C2F0D
:1047100090E04AD98AE993E00E94771680E090E021
:104720000E940DAD60E070E0CB0188C0B0E2A0E077
:104730006A2F70E0AB014B0F511D55954795411500
:10474000510559F4E7E8F7E065917491072E000CE4
:10475000880B990B0E94F8AF71C04A1711F04B13E8
:104760000BC0E3E0F8E065917491072E000C880B14
:10477000990B0E94F8AF62C0CA010197880F991F78
:10478000880F991FFC01EB57F84F059114919A017E
:10479000220F331F220F331FF901EB57F84FC5913A
:1047A000D4916016710614F4B42FC4CFA42FC6158B
:1047B000D7050CF4BDCF8957984FFC01E590F490D4
:1047C000F901E957F84FC590D490B7010F2C000CB0
:1047D000880B990B0E94F8AF4B015C01B301601B81
:1047E000710B072E000C880B990B0E94F8AF2B0160
:1047F0003C01B6016E197F09072E000C880B990B3E
:104800000E94F8AF9B01AC01C301B2010E9494B1B8
:104810006B017C01C01BD10BBE01DD0F880B990B16
:104820000E94F8AF9B01AC01C701B6010E945DAFC9
:104830009B01AC01C501B4010E947DAEDF91CF9117
:104840001F910F91FF90EF90DF90CF90BF90AF90AE
:104850009F908F907F906F905F904F9008954F92B0
:104860005F926F927F928F929F92AF92BF92CF9200
:10487000DF92EF92FF920F931F93CF93DF933C0150
:10488000BAE3A0E06A2F70E0AB014B0F511D5595C4
:1048900047954115510559F4EFE9F6E0659174919A
:1048A000072E000C880B990B0E94F8AF71C04A17B5
:1048B00011F04B130BC0E3E8F7E065917491072EFC
:1048C000000C880B990B0E94F8AF62C0CA010197D7
:1048D000880F991F880F991FFC01E356F94F059126
:1048E00014919A01220F331F220F331FF901E3564F
:1048F000F94FC591D4916016710614F4B42FC4CF4A
:10490000A42FC615D7050CF4BDCF8156994FFC01D5
:10491000E590F490F901E156F94FC590D490B701B4
:104920000F2C000C880B990B0E94F8AF4B015C0117
:10493000B301601B710B072E000C880B990B0E94B2
:10494000F8AF2B013C01B6016E197F09072E000C50
:10495000880B990B0E94F8AF9B01AC01C301B20117
:104960000E9494B16B017C01C01BD10BBE01DD0F15
:10497000880B990B0E94F8AF9B01AC01C701B601EF
:104980000E945DAF9B01AC01C501B4010E947DAEE8
:10499000DF91CF911F910F91FF90EF90DF90CF901B
:1049A000BF90AF909F908F907F906F905F904F904F
:1049B0000895CF93DF93C0EFD4E060E08A819B81BC
:1049C0008EDE6C837D838E839F83C2EDD4E08A81EB
:1049D0009B8145DF6C837D838E839F83A895109296
:1049E000C804DF91CF9108956D9A75988091010167
:1049F00080618093010180910201807180930001A8
:104A0000809101018860809301018091020188708A
:104A1000809300019D9AA598809101018062809306
:104A200001016AE770E088E00E94A118809101010D
:104A30008860809301016AE770E086E00E94A11817
:104A400087ED80937A0010927E0010927D00809115
:104A50007E00816080937E0080917E0084608093E0
:104A60007E0080E888BD80916E00846080936E0037
:104A70006AEF70E080E090E00E94201285E090E014
:104A800090931C0280931B0260E08091170290912A
:104A9000180225DE20E030E040EA50E40E9456AFE4
:104AA00087FF0AC080911702909118024097909357
:104AB000180280931702E8CF81E391E090931E02E1
:104AC00080931D0260E08091190290911A0207DE26
:104AD00020E030E848E953E40E9459B1181654F434
:104AE0008091190290911A02409690931A02809335
:104AF0001902E8CF8091210290912202B0DE20E0DD
:104B000030E040EA50E40E9456AF87FF0AC080912F
:104B100021029091220240979093220280932102D9
:104B2000E9CF8091D0049091D10499DE20E030E06B
:104B300046E153E40E9459B1181654F48091D00410
:104B40009091D10440969093D1048093D004E9CF02
:104B50000895CF92DF92EF92FF928091F8049091A6
:104B6000F9040097B9F0C090F404D090F504E090F7
:104B7000F604F090F7040D97BC01990F880B990B80
:104B80000E94F8AF9B01AC01C701B6010E9456AF6D
:104B900087FD09C01092EB041092EC041092ED0412
:104BA0001092EE041EC020E030E040E050E4C70167
:104BB000B6010E947DAE0E94CAAF7093EA04609372
:104BC000E9040E94EF11DC01CB01805E914BAF4FF5
:104BD000BF4F8093EB049093EC04A093ED04B0934B
:104BE000EE04FF90EF90DF90CF900895CF92DF9288
:104BF000EF92FF928091DA049091DB040097B9F074
:104C0000C090D604D090D704E090D804F090D90496
:104C10000897BC01990F880B990B0E94F8AF9B0174
:104C2000AC01C701B6010E9456AF87FD09C01092C2
:104C3000CC041092CD041092CE041092CF041EC06A
:104C400020E030E040E050E4C701B6010E947DAEB4
:104C50000E94CAAF7093CB046093CA040E94EF1104
:104C6000DC01CB01805A9541AF4FBF4F8093CC04FC
:104C70009093CD04A093CE04B093CF04FF90EF9017
:104C8000DF90CF90089580911D0290911E020F97A2
:104C90001816190614F480E090E09093F9048093BC
:104CA000F80480E056DF1092DB041092DA049EDFF5
:104CB00080911D0290911E020F971816190614F488
:104CC00080E090E09093F9048093F80480E041DF65
:104CD0001092FA0475981092DB041092DA04109284
:104CE000DC04A5980895EF92FF920F931F93CF9342
:104CF000C82F7B018A0180916E028823D1F00E9427
:104D00008816C7010E9477168CEB94E00E947716F4
:104D1000C7FD08C06AE070E08C2FCC0F990B0E9491
:104D2000D41C04C088EB94E00E9477168AE00E94AD
:104D3000E11B8091B80481110EC010926E0281E0D7
:104D40008093B804A0DFC801CF911F910F91FF900D
:104D5000EF900C940DADCF911F910F91FF90EF90BC
:104D600092CF8F3F19F043E954E002C047EA54E084
:104D700061E874E0B8CF8F3F19F04CE554E002C011
:104D800040E754E06AE474E0AECF2F923F924F9236
:104D90005F926F927F928F929F92BF92CF92DF929B
:104DA000EF92FF920F931F93CF93DF936C014B0110
:104DB000B22E180127FD04C0C22F220FDD0B02C046
:104DC000C1E0D0E0FA014080518062807380CC0F56
:104DD000DD1FCC0FDD1F8E0109571B4FA301920170
:104DE000F80160817181828193810E9456AF88238E
:104DF00091F0F801408251826282738211E020E0DA
:104E000030E0A901C301B2010E9459B118160CF09B
:104E100010E0F6011483F60184818230C9F08330FA
:104E200009F456C0813009F070C0FE01E957FB4F0C
:104E30002081318142815381F401608171818281BD
:104E400093810E9456AF87FD60C082E0F6018483A3
:104E5000C957DB4FB70180E090E00E94F6AF9B019D
:104E6000AC01688179818A819B810E947CAE9B0123
:104E7000AC01F40160817181828193810E9459B1FA
:104E800087FD15C00E94EF112B013C019101A8EE96
:104E9000B3E00E94DAB2DC01CB01840D951DA61DA2
:104EA000B71DF60180839183A283B3832EC00E9435
:104EB000EF11F6010081118122813381DC01CB01E8
:104EC000801B910BA20BB30BB7FD1FC083E0848343
:104ED000FFEFBF1619F04FE653E002C046E853E07B
:104EE0006FE573E08B2DDF91CF911F910F91FF90B4
:104EF000EF90DF90CF90BF909F908F907F906F90BA
:104F00005F904F903F902F90EECEDF91CF911F9109
:104F10000F91FF90EF90DF90CF90BF909F908F9078
:104F20007F906F905F904F903F902F9008958F9259
:104F30009F92AF92BF92CF92DF92EF92FF920F9328
:104F40001F93CF93DF93CDB7DEB728970FB6F894B2
:104F5000DEBF0FBECDBF80915804811117C0809174
:104F6000C804811118C028960FB6F894DEBF0FBE92
:104F7000CDBFDF91CF911F910F91FF90EF90DF9008
:104F8000CF90BF90AF909F908F90089580E090E079
:104F90000E940DADE4CF0DDD0E94EF114B015C01CD
:104FA0006D837E838F83988760911D0270911E02AE
:104FB000072E000C880B990B0E94F8AF9B01AC01E7
:104FC0006091F4047091F5048091F6049091F704D7
:104FD0000E9459B1181634F443E354E063E274E0DC
:104FE00080E081DE6091F8047091F904072E000CD6
:104FF000880B990B0E94F8AF69837A838B839C831B
:105000003EE1E32EF12C0FE010E020E0AE014F5F17
:105010005F4F64EF74E083EC94E0B7DEC090F4047B
:10502000D090F504E090F604F090F70480911B0214
:1050300090911C02BC01990F880B990B0E94F8AF4C
:105040009B01AC01C701B6010E9459B11816CCF4FE
:1050500060911D0270911E02072E000C880B990BA7
:105060000E94F8AF9B01AC01C701B6010E9456AF88
:1050700087FF07C080E095D80E94C5AF75956795FA
:1050800001C060E06093FA048091EB049091EC041D
:10509000A091ED04B091EE040097A105B10511F1C6
:1050A000881A990AAA0ABB0AB7FC1CC06091E904D5
:1050B0007091EA0480E090E00E94F6AF9B01AC01A1
:1050C0006091F4047091F5048091F6049091F704D6
:1050D0000E9456AF87FF85C04DE054E06EEF73E04D
:1050E00080E001DE20E030E046E153E46091D60448
:1050F0007091D7048091D8049091D9040E9459B13D
:1051000018160CF465C0BE016B5F7F4F8AEC94E00B
:105110000CD88823D9F06091CA047091CB0480E048
:1051200090E00E94F6AF2091D6043091D7044091D0
:10513000D8045091D9040E9459B118160CF04FC0F0
:1051400047EC53E068EB73E08FEFCDDD6091DA045C
:105150007091DB04072E000C880B990B0E94F8AFAE
:1051600069837A838B839C839AE0E92EF12C0FE08C
:1051700010E02FEFAE014F5F5F4F66ED74E08EEBF6
:1051800094E003DE8090D6049090D704A090D804D9
:10519000B090D90420E030E040EA50E4C501B40109
:1051A0000E9459B187FD0AC020E030E046E153E497
:1051B000C501B4010E9456AF181624F460E0609354
:1051C000DC04D1CE4CD90E94C5AF75956795F7CF59
:1051D0004AEE53E06AED73E08FEF85DD94CF06DD94
:1051E000B5CF80E0B6DC7ECFE0EFF4E08081918146
:1051F00093838283E2EDF4E08081918193838283C3
:1052000081E08093C80408951F93CF93DF9380912A
:10521000C804811101C0E8DF1092F1041092F0047B
:105220001092D3041092D204C091F204D091F304EE
:10523000D195C195D1098091F8049091F90411E0BC
:10524000181619062CF08091FA04811101C010E0A3
:105250008091190290911A029195819591098C176C
:105260009D0714F480E07DDD112361F08091170229
:1052700090911802919581959109C817D90714F456
:1052800080E079DD8091DA049091DB04C1E01816AA
:1052900019062CF08091DC04811101C0C0E020913E
:1052A000D4043091D5048091D0049091D104821718
:1052B000930714F08FEF55DDCC2381F0209121026C
:1052C000309122028091D4049091D50482179307E3
:1052D0002CF08FEFDF91CF911F914DCDDF91CF91CA
:1052E0001F9108950F930FB70F9300916E000B7FDE
:1052F00000936E0078940F930BB70F930CB70F9237
:105300001F922F933F934F935F936F937F938F934E
:105310009F93AF93BF93EF93FF931124C7D0FF9157
:10532000EF91BF91AF919F918F917F916F915F911D
:105330004F913F912F911F900F900CBF0F910BBF7A
:105340000F910460F89400936E000F910FBF0F91BE
:105350001895CF93809116028F3790F08F579091C8
:10536000FA0490938604992311F0759A01C07598F8
:105370009091DC0490938504992359F0A59A0AC072
:1053800090918604891708F0759890918504891783
:1053900008F0A598805F809316029091840481E0C4
:1053A0008927809384048091150285301CF4C1E024
:1053B000C80F01C0C0E08230A1F184F4882329F134
:1053C000813009F062C010927B0080E480937C0001
:1053D00080917A00806480937A0057C0843009F409
:1053E0003EC094F1853009F050C090918304911132
:1053F00002C080938304809183048150809383044E
:10540000882309F442C0C5E040C0809114028F5F38
:1054100080311CF48093140238C010921402F4DE20
:1054200034C080917A0086FD2DC0809178009091E3
:1054300079002091F0043091F104820F931F909332
:10544000F1048093F00421C010927B0082E48093E9
:105450007C0080917A00806480937A0016C08091ED
:105460007A0086FD11C0809178009091790020919A
:10547000D2043091D304820F931F9093D30480936E
:10548000D20403C0C2E001C0C4E0C09315020E9470
:1054900095348091AA069091AB06009729F0019768
:1054A0009093AB068093AA06CF91089552CFFF92B6
:1054B0000F931F93CF93DF93CDB7DEB728970FB627
:1054C000F894DEBF0FBECDBFF82E00EF14E0F80158
:1054D00060857185072E000C880B990B0E94F8AF30
:1054E00069837A838B839C83F80184819581A6816B
:1054F000B7818D839E83AF83B8874DEFBE016F5F09
:105500007F4FCE0105960E94602002ED14E0F80165
:1055100060857185072E000C880B990B0E94F8AFEF
:1055200069837A838B839C83F80184819581A6812A
:10553000B7818D839E83AF83B8874FEFBE016F5FC6
:105540007F4FCE0105960E9460208F2D0E94C320C0
:10555000BC018BE593E00E94A816F801628570E01B
:1055600086E593E00E94A81628960FB6F894DEBF51
:105570000FBECDBFDF91CF911F910F91FF90089586
:105580002F923F924F925F926F927F928F929F9253
:10559000AF92BF92CF92DF92EF92FF920F931F9341
:1055A000CF93DF93CDB7DEB7CD54D1090FB6F894C2
:1055B000DEBF0FBECDBF2E969FAF8EAF2E97162F9C
:1055C000742E26962FAF26970E94EF11688B798B49
:1055D0008A8B9B8B17FD04C0A4E1EA2EF12C03C03B
:1055E000FCE3EF2EF12C2E96AEADBFAD2E972D9194
:1055F0003D914D915C912FA738AB49AB5AAB17FD4C
:105600008FC4C12E012E000CDD08F60183E0EE0FE1
:10561000FF1F8A95E1F7E95EFD4F668177816F5044
:105620007109072E000C880B990B0E94F8AF9B01A3
:10563000AC016FA578A989A99AA90E9459B1181639
:10564000ECF482E796E0C35BDF4F0FB6F894DEBF61
:105650000FBECDBFDF91CF911F910F91FF90EF90C3
:10566000DF90CF90BF90AF909F908F907F906F9082
:105670005F904F903F902F900C9477168EE596E0B8
:105680000E94771600DB27E12C9DC0012D9D900D17
:105690001124FC01E051FB4F2FE7228780E090E0CE
:1056A000A0E5B1E423968CAF9DAFAEAFBFAF23971B
:1056B0009701A8EEB3E00E94DAB26BAF7CAF8DAF7A
:1056C0009EAF9B01AC0188899989AA89BB89280F63
:1056D000391F4A1F5B1F2BAB3CAB4DAB5EAB81E070
:1056E00080936D0288889988AA88BB888EA29FA221
:1056F000A8A6B9A6188E198E1A8E1B8E1C8A1D8A12
:105700001E8A1F8A1A821B821C821D821A8690E4BE
:105710009C8FACE1AD8FB6E4BE8F1F8E18A219A28C
:105720001AA21EA61FAA18AE19AE1AAE2FE730E0B5
:1057300040E050E02E833F8348875987EFE7CE2E25
:10574000D12CE12CF12C1AA61BA61CA61DA631E01B
:105750003BA31F861E86212C312C00E0198247E1D5
:105760001402C001112480519B4FDC011A9625962A
:10577000BFAFAEAF2597FC013496FDA3ECA3272D58
:10578000770C330B28963FAF2EAF289780916D0290
:10579000882309F48EC20E94EF112B013C018091F5
:1057A000C804882309F4F9C004D917FF0AC020905F
:1057B000D6043090D7040091D8043091D9043983AD
:1057C0000CC0ACA1BDA12C9011963C9011971296E3
:1057D0000C9112971396BC91B9839101402F598176
:1057E0006F8D78A189A19AA10E9456AF87FF05C04D
:1057F0002F8E38A209A3E981EAA39101402F598194
:105800006A857C8D8D8D9E8D0E9459B118162CF461
:105810002A863C8E0D8FF981FE8F2BA1222309F45D
:1058200063C02E96AEADBFAD2E972D913D914D919B
:105830005C91B101802F99810E9459B118160CF02A
:10584000ACC0A3019201281939094A095B092C96B9
:105850002CAF3DAF4EAF5FAF2C97DA01C90188582E
:105860009341A109B109B7FD98C0D701C6012E81A6
:105870003F8148855985821B930BA40BB50BB595C9
:10588000A7959795879517FF03C08093DC0405C003
:105890002596EEADFFAD259780832C962CAD3DADC2
:1058A0004EAD5FAD2C972AA73BA74CA75DA72E96C0
:1058B000AEADBFAD2E97BC91BF8F2E96EEADFFADB6
:1058C0002E97F181F8A32E96AEADBFAD2E9712960E
:1058D000BC91B9A32E96EEADFFAD2E97F381FAA33E
:1058E0004EA25FA268A679A62E96AEADBFAD2E974A
:1058F0002D913D914D915C91B101802F99810E9434
:1059000056AF87FF0BC3D301C2012EA13FA148A50B
:1059100059A5821B930BA40BB50BAC01BD014858D4
:1059200053416109710977FDF9C24E855F85452BA9
:1059300009F0DAC18E819F81A885B9858C0D9D1DE6
:10594000AE1DBF1DB595A7959795879517FFE0C22A
:105950008093DC042E853F852F5F3F4F3F872E8746
:105960002E96AEADBFAD2E97BC91BA872E96EEADFA
:10597000FFAD2E97F181FC8F2E96AEADBFAD2E9769
:105980001296BC91BD8F2E96EEADFFAD2E97F38192
:10599000FE8F5301420121E02BA320E030E040EADA
:1059A00051E42E96AEADBFAD2E976D917D918D9148
:1059B0009C910E947DAE9B01AC01B101802F998129
:1059C0000E9459B118162CF48AEE95E00E947716C1
:1059D00070C1D301C201288939894A895B89821B38
:1059E000930BA40BB50BB7FD8BC0812F17FD80E087
:1059F0005EDD8AE00E94E11BD301C2018053984F13
:105A0000AF4FBF4F888B998BAA8BBB8B9EA59111F3
:105A100055C02FA938AD49AD5AADB101802F99813C
:105A20000E9459B1181694F520E030E040E050E4AF
:105A3000B101802F99810E947DAE6FAB78AF89AFA5
:105A40009AAF2BAD3CAD4DAD5EAD240D351D461D61
:105A5000571D2BAB3CAB4DAB5EAB23962CAD3DAD98
:105A60004EAD5FAD23976FA578A989A99AA90E9429
:105A70007CAE9B01AC0181E08EA7B101802F9981A2
:105A80000E9459B11816E4F11EA63AC0D301C20112
:105A90002BA93CA94DA95EA9821B930BA40BB50BA6
:105AA000B7FD2EC01F3F19F041EC55E002C047ED95
:105AB00055E062EB75E0812F16D922C020E030E07E
:105AC00040EA51E42E96AEADBFAD2E976D917D911B
:105AD0008D919C910E947CAE9B01AC01B101802F05
:105AE00099810E9456AF87FF0BC01F3F19F047E80E
:105AF00055E002C04EE955E067E775E0812FF3D825
:105B0000D301C201880F991FAA1FBB1F2EA13FA15D
:105B100048A559A5821B930BA40BB50B88199909AD
:105B2000AA09BB0981389F44A241B10528F089E543
:105B300095E00E947716BDC04E855F8528968EAD94
:105B40009FAD2897841795070CF020CE4330510560
:105B50000CF41CCE8CEF94E00E94771617FD05C064
:105B600027EFE22E24E0F22E04C098EFE92E94E015
:105B7000F92E8AED94E00E947716C7010E947716ED
:105B80004A815B816C817D8183EF94E00E94C21623
:105B90008AE00E94E11B8AED94E00E947716C7011B
:105BA0000E9477164C895D896E897F898FEE94E01B
:105BB0000E94C2168AE00E94E11B8AED94E00E94D6
:105BC0007716C7010E947716488D598D6A8D7B8D97
:105BD0008BEE94E00E94C2168AE00E94E11B26969A
:105BE0009FAD2697992309F4BCC117FF31C02A81C4
:105BF0003B814C815D812093DD043093DE04409332
:105C0000DF045093E0042CEA35EC47E25EE36C8954
:105C10007D898E899F890E9494B16093E10470937D
:105C2000E2048093E3049093E4042CEA35EC47E229
:105C30005EE3688D798D8A8D9B8D0E945DAF609348
:105C4000E5047093E6048093E7049093E80489C127
:105C500047E1140290011124890100511B4F8A81F0
:105C60009B81AC81BD81F80183879487A587B68726
:105C70002CEA35EC47E25EE36C897D898E899F8949
:105C80000E9494B1D8011F966D937D938D939C9340
:105C900052972CEA35EC47E25EE3688D798D8A8D68
:105CA0009B8D0E945DAFF801638B748B858B968B07
:105CB00058C1C35BDF4F0FB6F894DEBF0FBECDBF38
:105CC000DF91CF911F910F91FF90EF90DF90CF90D8
:105CD000BF90AF909F908F907F906F905F904F900C
:105CE0003F902F900C9443268AA49BA4ACA4BDA4FF
:105CF000880E991EAA1EBB1E2AA53BA54CA55DA514
:105D0000281B390B4A0B5B0BCA01B9012E813F815D
:105D1000488559850E945EB2A50194010E94B6B2E1
:105D2000D701C601820F931FA41FB51F84319105AF
:105D3000A105B105FCF06C017D018C3E9105A1052A
:105D4000B1052CF06BEEC62ED12CE12CF12C40E8E5
:105D5000C416D104E104F104DCF08EEF90E0A0E081
:105D6000B0E08C199D09AE09BF098E839F83A88777
:105D7000B98712C054E1C52ED12CE12CF12C24E1BD
:105D800030E040E050E02E833F834887598704C0CD
:105D9000CE82DF82E886F986B701A60186E596E025
:105DA0000E94B2164E815F816885798581E596E013
:105DB0000E94B2164A855C8D6D8D7E8D8AE496E0D8
:105DC0000E94C2164F8D58A169A17AA183E496E082
:105DD0000E94C2164E855F85433051050CF4AACD52
:105DE0006E817F81888599850E94F8AF20E030E040
:105DF00040E850E40E9494B16A837B838C839D8346
:105E00002A853C8D4D8D5E8D6F8D78A189A19AA1DB
:105E10000E947CAE2BED3FE049E450E40E9494B137
:105E200020E030E040E05FE30E9494B19B01AC01D0
:105E30006A817B818C819D810E945DAF6A877B87AF
:105E40008C879D87C501B4010E94F8AF2FE632E12F
:105E500043E85AE30E9494B14B015C012AE939E915
:105E600049E15FE36A857B858C859D850E9494B1BD
:105E70006A837B838C839D839B01AC010E947DAEF2
:105E8000A50194010E945DAF6C8B7D8B8E8B9F8BE7
:105E9000A50194016A817B818C819D810E9494B1CE
:105EA00020E030E040E05EE30E9494B1688F798F9B
:105EB0008A8F9B8F4A855B856C857D858DE396E017
:105EC0000E94C216B501A40187E396E00E94C216A3
:105ED00087E296E00E9477164A815B816C817D8122
:105EE00081E296E00E94C2164C895D896E897F89A5
:105EF0008BE196E00E94C216488D598D6A8D7B8D8C
:105F000085E196E00E94C2168AE00E94E11B12CD54
:105F10002596EEADFFAD259780831CCD1BA23DCD10
:105F200020E030E047E053E46FA578A989A99AA959
:105F30000E9459B118160CF484CB8EE596E00E94AD
:105F400077160E9443268FE78093DC0420E030E040
:105F500040E051E423962CAF3DAF4EAF5FAF2397A7
:105F6000A7CBC35BDF4F0FB6F894DEBF0FBECDBF2C
:105F7000DF91CF911F910F91FF90EF90DF90CF9025
:105F8000BF90AF909F908F907F906F905F904F9059
:105F90003F902F900895CF92DF92EF92FF928091E1
:105FA000BD048823A1F10E94EF11C090B904D090E4
:105FB000BA04E090BB04F090BC04DC01CB018C1966
:105FC0009D09AE09BF09B7FD22C00E94EF116B0108
:105FD0007C012091BD0430E0A8EEB3E00E94DAB26B
:105FE000DC01CB018C0D9D1DAE1DBF1D8093B9043E
:105FF0009093BA04A093BB04B093BC0480E057DA3A
:106000008AE0FF90EF90DF90CF900C94E11BFF901F
:10601000EF90DF90CF9008952F923F924F925F9232
:106020006F927F928F929F92AF92BF92CF92DF92A8
:10603000EF92FF920F931F93CF93DF93CDB7DEB70D
:1060400064970FB6F894DEBF0FBECDBF898B6A8B05
:1060500081E080936D021A821B821C821D82198648
:106060001A861B861C8621E0288719821D863CE340
:106070003E874CE14F8756E4588BC12CD12C80E8E9
:10608000E82E9FEBF92E812C912C54016091F8049D
:106090007091F904072E000C880B990B0E94F8AF41
:1060A0006B8B7C8B182F092F9B01482F592FB60122
:1060B000C7010E9456AF882399F12091F4043091D2
:1060C000F5044091F6045091F7046B897C89812F87
:1060D000902F0E9456AF881F8827881F89838A893E
:1060E000882311F199819923F9F080916D026496CA
:1060F0000FB6F894DEBF0FBECDBFDF91CF911F91D9
:106100000F91FF90EF90DF90CF90BF90AF909F9056
:106110008F907F906F905F904F903F902F90089559
:10612000CB8ADC8A1E2D0F2D0E94EF116B017C01A2
:10613000DC01CB0129853A854B855C85821B930B5D
:10614000A40BB50BB7FD34C0D701C60188519C4FD5
:10615000AF4FBF4F89879A87AB87BC878989A7D9FB
:106160008FE493E00E94771681149104A104B10496
:10617000C9F0D501C40188519C4FAF4FBF4FBC013E
:10618000CD016C197D098E099F0928EE33E040E0AE
:1061900050E00E9494B2CA01B9014AE050E00E9466
:1061A000C31C03C08FE30E94E11B8AE00E94E11B35
:1061B0000E94E4AD0E94EF1160931A0C70931B0CC7
:1061C00080931C0C90931D0C2090F4043090F504E7
:1061D0009091F6049E83A091F704AF839101492F1B
:1061E0005A2F6B897C89812F902F0E947CAE2B01C6
:1061F0003C0120E030E0A9010E9459B187FF04C0B2
:10620000C301B201905802C0C301B20120E030E0E6
:1062100040E251E481149104A104B10481F40E948C
:1062200056AF87FF12C0B88546015701BB2369F0FE
:10623000E8EE8E0EE3E09E1EA11CB11C06C00E947B
:1062400059B1181614F446015701F981FF2391F151
:106250002A813B814C815D81211531054105510524
:1062600041F0D701C601821B930BA40BB50BB7FD00
:1062700021C091014E815F816D857E858F859889D2
:106280000E947CAE20E030E040EC5FE30E9456AF1D
:1062900087FD2BCFD701C601805A9541AF4FBF4F25
:1062A0008A839B83AC83BD832D863E869E819F8798
:1062B000AF81A88B80916D02882309F416CF8114D9
:1062C0009104A104B10431F41886CB88DC88E12E56
:1062D000F02EDCCEB8EECB1AB3E0DB0AE108F10811
:1062E000C818D908EA08FB08F7FCEECFFECE2F92BB
:1062F0003F924F925F926F927F928F929F92AF9256
:10630000BF92CF92DF92EF92FF920F931F93CF93A2
:10631000DF93CDB7DEB763970FB6F894DEBF0FBE3D
:10632000CDBF898B81E080936D021A821B821C8213
:106330001D8219861A861B861C8619821D862CE3EF
:106340002E873CE13F8746E4488BC12CD12C80E866
:10635000E82E9FEBF92E51E05887812C912C5401A7
:106360006091DA047091DB04072E000C880B990B06
:106370000E94F8AF6A8B7B8B182F092F9B01482F47
:10638000592FB601C7010E9456AF882399F1209179
:10639000D6043091D7044091D8045091D9046A8929
:1063A0007B89812F902F0E9456AF881F8827881FD6
:1063B00089838989882311F199819923F9F0809142
:1063C0006D0263960FB6F894DEBF0FBECDBFDF91AE
:1063D000CF911F910F91FF90EF90DF90CF90BF90E2
:1063E000AF909F908F907F906F905F904F903F9075
:1063F0002F900895CA8ADB8A1E2D0F2D0E94EF115F
:106400006B017C01DC01CB0129853A854B855C85DC
:10641000821B930BA40BB50BB7FD34C0D701C6018B
:1064200088519C4FAF4FBF4F89879A87AB87BC87F6
:1064300080E03DD88BE493E00E94771681149104AC
:10644000A104B104C9F0D501C40188519C4FAF4FDC
:10645000BF4FBC01CD016C197D098E099F0928EE43
:1064600033E040E050E00E9494B2CA01B9014AE032
:1064700050E00E94C31C03C08FE30E94E11B8AE02E
:106480000E94E11B0E94E4AD0E94EF1160931A0C80
:1064900070931B0C80931C0C90931D0C9091D60450
:1064A0009E83A091D704AF832090D8043090D90464
:1064B000292F3A2FA1016A897B89812F902F0E9471
:1064C0007CAE2B013C0120E030E0A9010E9459B1D3
:1064D00087FF04C0C301B201905802C0C301B201DA
:1064E00020E030E040EA50E481149104A104B104BA
:1064F00081F40E9456AF87FF12C0B885460157014C
:10650000BB2369F0E8EE8E0EE3E09E1EA11CB11CD9
:1065100006C00E9459B1181614F446015701F981BA
:10652000FF2391F12A813B814C815D812115310549
:106530004105510541F0D701C601821B930BA40B05
:10654000B50BB7FD21C02E813F81A1016D857E85F0
:106550008F8598890E947CAE20E030E040EC5FE3BC
:106560000E9456AF87FD2BCFD701C601805A9541B7
:10657000AF4FBF4F8A839B83AC83BD839E819D8732
:10658000AF81AE872F86388A80916D02882309F407
:1065900016CF81149104A104B10431F41886CA887D
:1065A000DB88E12EF02EDCCEB8EECB1AB3E0DB0AAE
:1065B000E108F108C818D908EA08FB08F7FCEECF93
:1065C000FECEE3ECF4E01082118212821382148278
:1065D0000895CF93C82F6115710519F0CB010E9462
:1065E000771684E198E00E947716C11103C085E018
:1065F00098E002C08AE098E00E9477168AE0CF9186
:106600000C94E11B80910F058093100508958091F3
:106610000E05882319F010920E05089580E798E082
:106620000C940DAD80911005811105C080910A0573
:10663000811101C0089562E070E080E090E00E9466
:10664000351680910B05882339F061E070E080E019
:1066500090E00E943516F5CF089580931005809341
:106660000F05E0CF26982E9A25982D9A24982C9ADB
:106670003F98479A0A98129A0998119A81E0EDCFAB
:1066800080931005CFCF80930A05CCCF80910E0563
:10669000882339F190910E0580910905981709F129
:1066A0000E94851681E698E00E94771680910E057B
:1066B00080FD1CC080910E0584FD18C080910E05E0
:1066C00081FD1EC080910E0585FD1AC080910E05CA
:1066D00082FD20C080910E0586FD1CC08AE00E94CC
:1066E000E11B80910E0580930905089580E00E94CA
:1066F0008E5EAB01BC018DE598E00E94C216DECF34
:1067000081E00E948E5EAB01BC0189E598E00E94A9
:10671000C216DCCF82E00E948E5EAB01BC0185E533
:1067200098E00E94C216DACFCF938BE398E00E94E4
:10673000771683B1C1E086FB882780F965E378E0AE
:106740008C2747DF86B180956FE278E0881F882725
:10675000881F3FDF83B185FB882780F969E278E0F5
:106760008C2737DF80B182FB882780F963E278E0ED
:106770008C272FDF83B1829581706DE178E08C27C3
:1067800028DF80B18695817067E178E08C27CF9112
:1067900020CF80910D051E9904C0816080930D0566
:1067A00003C08E7F80930D0580910D05379904C03D
:1067B000806180930D0503C08F7E80930D058091CD
:1067C0000D051D9904C0826080930D0503C08D7F67
:1067D00080930D0580910D05029904C0806280931D
:1067E0000D0503C08F7D80930D0580910D051C99CB
:1067F00004C0846080930D0503C08B7F80930D05DA
:1068000080910D05019904C0806480930D0503C03B
:106810008F7B80930D059091080580910D05981749
:1068200031F092E090930B058093080509C08091A8
:106830000B05882329F0815080930B05882349F0AC
:1068400080911005811108C080910A05811104C052
:10685000089590930C05F4CF80917F0580FF1BC0B5
:106860009091800580910C0590FF0BC080FF13C0B4
:1068700080910E05816080930E0580E00E948C5E01
:106880000AC084FF08C080910E05806180930E05C8
:1068900080E00E948C5E80917F05869580FF1CC001
:1068A00080918005869590910C0580FF0BC091FF2B
:1068B00013C080910E05826080930E0581E00E94D6
:1068C0008C5E0AC095FF08C080910E05806280939F
:1068D0000E0581E00E948C5E80917F0586958695ED
:1068E00080FF22C0809180058695869580FF10C02C
:1068F00080910A058823C1F080910C0582FF14C0A5
:1069000080910E05846080930E0582E00C948C5E6D
:1069100080910C0586FF08C080910E0580648093ED
:106920000E0582E00C948C5E089533CFCF938823BC
:10693000A1F0C82F0E94851684E50E94E11B6AE041
:1069400070E08C2F90E00E94D41C80E20E94E11B3A
:106950008EE798E0CF910C947716CF910895089523
:106960008091AF069091AC06891B8F7019F480E07E
:1069700090E008959091A906992351F0833030F466
:106980008FEF890F19F08093A906F1CF1092A90615
:10699000E091AC0686E5E89FF0011124E055F94F3F
:1069A000808180FDE4CF8091AC068F5F8F708093F3
:1069B000AE069091AC068091AD06981306C080910A
:1069C000AE068093AD06CF010895CF010895EFE69E
:1069D000F0E080818260808308958091800580FF4F
:1069E00009C080910B018270809309018FEF809321
:1069F000110509C080910B01809582708093090177
:106A000081E08093110580918005869580FF0AC002
:106A100080910B0180958170809309018FEF8093A5
:106A2000120508C080910B0181708093090181E0FB
:106A300080931205809180058695869580FF09C018
:106A400080910B018470809309018FEF809313056F
:106A500009C080910B01809584708093090181E0C9
:106A60008093130500000000000008950F930FB7F6
:106A70000F9300916E000F930B7F00936E000091B7
:106A80006F000D7F00936F000F930BB70F930CB740
:106A90000F921F922F933F934F935F936F937F9328
:106AA0008F939F93AF93BF93EF93FF9311240E9413
:106AB000163EFF91EF91BF91AF919F918F917F9182
:106AC0006F915F914F913F912F911F900F900CBF4D
:106AD0000F910BBF0F910260F89400936F000F911C
:106AE00000936E000F910FBF0F911895CF92DF9218
:106AF000EF92FF920F931F9380917E058823D1F030
:106B000010927E058091810590918205892B91F0EC
:106B100010927F0510928205109281059091AF0628
:106B20008091AC06981731F08091AC068F5F8F7022
:106B30008093AC068091810590918205892B09F4A0
:106B4000AAC140914D0550914E0560914F0570913D
:106B500050059091750500914105109142052091D5
:106B6000430530914405041B150B260B370B892F69
:106B700090E0A0E0B0E0081719072A073B0710F4DF
:106B8000D901C801E82F840F951FA61FB71F809356
:106B90004D0590934E05A0934F05B093500520915D
:106BA000840030918500225E3F4F409165055091F1
:106BB0006605609167057091680580915505909113
:106BC0005605A0915705B0915805840F951FA61F33
:106BD000B71F8093650590936605A0936705B093F2
:106BE0006805B7FD1CC0409A4091150550911605E7
:106BF000609117057091180580911105082E000C01
:106C0000990BAA0BBB0B840F951FA61FB71F809370
:106C1000150590931605A0931705B093180540919C
:106C2000690550916A0560916B0570916C058091C2
:106C3000590590915A05A0915B05B0915C05840FB0
:106C4000951FA61FB71F8093690590936A05A093AF
:106C50006B05B0936C05B7FD1CC0419A40911905B6
:106C600050911A0560911B0570911C0580911205C9
:106C7000082E000C990BAA0BBB0B840F951FA61FA7
:106C8000B71F8093190590931A05A0931B05B09325
:106C90001C0540916D0550916E0560916F057091D6
:106CA000700580915D0590915E05A0915F05B091A2
:106CB0006005840F951FA61FB71F80936D059093E5
:106CC0006E05A0936F05B0937005B7FD1CC0429A86
:106CD00040911D0550911E0560911F057091200582
:106CE00080911305082E000C990BAA0BBB0B840F87
:106CF000951FA61FB71F80931D0590931E05A09397
:106D00001F05B09320054091710550917205609167
:106D10007305709174058091610590916205A09151
:106D20006305B0916405840F951FA61FB71F80935C
:106D3000710590937205A0937305B0937405B7FD28
:106D40003CC0C0902105D0902205E0902305F09032
:106D5000240540911405042E000C550B660B770B8F
:106D60004C0D5D1D6E1D7F1D409321055093220526
:106D7000609323057093240540915105509152056D
:106D80006091530570915405841B950BA60BB70BAE
:106D90008093710590937205A0937305B093740569
:106DA000909180058091360593FF04C081508093B7
:106DB000360503C08F5F80933605809184009091E3
:106DC000850082179307C8F3809165059091660549
:106DD000A0916705B0916805B7FD15C040915105B8
:106DE000509152056091530570915405841B950B89
:106DF000A60BB70B8093650590936605A093670576
:106E0000B093680540988091690590916A05A091BA
:106E10006B05B0916C05B7FD15C0409151055091BF
:106E200052056091530570915405841B950BA60B78
:106E3000B70B8093690590936A05A0936B05B09397
:106E40006C05419880916D0590916E05A0916F053C
:106E5000B0917005B7FD15C0409151055091520594
:106E60006091530570915405841B950BA60BB70BCD
:106E700080936D0590936E05A0936F05B093700598
:106E80004298E15041F080918400909185008217F2
:106E90009307C8F388CE1F910F91FF90EF90DF907A
:106EA000CF900895CF92DF92EF92FF9280913505B7
:106EB000882309F465C0C0904D05D0904E05E09040
:106EC0004F05F09050054091450550914605609161
:106ED000470570914805809136054C155D056E0596
:106EE0007F05E8F420913B0530913C05E0913905A0
:106EF000F0913A05E217F30790F48150809336053C
:106F00002150310930933C0520933B0540912702E5
:106F1000509128026091290270912A0234C0C4164F
:106F2000D506E606F706E8F420913B0530913C05CE
:106F300040913705509138052417350790F48F5F3D
:106F4000809336052F5F3F4F30933C0520933B05E0
:106F500040912702509128026091290270912A02E3
:106F600012C08FEF9FEFDC018093270290932802DD
:106F7000A0932902B0932A024FEF5FEFBA0103C03A
:106F80004FEF5FEFBA018091360587FD06C0809113
:106F90000B0180748093090106C080910B018095DC
:106FA0008074809309012091840030918500225ED5
:106FB0003F4F80913605882311F1439A80918400D8
:106FC0009091850082179307C8F38091360587FF5B
:106FD00004C08F5F8093360503C0815080933605CF
:106FE000439880913605882321F380918400909105
:106FF000850082179307C8F3225E3F4FDACFCB019B
:10700000BA01FF90EF90DF90CF900895BC012091DE
:1070100081053091820540918105509182052417A8
:10702000350711F09A01F7CF81E06217730709F075
:1070300080E00895CF93DF93EC0188819981AA8144
:10704000BB81E5E1F5E080839183A283B383EB010B
:1070500088819981AA81BB8184839583A683B78324
:10706000EA0188819981AA81BB8180879187A28763
:10707000B387E90188819981AA81BB81848795873B
:10708000A687B787DF91CF9108953F924F925F9285
:107090006F927F928F929F92AF92BF92CF92DF9228
:1070A000EF92FF920F931F93CF93DF93CDB7DEB78D
:1070B00028970FB6F894DEBF0FBECDBFA091810513
:1070C000B0918205109739F180904D0590904E0552
:1070D000A0904F05B0905005409141055091420558
:1070E000609143057091440584169506A606B7067F
:1070F000C8F010927F051092820510928105909140
:10710000AF068091AC06981731F08091AC068F5F86
:107110008F708093AC0670EDC72E77E0D72EE12CF0
:10712000F12C97C14091490550914A0560914B055A
:1071300070914C05481559056A057B0508F46EC029
:1071400000917A0510917B0520917C0530917D0599
:10715000D1964D915D916D917C91D497EE27059FCD
:10716000F12D169FC001269F900D259F800D911D2A
:10717000069FF00D811D9E1F159FF00D811D9E1F06
:10718000249FF00D811D9E1F149FF10D8E1F9E1FC9
:10719000F6958E1F9E1F709F800D911D719F900D03
:1071A0001124FD01EB5BFF4F4081518162817381AE
:1071B000480F591F611D711D4093310550933205D1
:1071C00060933305709334053497C080D180E2809A
:1071D000F380C416D506E606F70640F4C0923105E2
:1071E000D0923205E0923305F0923405409131059A
:1071F0005091320560913305709134058CED98E023
:10720000BB24B394FC01C590D590E590F490C416CE
:10721000D506E606F70608F475C27FC2409045051C
:1072200050904605609047057090480548145904F1
:107230006A047B0408F080C02091760530917705C0
:1072400040917805509179052D833E834F8358876F
:10725000D1960D911D912D913C91D4974D815E81D8
:107260006F817885EE27419FF12D529FC001629F6B
:10727000900D619F800D911D429FF00D811D9E1FFD
:10728000519FF00D811D9E1F609FF00D811D9E1F5F
:10729000509FF10D8E1F9E1FF6958E1F9E1F349FCF
:1072A000800D911D359F900D11248C0120E030E060
:1072B000C0903105D0903205E0903305F090340550
:1072C000CD01875B9F4FFC010C151D052E053F0569
:1072D000C0F4408151816281738149835A836B83F9
:1072E0007C83C01AD10AE20AF30AC416D506E60660
:1072F000F70610F46A017B018CED98E03324339497
:1073000010C0C080D180E280F380F6CFF694E7947D
:10731000D794C794330C049628E0883F920709F469
:1073200080C2FC0105911591259134910C151D0524
:107330002E053F0558F375C2809136058823D9F094
:10734000D7964D915C91D89760E070E0009127024C
:10735000109128022091290230912A020417150762
:107360002607370741F010922B0210922C02109240
:107370002D0210922E02409123025091240260911E
:1073800025027091260277FF5CC0AF5BBF4F8D91E5
:107390009D910D90BC91A02D2CED38E041E0F901BC
:1073A000C590D590E590F490C816D906EA06FB067C
:1073B00058F4B695A79597958795440F2C5F3F4F46
:1073C00058E0283F350759F74093750580329105FD
:1073D000A105B10520F480E290E0A0E0B0E0809744
:1073E000A109B109811578E09707A105B10508F455
:1073F000CEC224E0929FF00111249F012450334F0C
:10740000F901329665917491EE27879FA001869FBE
:10741000410D5E1F06944E1F5E1F112460E070E058
:10742000F90185919491A0E0B0E0841B950BA60B27
:10743000B70B8093230290932402A0932502B0936C
:107440002602C0902302D0902402E0902502F09002
:1074500026028091810590918205892B09F01DC338
:107460007FDA9093820580938105892B09F415C3F7
:10747000E0918105F0918205808183FF19C09F0111
:107480002F5D3F4FAF01435E5F4FBF01675E7F4F90
:10749000CF014596CFDD9091AF068091AC0698174D
:1074A000F9F28091AC068F5F8F708093AC06D8CFD5
:1074B000C588D688E788F08C81E0C114D104E10446
:1074C000F10409F480E0018D128D238D348D0115B6
:1074D00011052105310509F08260458D568D678DB6
:1074E00070A1411551056105710509F08460809313
:1074F0007F0510927605109277051092780510920C
:10750000790510927A0510927B0510927C051092F5
:107510007D0585A196A1A7A1B0A580934105909373
:107520004205A0934305B09344058824992454014F
:10753000881A990AAA0ABB0A80927105909272056C
:10754000A0927305B092740580926D0590926E05BD
:10755000A0926F05B09270058092690590926A05BD
:10756000A0926B05B0926C058092650590926605BD
:10757000A0926705B0926805CC0CDD1CEE1CFF1CC8
:10758000C0925505D0925605E0925705F0925805E5
:10759000000F111F221F331F0093590510935A0526
:1075A00020935B0530935C05440F551F661F771FC2
:1075B00040935D0550935E0560935F057093600591
:1075C00041A152A163A174A1440F551F661F771FEB
:1075D0004093610550936205609363057093640561
:1075E000880F991FAA1FBB1F8093510590935205C6
:1075F000A0935305B093540510924D0510924E057B
:1076000010924F051092500581A592A5A3A5B4A58F
:107610008093490590934A05A0934B05B0934C0580
:1076200085A596A5A7A5B0A9809345059093460585
:10763000A0934705B093480586A980933505882314
:1076400009F183AD94AD90933A058093390581ADEE
:1076500092AD909338058093370510922B021092CB
:107660002C0210922D0210922E0287A990ADA0E05C
:10767000B0E08093270290932802A0932902B09350
:107680002A020BC08FEF9FEFDC01809327029093BB
:107690002802A0932902B0932A0285A9909180051F
:1076A000891719F08093800598D973D88FEF9FEFD1
:1076B000DC018093230290932402A0932502B093CF
:1076C0002602E0918105F0918205EB5BFF4F8081FE
:1076D0009181A281B3818093310590933205A0936B
:1076E0003305B09334052CED38E041E0F901C59045
:1076F000D590E590F490C816D906EA06FB0608F482
:107700006BC176C17695679557954795BB0C0496E6
:10771000E8E0883F9E0709F075CDB09275054032CC
:1077200051056105710520F440E250E060E070E031
:107730004052510961097109411588E058076105F6
:10774000710500F194E0599FF0011124CF0184509C
:10775000934FFC013296E590F490F701DD244F9FA2
:1077600050014E9FA10CBD1C0694AD1CBD1C1124E4
:10777000FC01C590D490E12CF12CCA18DB08E1087B
:10778000F10824C06A017B01F694E794D794C7946A
:10779000F601EC7FCF018450974F7C01FC0185916D
:1077A0009491F7013296E590F49047704E9DB001A8
:1077B0004F9D700D1124AB0163E0569547956A9576
:1077C000E1F76C01C41AD50AE12CF12C0C0D1D1D3A
:1077D0002E1D3F1D00937A0510937B0520937C0599
:1077E00030937D059091350580913605992309F4F4
:1077F00065C0882309F42DCED7968D919C91D8979A
:10780000A0E0B0E040912702509128026091290247
:1078100070912A02481759076A077B0709F051C07F
:1078200018CE30927505F0E2CF16D104E104F104D0
:1078300028F430E2C32ED12CE12CF12CF0E2CF1A47
:10784000D108E108F108C11428E0D206E104F104EE
:1078500008F440C034E0D39EC00111248450934FFB
:10786000FC013296059114916C2D3327619FA00184
:10787000609F410D531F0694431F531F1124FC01A9
:10788000C590D490E12CF12CC41AD50AE108F10876
:107890004D815E816F8178854C0D5D1D6E1D7F1D54
:1078A000409376055093770560937805709379053A
:1078B00080913505811132C080913605882309F405
:1078C000C8CD10922B0210922C0210922D02109211
:1078D0002E02BFCD970186013695279517950795FE
:1078E000F801EC7FCF018450974FFC010591149172
:1078F000FC013296459154913C2D3770349FC00164
:10790000359F900D112423E0969587952A95E1F7F0
:107910006801C81AD90AE12CF12CBACF430C511CCA
:10792000611C711C481459046A047B04C8F48091DA
:107930003605882309F48DCDD7964D915C91D89763
:1079400060E070E000912702109128022091290246
:1079500030912A02041715072607370709F479CD55
:1079600010922B0210922C0210922D0210922E02D5
:10797000D7968D919C91D897A0E0B0E08093270294
:1079800090932802A0932902B0932A0262CDAC0101
:10799000BD017695679557954795FA01EC7FAF0144
:1079A0004450574FFA0125913491FA01329665916E
:1079B00074918770869FA001879F500D1124CA0182
:1079C000F3E096958795FA95E1F7A901481B590BC5
:1079D000CA01A0E0B0E02DCDB695A7959795879503
:1079E000440F2C5F3F4F68E0283F360709F07ECEFA
:1079F0004093750580329105A105B10520F480E220
:107A000090E0A0E0B0E08097A109B109811558E0AD
:107A10009507A105B105F8F064E0969FF0011124E7
:107A20009F012450334FF901329665917491EE27EE
:107A3000879FA001869F410D5E1F06944E1F5E1F0B
:107A40001124F901C590D490E12CF12CC41AD50A67
:107A5000E108F10822C0AC01BD0176956795579504
:107A60004795FA01EC7FAF014450574FFA01C5909A
:107A7000D490FA013296459154918770849F900179
:107A8000859F300D1124C901A3E096958795AA958D
:107A9000E1F7C81AD90AE12CF12CC701B6012896E2
:107AA0000FB6F894DEBF0FBECDBFDF91CF911F910F
:107AB0000F91FF90EF90DF90CF90BF90AF909F908D
:107AC0008F907F906F905F904F903F900895CF92EE
:107AD000DF92EF92FF921F93CF93DF938FEF9FEF91
:107AE00090938900809388001AE0C0E0D0E07894F9
:107AF00080913D0590913E05A0913F05B0914005D4
:107B0000892B8A2B8B2B11F40E94763580912B02C6
:107B100090912C02A0912D02B0912E02892B8A2BDC
:107B20008B2B49F4BFD960932B0270932C02809366
:107B30002D0290932E0280913D0590913E05A091DB
:107B40003F05B0914005892B8A2B8B2B49F49DDA98
:107B500060933D0570933E0580933F0590934005EB
:107B6000C0903D05D0903E05E0903F05F090400567
:107B700040912B0250912C0260912D0270912E02A7
:107B8000FC2DED2D3E2D2F2D4C155D056E057F0531
:107B900020F4F42FE52F362F272F8F2F9E2FA32F82
:107BA000B22F009721E0A207B10520F08FEF9FEFE1
:107BB000A0E0B0E0C81AD90AEA0AFB0AC0923D0563
:107BC000D0923E05E0923F05F09240054F3F2FEFE7
:107BD00052076207720761F0481B590B6A0B7B0B57
:107BE00040932B0250932C0260932D0270932E022F
:107BF000F8942091840030918500205F3F4F115010
:107C000039F0C80FD91FC217D30708F470CF01C0CD
:107C1000E901D0938900C09388007894DF91CF91D7
:107C20001F91FF90EF90DF90CF90089550CF9091EB
:107C30006F0091FB222720F991FF05C090916F0002
:107C40009D7F90936F0094E0899FF0011124EB5E7B
:107C5000FA4F6081718182819381222329F02091E2
:107C60006F00226020936F00089590916F0091FB48
:107C7000222720F991FF05C090916F009D7F90937E
:107C80006F0034E0839FC0011124FC01EB5EFA4FCA
:107C90004081518162817381FC01EB5DFA4F408329
:107CA00051836283738381E080937E05222329F0D0
:107CB00080916F00826080936F00089590916F00B3
:107CC00091FB222720F991FF05C090916F009D7FC5
:107CD00090936F0094E0899FF0011124EB5DFA4FBF
:107CE0006081718182819381222329F020916F002C
:107CF000226020936F0008954F925F926F927F925F
:107D00008F929F92AF92BF92CF92DF92EF92FF92AB
:107D100080916F0081FB992790F981FF05C08091C8
:107D20006F008D7F80936F00409015055090160571
:107D300060901705709018058090190590901A05AD
:107D4000A0901B05B0901C05C0901D05D0901E058D
:107D5000E0901F05F0902005992329F080916F0095
:107D6000826080936F0082ED98E00E9477164AE06F
:107D700050E0C301B2010E94C31C8EEC98E00E9447
:107D800077164AE050E0C501B4010E94C31C8AEC9A
:107D900098E00E9477164AE050E0C701B6010E94C1
:107DA000C31C8AE0FF90EF90DF90CF90BF90AF9020
:107DB0009F908F907F906F905F904F900C94E11BFD
:107DC000DB0190918F05992309F440C0833070F452
:107DD00094E0899FF0011124ED57FA4FAB01770F22
:107DE000660B770B4083518362837383813091F0FC
:107DF00018F08230E9F008952FEF30E00E94E9B2E8
:107E000020ED37E040E050E00E94B6B2B9018EE2CA
:107E10000C94C6122FEF30E00E94E9B220ED37E05B
:107E200040E050E00E94B6B2B9018DE20C94C61257
:107E30002FEF30E00E94E9B220ED37E040E050E063
:107E40000E94B6B2B9018CE20C94C61208958091DA
:107E50008F05882391F0609183057091840580E0FF
:107E6000AFDF609187057091880581E0A9DF60919F
:107E70008B0570918C0582E0A3CF0895EAE0F1E0D4
:107E8000808188608083808180618083808180623E
:107E90008083DDDFE1E2F1E08081887F81608083A3
:107EA000089567FD2CC0813061F028F0823099F090
:107EB0008330D9F024C0662311F0A19A2AC0A1987A
:107EC00028C0809108016111809580788093060117
:107ED00047FF27C008958091080161118095807443
:107EE0008093060147FF23C0089580910801611126
:107EF000809588708093060147FF21C0089547FD53
:107F000026C0813071F038F0823089F08330B9F0CA
:107F1000089547FD1CC0442311F0A09A0895A0982D
:107F20000895442311F0A29A0895A298089580918B
:107F30000801411180958072809306010895809117
:107F4000080141118095807180930601089508957C
:107F5000643091F040F4613059F06230A9F420E0CF
:107F600040E061E09ECF683059F0603149F00CC0CC
:107F700020E040E060E095CF20E041E060E091CF7C
:107F800020E041E061E08DCF0E94881682EB98E00E
:107F90000C9477160F931F93CF93999A989A809188
:107FA00007018068809307019A9A80910701806495
:107FB000809307018091070180628093070180917F
:107FC0000701886080930701809107018061809399
:107FD00007010FE213E0C0E0F80161918F018C2FDF
:107FE000B7DFCF5FC630C1F7CF911F910F910895D2
:107FF000D1DFEAE0F1E0808182608083808181606E
:1080000080838081846080838081806480830F9AF4
:10801000179A0E9A169A0D9A159A0C9A149A389ADB
:108020004098179A8091B9058E7F8093B905399A47
:108030004198169A8091B9058D7F8093B9053A9A37
:108040004298159A8091B9058B7F8093B9053B9A28
:108050004398149AA0E8B0E08C918C7F8C93E1E86F
:10806000F0E08081877E886080838C918F738C9311
:108070008081887F8260808380E090E49093890093
:10808000809388001092850010928400EFE6F0E063
:10809000808182608083789482E0809380050E9452
:1080A000ED3481E080938F05E9CE8DE998E00E9460
:1080B0007716919902C080E301C081E30E94E11B21
:1080C000909902C080E301C081E30E94E11B89E92D
:1080D00098E00E94771680910601881F8827881FE4
:1080E000805D0E94E11B929902C080E301C081E3A0
:1080F0000E94E11B85E998E00E94771680910601B5
:1081000086FD02C080E301C081E30E94E11B8091F3
:10811000060185FD02C080E301C081E30E94E11BEE
:1081200080E998E00E9477168091060183FD02C0E5
:1081300080E301C081E30E94E11B8091060184FD80
:1081400002C080E301C081E30C94E11BCF93DF9375
:10815000CDB7DEB760970FB6F894DEBF0FBECDBFC8
:108160008091520290915302A0915402B091550215
:1081700089839A83AB83BC83809156029091570286
:10818000A0915802B09159028D839E83AF83B88726
:1081900080915A0290915B02A0915C02B0915D02C5
:1081A00089879A87AB87BC8780915E0290915F0236
:1081B000A0916002B09161028D879E87AF87B88BD6
:1081C0000E94E76D6091660270916702072E000CB5
:1081D000880B990B0E94F8AF2AE037ED43E25CE38D
:1081E0000E9494B160936202709363028093640270
:1081F0009093650280E00E94AB5481E00E94AB54F2
:1082000082E00E94AB5423DE0E942E6E40E150E0DB
:1082100062E572E0CE0101960E9421B7892B51F0F0
:1082200060960FB6F894DEBF0FBECDBFDF91CF9141
:108230000C94735260960FB6F894DEBF0FBECDBF9C
:10824000DF91CF9108958E35924041F00E948816BB
:1082500082E894E10E94771681E0089580E0089515
:10826000EF92FF920F931F93CF93DF93CDB7DEB7BB
:10827000C458D1090FB6F894DEBF0FBECDBFED963E
:108280001CAE1DAE1EAE1FAEED9785E492E5A2E5D5
:10829000B0E0E9968CAF9DAFAEAFBFAFE997CF57D7
:1082A000DF4F19821882C158D04084E690E0C1584F
:1082B000DF4F99838883CF57D0400E9424171092B4
:1082C00091059E012F573F4F44E050E0BE016B588F
:1082D0007F4FCE0181589F4F0E942817C158DF4F12
:1082E00088819981CF57D0400296C158DF4F99833A
:1082F0008883CF57D040CF57DF4F19821882C1589B
:10830000D04081E0CC57DF4F8883C458D0409E01D5
:108310002F573F4F41E050E0BE016C577F4FCE01D9
:1083200081589F4F0E9428179E012F573F4F48E4C6
:1083300050E061E676E0CE0181589F4F0E942817F9
:108340009E012F573F4F40E150E061E376E0CE01C0
:1083500081589F4F0E9428178AE097EDA3EABCE35B
:10836000ED968CAF9DAFAEAFBFAFED979E012F578F
:108370003F4F44E050E0BE0167587F4FCE01815827
:108380009F4F0E9428178E010F5F1F4F8CE0F8014E
:1083900011928A95E9F79E012F573F4F4CE050E02C
:1083A000B801CE0181589F4F0E942817AE961FAE8C
:1083B000AE9719821A821B821C829E012F573F4F53
:1083C00041E050E0BE0163597F4FCE0181589F4F7D
:1083D0000E9428179E012F573F4F44E050E0B801FC
:1083E000CE0181589F4F0E94281780E090E0A0E2C4
:1083F000B1E489839A83AB83BC839E012F573F4F9F
:1084000044E050E0B801CE0181589F4F0E942817E8
:10841000ED961CAE1DAE1EAE1FAEED9783E0AE9680
:108420008FAFAE9789839E012F573F4F44E050E0B6
:10843000BE0167587F4FCE0181589F4F0E94281779
:108440009E012F573F4F41E050E0BE0163597F4FDF
:10845000CE0181589F4F0E9428179E012F573F4FF2
:1084600041E050E0B801CE0181589F4F0E9428178B
:108470002AE0F22EFA949E012F573F4F44E050E03D
:10848000FF2049F0BE0167587F4FCE0181589F4FB2
:108490000E942817EFCF62E975E0CE0181589F4F07
:1084A0000E9428179E012F573F4F44E250E06CE096
:1084B00076E0CE0181589F4F0E94281783E0CD5768
:1084C000DF4F8883C358D040EE968FAFEE97E1968A
:1084D0001CAE1DAE1EAE1FAEE19719821A821B8222
:1084E0001C82ED961CAE1DAE1EAE1FAEED979E011A
:1084F0002F573F4F41E050E0BE016D577F4FCE01F7
:1085000081589F4F0E9428179E012F573F4F41E0EF
:1085100050E0BE0163587F4FCE0181589F4F0E94AB
:1085200028179E012F573F4F44E050E0B801CE017D
:1085300081589F4F0E9428179E012F573F4F44E0BC
:1085400050E0BE0163597F4FCE0181589F4F0E947A
:1085500028179AE0E92EF12CF1E0EF1AF10871F0FA
:108560009E012F573F4F44E050E0BE0167587F4FB8
:10857000CE0181589F4F0E942817EECFAE961FAEB6
:10858000AE978FEF89839E012F573F4F41E050E018
:10859000BE0163597F4FCE0181589F4F0E9428171B
:1085A0009E012F573F4F41E050E0B801CE01815866
:1085B0009F4F0E94281780E1F82EF8018F2D11920D
:1085C0008A95E9F79E012F573F4F40E150E0B801EF
:1085D000CE0181589F4F0E94281719829E012F5764
:1085E0003F4F41E050E0B801CE0181589F4F0E94BB
:1085F000281788EC90E0AF969FAF8EAFAF9780EFD3
:1086000090E0E1969FAF8EAFE19786E490E09A8389
:1086100089838EE690E09C838B83EE961FAEEE9767
:10862000EF961FAEEF979E012F573F4F44E050E06B
:10863000BE0163597F4FCE0181589F4F0E9428177A
:108640009E012F573F4F44E050E0B801CE018158C2
:108650009F4F0E9428179E012F573F4F42E050E046
:10866000BE0163587F4FCE0181589F4F0E9428174B
:10867000F8011192FA94E9F780E090E0A0E8BFE3F6
:108680008D879E87AF87B88B8091FB049091FC0407
:10869000A091FD04B091FE0489839A83AB83BC83CF
:1086A0008091FF0490910005A0910105B091020511
:1086B0008D839E83AF83B8878091030590910405D5
:1086C000A0910505B091060589879A87AB87BC877D
:1086D0009E012F573F4F40E150E0B801CE01815835
:1086E0009F4F0E94281784E190E09A8389839E011E
:1086F0002F573F4F42E050E0B801CE0181589F4FC5
:108700000E9428179E012F573F4F4CE050E06DED1F
:1087100074E0CE0181589F4F0E94281780E290E0BC
:108720009A8389839E012F573F4F42E050E0B80162
:10873000CE0181589F4F0E94281781E089839E01B6
:108740002F573F4F41E050E0B801CE0181589F4F75
:108750000E94281780E2EFE7F2E0D80101900D9225
:108760008A95E1F79E012F573F4F40E250E0B80154
:10877000CE0181589F4F0E942817AE961FAEAE972C
:108780009E012F573F4F41E050E0BE0163597F4F9C
:10879000CE0181589F4F0E942817198280E090E0F7
:1087A000A0E4B0E4ED968CAF9DAFAEAFBFAFED9758
:1087B0009E012F573F4F41E050E0B801CE01815854
:1087C0009F4F0E9428179E012F573F4F44E050E0D3
:1087D000BE0167587F4FCE0181589F4F0E942817D6
:1087E0008AE1F80111928A95E9F79E012F573F4FD0
:1087F0004AE150E0B801CE0181589F4F0E942817EE
:1088000084E3EFE9F2E0D80101900D928A95E1F757
:108810009E012F573F4F44E350E0B801CE018158ED
:108820009F4F0E9428171A8219821C821B821E8267
:108830001D829E012F573F4F46E050E0B801CE0108
:1088400081589F4F0E9428178DE0F80111928A9558
:10885000E9F79E012F573F4F4DE050E0B801CE01A0
:1088600081589F4F0E9428179E012F573F4F44E089
:1088700050E063ED75E0CE0181589F4F0E942817AC
:108880009E012F573F4F4CE050E063E875E0CE016A
:1088900081589F4F0E9428178CE6F80111928A9503
:1088A000E9F79E012F573F4F4CE650E0B801CE014B
:1088B00081589F4F0E9428179E012F573F4F4CE031
:1088C00050E060E076E0CE0181589F4F0E9428176B
:1088D000E1961CAE1DAE1EAE1FAEE197E5961CAE36
:1088E0001DAE1EAE1FAEE5979E012F573F4F48E0CD
:1088F00050E0BE0163597F4FCE0181589F4F0E94C7
:1089000028179E012F573F4F44E050E067E774E07F
:10891000CE0181589F4F0E9428179E012F573F4F2D
:1089200044E050E06BE774E0CE0181589F4F0E9415
:1089300028179E012F573F4F44E050E06FE774E047
:10894000CE0181589F4F0E9428179E012F573F4FFD
:1089500041E050E066E774E0CE0181589F4F0E94ED
:1089600028179E012F573F4F44E050E060E172E02E
:10897000CE0181589F4F0E94281780919105811147
:108980004FC0C158DF4F08811981CF57D0400456DE
:108990001109CF57DF4F88819981C158D040AF96D8
:1089A0009FAF8EAFAF9784E690E0C158DF4F9983B9
:1089B0008883CF57D0409E012F573F4F44E050E06F
:1089C00065E373E0CE0181589F4F0E9428179E01F6
:1089D0002F573F4F42E050E0BE0163597F4FCE0119
:1089E00081589F4F0E9428170E948516B80180E782
:1089F00094E10E94E216AF964EAD5FADAF9760E096
:108A000070E083E694E10E94EC1680E694E10E9417
:108A10007716C80118DC90919105892B80939105F8
:108A20000E9426179091910581E08927CC57DF4F4E
:108A30000FB6F894DEBF0FBECDBFDF91CF911F916F
:108A40000F91FF90EF9008951F93CF93DF93CDB7D1
:108A5000DEB72C970FB6F894DEBF0FBECDBFA1E6F0
:108A6000B6E020E030E0C9012430310510F083E0A9
:108A700090E0880F991F880F991FFC01E556FC4E66
:108A8000459155916591749154964D935D936D9375
:108A90007C935797FC01E557FC4E459155916591A4
:108AA000749194964D935D936D937C939797FC018D
:108AB000E558FC4E45915591659174914D935D93A8
:108AC0006D937D932F5F3F4F2430310509F0CBCF5D
:108AD00080E29EE4A0E0B0E080937106909372067D
:108AE000A0937306B093740680E090E0AAEFB4E41C
:108AF0008093950690939606A0939706B093980658
:108B000040E050E86BE375E44093990650939A0671
:108B100060939B0670939C0680939D0690939E069F
:108B2000A0939F06B093A0061092A1061092A206F1
:108B30001092A3061092A4061092A5061092A60603
:108B40001092A7061092A80680E090E0A0E4B1E49D
:108B50008093310690933206A0933306B093340687
:108B60008093350690933606A0933706B093380667
:108B70008DEC9CECACECBEE38093390690933A0606
:108B8000A0933B06B0933C0680E090E0A0E2B1E405
:108B900080933D0690933E06A0933F06B093400617
:108BA000109276041092770410927804109279044F
:108BB00010927A0410927B0410927C0410927D042F
:108BC00010927E0410927F0410928004109281040F
:108BD0001092820480E090E0A0E4B0E48093100260
:108BE00090931102A0931202B09313020E94F41DFD
:108BF00080E090E0A0EBBFEB80939205909393050B
:108C0000A0939405B093950580E090E0A8EAB1E4C4
:108C10008093FB049093FC04A093FD04B093FE04A6
:108C200085E391E5A5E9BEE38093FF0490930005F9
:108C3000A0930105B093020580ED9EEFACEBB3E489
:108C40008093030590930405A0930505B093060552
:108C500080E090E0A3E9B3E48093DD049093DE0428
:108C6000A093DF04B093E00483EC94E6AAE2B1E4BD
:108C70008093E1049093E204A093E304B093E404AE
:108C800080EB98EBA1E1B5E48093E5049093E604D2
:108C9000A093E704B093E80481E00E942D330E9482
:108CA000AF341092D3051092D4051092D5051092CE
:108CB000D6058CE0E3EDF2E0DE01119601900D9215
:108CC0008A95E1F713E01150C0F084E0189F9001FD
:108CD0001124E1E0F0E0EC0FFD1FE20FF31F6081D3
:108CE000718182819381F901ED57FA4F608371831D
:108CF00082839383812F64D8E6CF28DA0E94851679
:108D000088E593E12C960FB6F894DEBF0FBECDBF79
:108D1000DF91CF911F910C947716CF93C82F8111BB
:108D200002C00E94851681E493E10E9477168FEFBE
:108D300090E10E9477168AE00E94E11B8AE00E947F
:108D4000E11BC11106C00E94851680E393E10E94D9
:108D500077166FEF81E08C270E946396C11108C0DF
:108D60000E94851682E193E10E9477160E94851683
:108D7000409185065091860660918706709188061D
:108D800089E093E10E94C2164091890650918A06BB
:108D900060918B0670918C0686E093E10E94C2166A
:108DA00040918D0650918E0660918F0670919006CD
:108DB00083E093E10E94C216409191065091920681
:108DC000609193067091940680E093E10E94C21630
:108DD0008AE00E94E11BC11108C00E9485168EED39
:108DE00092E10E9477160E9485166091610670914B
:108DF000620680916306909164060E94F6AFAB0113
:108E0000BC0185ED92E10E94C216609165067091E9
:108E1000660680916706909168060E94F6AFAB01E6
:108E2000BC0182ED92E10E94C216609169067091C8
:108E30006A0680916B0690916C060E94F6AFAB01BA
:108E4000BC018FEC92E10E94C21660916D06709198
:108E50006E0680916F06909170060E94F6AFAB018E
:108E6000BC018CEC92E10E94C2168AE00E94E11BD8
:108E7000C11108C00E94851682E892E10E9477160F
:108E80000E9485164091950650919606609197062E
:108E90007091980689E792E10E94C2164091990666
:108EA00050919A0660919B0670919C0686E792E12C
:108EB0000E94C21640919D0650919E0660919F06A9
:108EC0007091A00683E792E10E94C2168AE00E9498
:108ED000E11BC11113C00E9485168BE292E10E9432
:108EE000771680E092E10E94771681EF91E10E946F
:108EF00077168AE00E94E11B0E9485166091710638
:108F00007091720680917306909174060E94F6AF7C
:108F1000AB01BC0188EE91E10E94C2164091A1060E
:108F20005091A2066091A3067091A40685EE91E18E
:108F30000E94C2164091A5065091A6066091A70610
:108F40007091A80682EE91E10E94C216409131060E
:108F50005091320660913306709134068FED91E1A5
:108F60000E94C21640913506509136066091370630
:108F7000709138068CED91E10E94C216409139063D
:108F800050913A0660913B0670913C0689ED91E163
:108F90000E94C21640913D0650913E0660913F06E8
:108FA0007091400686ED91E10E94C2168AE00E940F
:108FB000E11BC11108C00E94851682EC91E10E945C
:108FC00077160E9485166091300670E089EB91E17A
:108FD0000E94A8168AE00E94E11BC11108C00E94ED
:108FE00085168AEA91E10E9477160E9485164091C3
:108FF000FB045091FC046091FD047091FE0481EA31
:1090000091E10E94C2162CEA35EC47E25EE36091E2
:10901000FF047091000580910105909102050E9466
:109020005DAFAB01BC018EE991E10E94D2162CEA42
:1090300035EC47E25EE36091030570910405809191
:109040000505909106050E9494B1AB01BC018BE926
:1090500091E10E94D2168AE00E94E11BC11102C078
:109060000E9485164091DD045091DE046091DF047A
:109070007091E00482E991E10E94C2162CEA35EC7D
:1090800047E25EE36091E1047091E2048091E304C1
:109090009091E4040E945DAFAB01BC018FE891E1C7
:1090A0000E94D2162CEA35EC47E25EE36091E504BB
:1090B0007091E6048091E7049091E8040E9494B1D5
:1090C000AB01BC018CE891E10E94D2168AE00E94BB
:1090D000E11BC11110C00E9485168DE791E10E942D
:1090E00077168FEF90E10E9477168CEF90E10E9447
:1090F00077160E94851640919205509193056091D4
:1091000094057091950584E791E10E94C2168AE06A
:109110000E94E11BC11108C00E94851683E691E1FF
:109120000E9477160E9485164091D3055091D40570
:109130006091D5057091D6058AE591E10E94C2162D
:109140008AE00E94E11BC11108C00E94851681E4DB
:1091500091E10E9477160E948516409183055091F7
:109160008405609185057091860588E391E10E94F0
:10917000EC164091870550918805609189057091A2
:109180008A0585E391E10E94EC1640918B05509190
:109190008C0560918D0570918E0582E391E10E94AE
:1091A000EC168AE00E94E11BC11108C00E948516DE
:1091B0008AE191E10E9477160E94851680917604DB
:1091C00024E6829FC001112481589F4F6FEF70E009
:1091D0000E9481B270E080E090E00E94F6AF20E053
:1091E00030E048EC52E40E945DAFAB01BC0181E18C
:1091F00091E10E94C21640917704509178046091E9
:10920000790470917A048EE091E10E94C216409137
:109210007B0450917C0460917D0470917E048BE00E
:1092200091E10E94C21640917F04509180046091A8
:1092300081047091820488E091E10E94C2164091FD
:10924000100250911102609112027091130285E098
:1092500091E10E94C2168AE0CF910C94E11B2F92FB
:109260003F924F925F926F927F928F929F92AF92B6
:10927000BF92CF92DF92EF92FF920F931F93CF9303
:10928000DF93CDB7DEB7C25AD1090FB6F894DEBF6F
:109290000FBECDBF2DB73EB7CF55DF4F39832883E3
:1092A000C15AD040C756DF4F19821882C959D040E1
:1092B00084E690E0C956DF4F99838883C759D04030
:1092C0000E94241701E09E0127563F4F44E050E0E2
:1092D000BE016F567F4FCE0189569F4F0E947D176A
:1092E0009E0127563F4F42E050E0BE016B567F4F34
:1092F000CE0189569F4F0E947D1743E050E0BE018A
:109300006F567F4F85E393E00E9440B7892B19F198
:10931000CC56DF4F8881C459D040882359F08FE361
:10932000CF56DF4F8883C159D040CE56DF4F1882C9
:10933000C259D0400E948516BE016F567F4F8FE301
:1093400094E10E948B1681E394E10E94771681E0FC
:10935000809391059DC5C357DF4F188219821A82E9
:109360001B82CD58D040C756DF4F19821882C95989
:10937000D04001E09E0127563F4F41E050E0BE0142
:1093800064567F4FCE0189569F4F0E947D178DB73F
:109390009EB7C156DF4F99838883CF59D0407E0155
:1093A0009DE7E90EF11C80E1EFEDF2E0D7010190BD
:1093B0000D928A95E1F76E01EDE6CE0ED11C80E1AB
:1093C000EFEEF2E0D60101900D928A95E1F780E18F
:1093D000EFEFF2E09E012F5F3F4F5901D90101905D
:1093E0000D928A95E1F7C456DF4F4881CC59D040A1
:1093F00050E04D5F5F4F440F551F440F551F8DB711
:109400009EB7841B950B0FB6F8949EBF0FBE8DBF01
:10941000EDB7FEB731961F010091900511E00127CD
:1094200028563F4FBF01CE0189569F4F0E947D179E
:109430000091900501279E0127563F4F44E050E0E0
:1094400061E776E0CE0189569F4F0E947D17C45692
:10945000DF4F6880CC59D040712CF3E06F0E711C47
:10946000660C771C660C771C2DB73EB7261937099A
:109470000FB6F8943EBF0FBE2DBF8DB79EB70196B5
:109480002C01EDB7FEB7E619F7090FB6F894FEBF49
:109490000FBEEDBF2DB73EB72F5F3F4F4901009183
:1094A000900501279E0127563F4FA301BC01CE0125
:1094B00089569F4F0E947D170091900501279E01BC
:1094C00027563F4FA301B401CE0189569F4F0E94FA
:1094D0007D1730919005C256DF4F3883CE59D0406A
:1094E000332309F4EEC011E0C256DF4F0881CE5994
:1094F000D04001279E0127563F4F44E050E065E9E8
:1095000076E0CE0189569F4F0E947D17009190050D
:1095100001279E0127563F4F44E050E069E976E07D
:10952000CE0189569F4F0E947D170091900501271B
:109530009E0127563F4F44E050E06DE976E0CE01B2
:1095400089569F4F0E947D170091900501279E012B
:1095500027563F4F44E050E061EA76E0CE0189565D
:109560009F4F0E947D170091900501279E0127566D
:109570003F4F44E050E065EA76E0CE0189569F4FC8
:109580000E947D170091900501279E0127563F4FAD
:1095900040E150E061E376E0CE0189569F4F0E94A2
:1095A0007D170091900501279E0127563F4F44E00B
:1095B00050E0BE0163577F4FCE0189569F4F0E94F6
:1095C0007D17C156DF4F88819981CF59D0400FB6A2
:1095D000F8949EBF0FBE8DBF0091900501279E019C
:1095E00027563F4F4CE050E0BE016F5F7F4FCE01EA
:1095F00089569F4F0E947D170091900501279E017B
:1096000027563F4F41E050E0BE0163597F4FCE01E6
:1096100089569F4F0E947D170091900501279E015A
:1096200027563F4F44E050E0BE016F5F7F4FCE01B1
:1096300089569F4F0E947D170091900501279E013A
:1096400027563F4F44E050E0BE0163577F4FCE01A5
:1096500089569F4F0E947D170091900501279E011A
:1096600027563F4F44E050E0BE0163577F4FCE0185
:1096700089569F4F0E947D1701E09E0127563F4F5C
:1096800041E050E0BE0163597F4FCE0189569F4FA4
:109690000E947D179E0127563F4F41E050E0BE01DA
:1096A0006F5F7F4FCE0189569F4F0E947D17AE9608
:1096B000CFACAE978981C89E60011124A12CB12C3A
:1096C00090C0C456DF4F6880CC59D040712C92E0D6
:1096D000690E711CA1E6B6E040E050E080E090E049
:1096E000B701E1E0C356DF4FE883CD59D04068169B
:1096F000790664F4C356DF4F1882CD59D0409C01DF
:109700008430910558F023E030E008C0F101E40F07
:10971000F51F00811181228133810BC0220F331F7D
:10972000220F331FFB01E20FF31F00811181228101
:1097300033810D931D932D933D93C356DF4FF881D5
:10974000CD59D040FF2341F0F201E40FF51F008115
:1097500011812281338111C09C018430910510F068
:1097600023E030E0220F331F220F331FF601E20FF8
:10977000F31F008111812281338150960D931D9337
:109780002D933C935397C356DF4F2881CD59D0403A
:10979000222341F0F401E40FF51F008111812281A1
:1097A000338111C09C018430910510F023E030E03A
:1097B000220F331F220F331FF501E20FF31F008129
:1097C00011812281338190960D931D932D933C93AB
:1097D000939701964C5F5F4F8430910509F081CFDC
:1097E00082CE00919005AC14BD0491F001279E013A
:1097F00027563F4F44E050E0BE0163577F4FCE01F4
:1098000089569F4F0E947D173FEFA31AB30AE9CFF5
:1098100011E001279E0127563F4F44E050E062E9E6
:1098200075E0CE0189569F4F0E947D1700919005EB
:1098300001279E0127563F4F44E250E06CE076E05E
:10984000CE0189569F4F0E947D1701E09E01275649
:109850003F4F41E050E0BE0165567F4FCE01895633
:109860009F4F0E947D179E0127563F4F41E050E0D9
:10987000B701CE0189569F4F0E947D170091900538
:1098800001279E0127563F4F44E050E0BE01635937
:109890007F4FCE0189569F4F0E947D170091900502
:1098A00001279E0127563F4F44E050E0BE016F5F05
:1098B0007F4FCE0189569F4F0E947D17C556DF4FBF
:1098C000C880CB59D040F7018081C89E6001112427
:1098D000A12CB12C00919005AC14BD0491F001278E
:1098E0009E0127563F4F44E050E0BE0163577F4F33
:1098F000CE0189569F4F0E947D17FFEFAF1ABF0A16
:10990000E9CF11E001279E0127563F4F41E050E08B
:10991000BE0163597F4FCE0189569F4F0E947D172C
:109920000091900501279E0127563F4F41E050E0EE
:10993000BE016F5F7F4FCE0189569F4F0E947D17FA
:109940000091900501279E0127563F4F40E150E0CE
:10995000BE016F5F7F4FCE0189569F4F0E947D17DA
:109960000091900501279E0127563F4F41E050E0AE
:10997000BE016F5F7F4FCE0189569F4F0E947D17BA
:109980000091900501279E0127563F4F44E050E08B
:10999000BE0163597F4FCE0189569F4F0E947D17AC
:1099A0000091900501279E0127563F4F44E050E06B
:1099B000BE016F5F7F4FCE0189569F4F0E947D177A
:1099C0000091900501279E0127563F4F42E050E04D
:1099D000B701CE0189569F4F0E947D1700919005D7
:1099E00001279E0127563F4F40E150E0BE016F5FC7
:1099F0007F4FCE0189569F4F0E947D1700919005A1
:109A000001112EC0C980DA80EB80FC8020E030E8B4
:109A10004BE355E4C701B6010E9456AF882301F11C
:109A2000C092FB04D092FC04E092FD04F092FE048C
:109A30008D819E81AF81B8858093FF04909300054E
:109A4000A0930105B093020589859A85AB85BC85F5
:109A50008093030590930405A0930505B093060534
:109A600011E001279E0127563F4F42E050E0BE0122
:109A70006F5F7F4FCE0189569F4F0E947D170091E7
:109A8000900501279E0127563F4F4CE050E0BE0154
:109A90006F5F7F4FCE0189569F4F0E947D170091C7
:109AA0009005011115C020E030E84BE355E46981D1
:109AB0007A818B819C810E9456AF882349F08CE08B
:109AC000FE013196ADEDB4E001900D928A95E1F77B
:109AD00011E001279E0127563F4F42E050E0BE01B2
:109AE0006F5F7F4FCE0189569F4F0E947D17009177
:109AF000900501279E0127563F4F41E050E0BE01EF
:109B00006F5F7F4FCE0189569F4F0E947D17009156
:109B1000900501279E0127563F4F40E250E0BE01CD
:109B20006F5F7F4FCE0189569F4F0E947D17009136
:109B3000900501279E0127563F4F41E050E0BE01AE
:109B400063597F4FCE0189569F4F0E947D17009128
:109B5000900501279E0127563F4F45E050E0BE018A
:109B60006F5F7F4FCE0189569F4F0E947D17809176
:109B70009005811102C00E94AF340091900511E060
:109B800001279E0127563F4F4AE150E0BE016F5F1B
:109B90007F4FCE0189569F4F0E947D1700919005FF
:109BA00001279E0127563F4F44E350E0BE016F5FFF
:109BB0007F4FCE0189569F4F0E947D1700919005DF
:109BC00001279E0127563F4F46E050E0BE016F5FE0
:109BD0007F4FCE0189569F4F0E947D1700919005BF
:109BE00001279E0127563F4F4DE050E0BE016F5FB9
:109BF0007F4FCE0189569F4F0E947D17009190059F
:109C000001279E0127563F4F44E050E0BE016F5FA1
:109C10007F4FCE0189569F4F0E947D17009190057E
:109C200001110CC089819A81AB81BC818093D305DD
:109C30009093D405A093D505B093D60581E008276D
:109C40009E0127563F4F4CE050E0BE016F5F7F4FB3
:109C5000CE0189569F4F0E947D17009190050111FA
:109C600009C08CE0FE013196A3E8B5E001900D92A9
:109C70008A95E1F711E001279E0127563F4F4CE6F8
:109C800050E0BE016F5F7F4FCE0189569F4F0E940B
:109C90007D1719821A821B821C821D821E821F82DE
:109CA000188619861A861B861C8600919005012746
:109CB0009E0127563F4F4CE050E0BE016F5F7F4F43
:109CC000CE0189569F4F0E947D1700919005012774
:109CD0009E0127563F4F48E050E0BE016F5F7F4F27
:109CE000CE0189569F4F0E947D1700919005012754
:109CF0009E0127563F4F44E050E067E774E0CE01F5
:109D000089569F4F0E947D170091900501279E0163
:109D100027563F4F44E050E06BE774E0CE01895690
:109D20009F4F0E947D170091900501279E012756A5
:109D30003F4F44E050E06FE774E0CE0189569F4FFB
:109D40000E947D170091900501279E0127563F4FE5
:109D500041E050E066E774E0CE0189569F4F0E94D3
:109D60007D170091900501279E0127563F4F44E043
:109D700050E060E172E0CE0189569F4F0E947D174E
:109D8000C956DF4F88819981C759D04084569109BF
:109D90000E942341809391058823C1F00E9485167B
:109DA000C956DF4F68817981C759D040645671091F
:109DB00089E294E10E94A8166EE572E081E294E1E6
:109DC0000E94E2168AE00E94E11B58C0C756DF4F8E
:109DD00028813981C959D040CB56DF4F888199817C
:109DE000C559D04028173907E9F0109391050E9412
:109DF0008816CB56DF4F68817981C559D04081E004
:109E000094E10E94E216C756DF4F68817981C959F3
:109E1000D0408CEF93E10E94E2168CEE93E10E9419
:109E200077162CC080919005811128C00E9485165C
:109E300005E313E0F80181918F01882319F00E9456
:109E4000E11BF8CFC956DF4F68817981C759D040EF
:109E5000645671098FEC93E10E94A816C756DF4F34
:109E600048815981C959D04060E070E082EC93E1AB
:109E70000E94EC168FEB93E10E947716809190057B
:109E8000811106C080919105811102C00E94A640F7
:109E900080919005811102C00E948D460E94261774
:109EA0009091910581E08927CF55DF4F2881398135
:109EB000C15AD0400FB6F8943EBF0FBE2DBFCE554D
:109EC000DF4F0FB6F894DEBF0FBECDBFDF91CF914D
:109ED0001F910F91FF90EF90DF90CF90BF90AF90C8
:109EE0009F908F907F906F905F904F903F902F90BA
:109EF000089581E080939005B2D91092900508955D
:109F0000F8DF8111ACC90E9424450E9430410E94B3
:109F100085168BEA93E10E94771681E00895BF923F
:109F2000CF92DF92EF92FF920F931F93CF93DF9325
:109F3000CDB7DEB728970FB6F894DEBF0FBECDBF02
:109F400090910A05981709F47AC0B82E882309F46D
:109F500053C080E090E0A0EAB0E48D839E83AF839D
:109F6000B887C0909205D0909305E0909405F0904A
:109F7000950520E030E0A901C701B6010E9456AF67
:109F800087FF0CC0A701960160E070E080EA90E4D2
:109F90000E947CAE6D837E838F83988720E030E0C3
:109FA0004FE153E46D817E818F8198850E9459B184
:109FB000181644F480E090E0AFE1B3E48D839E8313
:109FC000AF83B88720915A0230915B0240915C02C6
:109FD00050915D026D817E818F8198850E9459B17B
:109FE000181654F419821A821B821C82BE016F5FFC
:109FF0007F4FCE01059638D4609152027091530282
:10A00000809154029091550220915602309157024E
:10A01000409158025091590219821A821B821C8267
:10A02000E0905A02F0905B0200915C0210915D0298
:10A03000FE0131966F0164D38B2D0E94433380E083
:10A0400028960FB6F894DEBF0FBECDBFDF91CF913B
:10A050001F910F91FF90EF90DF90CF90BF900895E8
:10A060002F923F924F925F926F927F928F929F9228
:10A07000AF92BF92CF92DF92EF92FF920F931F9316
:10A08000CF93DF93CDB7DEB7A0970FB6F894DEBFBE
:10A090000FBECDBF1C017F8F6E8F498F28A3DC01BF
:10A0A0008D909D90AD90BC90FB014080518062806E
:10A0B00073802CE933E343E651ECC301B201002382
:10A0C00009F43BC00E9459B187FDD5C124ED3CEC99
:10A0D00046E353E4C301B2010E9456AF18160CF4D4
:10A0E000CAC123EA31E040E450ECC501B4010E944A
:10A0F00059B187FDC0C127E030E042E253E4C50119
:10A10000B4010E9456AF18160CF4B5C127E030E038
:10A1100041E253E4C501B4010E9456AF18160CF495
:10A12000AAC127E030E041E253E4C301B2010E943A
:10A1300056AF18160CF49FC124C00E9459B187FD78
:10A140009AC124ED3CEC46E353E4C301B2010E9402
:10A1500056AF18160CF48FC123EA31E040E450ECFE
:10A16000C501B4010E9459B187FD85C127E030E0E7
:10A1700042E253E4C501B4010E9456AF18160CF434
:10A180007AC1E0905A02F0905B0200915C0210915B
:10A190005D0280914E0290914F02A0915002B091C9
:10A1A00051028A8F9B8FAC8FBD8F80914802909116
:10A1B0004902A0914A02B0914B0280934E029093C3
:10A1C0004F02A0935002B093510219821A821B824F
:10A1D0001C82DE0111966D01A3019201C501B4013B
:10A1E0008FD281E09CDE8111DEC08091B90582FFB3
:10A1F00011C02091920530919305409194055091A2
:10A20000950560E070E080E890EC0E947CAE2B0148
:10A210003C0106C0412C512C40E2642E41EC742ECE
:10A220004D865E866F86788AC12CD12CE12C31E474
:10A23000F32EC986DA86EB86FC86BE01675F7F4F08
:10A24000CE010D9611D310910E0510920E0582E0ED
:10A250009CD171D112FD05C060E070E080EC9FE7F9
:10A260005DC080905A0290905B02A0905C02B0901A
:10A270005D02C982DA82EB82FC8220E030E040EAB3
:10A2800050E4C501B4010E947DAE6D837E838F834F
:10A290009887BE016F5F7F4FCE010596E5D24D8254
:10A2A0005E826F82788680E090E0A0E8BFE38983D9
:10A2B0009A83AB83BC83BE016F5F7F4FCE0105964F
:10A2C000D3D210910E0510920E0582E05ED133D1EB
:10A2D00012FFC2CF0E94A91F20E030E040E450E40A
:10A2E00060915A0270915B0280915C0290915D02D4
:10A2F0000E9494B12B013C01A5019401C501B40158
:10A300000E947DAE9B01AC01C301B2010E947DAEF3
:10A310002DEC3CEC4CE45EE30E9494B1209192055C
:10A320003091930540919405509195050E947DAE22
:10A330005B018C01898D8250823048F580E090E08D
:10A34000A0E0B1E4898B9A8BAB8BBC8B60915A02F5
:10A3500070915B0280915C0290915D02B98DB33087
:10A3600029F020E030E040EA50E404C020E030E092
:10A3700048EC51E40E947DAE6D8B7E8B8F8B988F65
:10A38000BE016F5E7F4FCE0145966ED207C0E98D4C
:10A39000E13021F480E0C3DD811105C0F8A1F33084
:10A3A00008F449C008C098A1933008F46DC0A12CEE
:10A3B000B12C00EC1FE729E3822E23E0922ED4017A
:10A3C0008D914D01882319F00E94E11BF8CFF10116
:10A3D000608171818281938143E050E00E945F1D22
:10A3E00091E4892E93E0992ED4018D914D0188231B
:10A3F00019F00E94E11BF8CFEE8DFF8D6081718115
:10A400008281938143E050E00E945F1D86E4882EA4
:10A4100083E0982ED4018D914D01882319F00E947C
:10A42000E11BF8CF43E050E0B501C8010E945F1D79
:10A430008AE00E94E11B8A8D9B8DAC8DBD8D80933F
:10A440004E0290934F02A0935002B0935102950197
:10A45000A801B501C8010E9442B2882389F080E0BA
:10A460005EDD0E9488168AE994E10E9477162A2D03
:10A470007B2DC8011AC020E070E080EC9FE715C07A
:10A480002A2D7B2DC80111C08A8D9B8DAC8DBD8D71
:10A4900080934E0290934F02A0935002B0935102CA
:10A4A000A12CB12C00EC1FE7DACF822E972E5C0195
:10A4B000C501B401A0960FB6F894DEBF0FBECDBFA4
:10A4C000DF91CF911F910F91FF90EF90DF90CF9090
:10A4D000BF90AF909F908F907F906F905F904F90C4
:10A4E0003F902F900895CF93DF93C2E5D2E048814B
:10A4F00059816A817B8185E295E10E94C2164C8177
:10A500005D816E817F8181E295E10E94C21648855E
:10A5100059856A857B858DE195E10E94C2164C853F
:10A520005D856E857F8589E195E10E94C216DF9188
:10A53000CF910C947C3E2EE532E04AE552E066E590
:10A5400072E082E592E00C943E6D8EE592E00C9410
:10A550008B6DCF93DF9380E00E94B35ECCE9D5E0B2
:10A56000688379838A839B8381E00E94B35E6C83D6
:10A570007D838E839F8382E00E94B35E68877987A4
:10A580008A879B87DF91CF9108951F93CF93DF93A5
:10A59000CDB7DEB760970FB6F894DEBF0FBECDBF64
:10A5A000182FD7DF80919C0590919D05A0919E0565
:10A5B000B0919F0589839A83AB83BC838091A0056A
:10A5C0009091A105A091A205B091A3058D839E83D2
:10A5D000AF83B8878091A4059091A505A091A605A9
:10A5E000B091A70589879A87AB87BC8780915E0267
:10A5F00090915F02A0916002B09161028D879E8769
:10A60000AF87B88BCE0101960E94F85D1E3F51F4D2
:10A6100080E1FE013196A2E5B2E001900D928A95AB
:10A62000E1F716C024E0129FC0011124FC01EE5A8C
:10A63000FD4FA1E0B0E0AC0FBD1FA80FB91F8D9179
:10A640009D910D90BC91A02D80839183A283B383B3
:10A6500060960FB6F894DEBF0FBECDBFDF91CF91ED
:10A660001F910895AF92BF92CF92DF92EF920F9316
:10A670001F93A12CB12C6501E12C8C012EE532E059
:10A680004AE552E066E572E082E592E00E94026CE3
:10A690001F910F91EF90DF90CF90BF90AF900895F2
:10A6A000AF92BF92CF92DF92EF920F931F93CF930F
:10A6B000DF9300D01F92CDB7DEB769837A838B8397
:10A6C0009C83A12CB12C6501E12C8E010F5F1F4FE3
:10A6D00024EB35E040EB55E06CEA75E088EA95E064
:10A6E0000E94026C0F900F900F900F90DF91CF910E
:10A6F0001F910F91EF90DF90CF90BF90AF90089592
:10A700004F925F926F927F928F929F92AF92BF9281
:10A71000CF92DF92EF92FF920F931F93CF93DF932D
:10A72000CDB7DEB72C970FB6F894DEBF0FBECDBF06
:10A730002B013C0129873A874B875C8747015801E9
:10A74000F601E080F1800281138120E030E0A90170
:10A75000B701C8010E9456AF811107C0E0E3F5E1DF
:10A7600085919591A591B49102C0C701D8018D83BF
:10A770009E83AF83B88720E030E0A901B701C8010C
:10A780000E9456AF811108C0E0904802F090490243
:10A7900000914A0210914B02C701D80189839A8324
:10A7A000AB83BC83A501940160915A0270915B0256
:10A7B00080915C0290915D020E9456AF87FF0BC0B2
:10A7C00080925A0290925B02A0925C02B0925D026B
:10A7D000CE01059647DF409252025092530260929A
:10A7E00054027092550289859A85AB85BC85809309
:10A7F000560290935702A0935802B0935902CE018B
:10A80000019630DFA501940160915A0270915B02BC
:10A8100080915C0290915D020E9459B118165CF41F
:10A8200080925A0290925B02A0925C02B0925D020A
:10A83000CE01059617DF0E94C75E2C960FB6F894DE
:10A84000DEBF0FBECDBFDF91CF911F910F91FF9063
:10A85000EF90DF90CF90BF90AF909F908F907F90C0
:10A860006F905F904F900895CF92DF92EF92FF929A
:10A870000F931F936B01FC01E080F1800281138133
:10A88000E2E5F2E024813581468157816081718162
:10A890008281938135DF1F910F91FF90EF90DF90C0
:10A8A000CF900895CF92DF92EF92FF920F931F9374
:10A8B0006A01E0905A02F0905B0200915C021091F4
:10A8C0005D02FB012081318142815381FC01608165
:10A8D00071818281938114DF1F910F91FF90EF901E
:10A8E000DF90CF90089580914E0290914F02A091F9
:10A8F0005002B09151028093980590939905A093CE
:10A900009A05B0939B0580914C0290914D029093D3
:10A9100097058093960584E690E090934D0280938E
:10A920004C0208958091980590919905A0919A05FF
:10A93000B0919B0580934E0290934F02A0935002DA
:10A94000B0935102809196059091970590934D0296
:10A9500080934C020895A82FB0E0CD01880F991F75
:10A96000880F991FFC01E959FA4E4591559165915F
:10A97000749133E0AA0FBB1F3A95E1F7A15DBD4F7B
:10A980004D935D936D937C931397FC01E55AFA4EBA
:10A99000459155916591749114964D935D936D9386
:10A9A0007C9317970895CF92DF92EF92FF92CF9307
:10A9B000DF9320914702222309F485C0EC01C09067
:10A9C0002F02D0903002E0903102F0903202A701C5
:10A9D0009601688179818A819B810E9456AF87FFA9
:10A9E00004C0C882D982EA82FB82C0903302D09030
:10A9F0003402E0903502F0903602A701960168819A
:10AA000079818A819B810E9459B1181624F4C882E9
:10AA1000D982EA82FB82C0903702D0903802E0905F
:10AA20003902F0903A02A70196016C817D818E81F6
:10AA30009F810E9456AF87FF04C0CC82DD82EE82E8
:10AA4000FF82C0903B02D0903C02E0903D02F0902B
:10AA50003E02A70196016C817D818E819F810E94BB
:10AA600059B1181624F4CC82DD82EE82FF82C090A8
:10AA70003F02D0904002E0904102F0904202A701D4
:10AA80009601688579858A859B850E9456AF87FFE8
:10AA900004C0C886D986EA86FB86C0904302D0905F
:10AAA0004402E0904502F0904602A70196016885B5
:10AAB00079858A859B850E9459B1181624F4C88629
:10AAC000D986EA86FB86DF91CF91FF90EF90DF90E9
:10AAD000CF9008958F929F92AF92BF92CF92DF92C4
:10AAE000EF92FF9288EA95E05EDF8091A70383FDF5
:10AAF0007DC0C090B405D090B505E090B605F0904B
:10AB0000B70520915E0230915F0240916002509142
:10AB10006102C701B6010E9456AF882309F466C0DE
:10AB20006091F4047091F5048091F6049091F7041B
:10AB30002091C904211117C00E94C5AF20911F02A6
:10AB4000309120026217730774F4C0925E02D092B3
:10AB50005F02E0926002F09261020E9485168EEF21
:10AB600094E10E9477168090B4059090B505A0906E
:10AB7000B605B090B70520915E0230915F0240911A
:10AB8000600250916102C501B4010E947CAE6B016C
:10AB90007C0120E030E0A9010E9459B187FF04C088
:10ABA000C701B601905802C0C701B60120916202E8
:10ABB0003091630240916402509165020E9494B109
:10ABC00020E030E048E453E40E9459B1181674F4D0
:10ABD00080925E0290925F02A0926002B092610247
:10ABE0000E9485168FED94E10E94771660914C02C9
:10ABF00070914D02072E000C880B990B0E94F8AF44
:10AC000020914E0230914F024091500250915102DA
:10AC10000E9494B12AE037ED43E25CE30E9494B1D4
:10AC20003FDD80E1E8EAF5E0A2E5B2E001900D92B7
:10AC30008A95E1F7FF90EF90DF90CF90BF90AF90B3
:10AC40009F908F9008951F93CF93DF93882329F0CF
:10AC5000D091BA05D095D17001C0D0E0662339F00B
:10AC60001091BA051695117081E0182701C010E007
:10AC7000442341F0C091BA05C2FBCC27C0F981E062
:10AC8000C82701C0C0E0D11104C0111102C0CC23FB
:10AC9000D1F00E94851689ED94E10E947716DD239C
:10ACA00019F088E50E94E11B112319F089E50E9443
:10ACB000E11BCC2319F08AE50E94E11B81ED94E1B0
:10ACC0000E947716C1E08C2FDF91CF911F910895DC
:10ACD000CF92DF92EF92FF92CF93DF93C82FD0E015
:10ACE000FE01E253FB4E8491811107C00E9485163C
:10ACF0008CEA94E10E9477168AE0FE01EE0FFF1FB6
:10AD0000EE0FFF1FE85DFA4EC590D590E590F490E8
:10AD1000682F70E080E090E00E94F8AF9B01AC01EA
:10AD2000C701B6010E945DAFDF91CF91FF90EF9018
:10AD3000DF90CF9008954F925F926F927F928F92A3
:10AD40009F92AF92BF92CF92DF92EF92FF920F93BA
:10AD50001F93CF93DF93CDB7DEB768970FB6F89404
:10AD6000DEBF0FBECDBF2A013B016901E82EF12CE9
:10AD7000F701EC5CFA4EE491AA24A3941E160CF49D
:10AD8000A12CBB24B39420E030E0A901C301B2019F
:10AD90000E9459B118160CF0B12C80E0E4D76983F9
:10ADA0007A838B839C8381E0DED76D837E838F8360
:10ADB000988782E0D8D769877A878B879C8783E0DA
:10ADC000D2D76D877E878F87988BEE0CFF1CEE0C99
:10ADD000FF1C88248394912C8C0E9D1E8E0C9F1C2E
:10ADE000F40110821182128213829E01235F3F4F71
:10ADF000AE01475F5F4FBE016B5F7F4FCE01019693
:10AE00000E94636CF4014082518262827382198ACB
:10AE10001A8A1B8A1C8A20E030E0A901B801C60109
:10AE20000E9456AF811108C0F701E85DFA4E859186
:10AE30009591A591B49102C0C801D6018D8B9E8BCE
:10AE4000AF8BB88FCE0141966C01E12C8E010B5E69
:10AE50001F4F9E01235F3F4FAE01475F5F4FBE0113
:10AE60006B5F7F4F40970E941F6B91D7AB100E9482
:10AE7000073368960FB6F894DEBF0FBECDBFDF91E3
:10AE8000CF911F910F91FF90EF90DF90CF90BF90E7
:10AE9000AF909F908F907F906F905F904F900895AC
:10AEA00041E050E060E070E0082E04C0440F551F00
:10AEB000661F771F0A94D2F79091B905942B90934F
:10AEC000B9059091BA05492B4093BA0524E0829FB9
:10AED000C0011124FC01E15BFA4E45915591659149
:10AEE0007491FC01EE5AFD4F40835183628373835A
:10AEF00008954F925F926F927F928F929F92AF923E
:10AF0000BF92FF920F931F93CF93DF93833008F08C
:10AF10006AC0F82EC82FD0E0FE01EC5CFA4E849196
:10AF2000CC0FDD1FCC0FDD1FFE01ED5BFA4E45900F
:10AF3000559065907490682F880F770B880B990B4C
:10AF40000E94F8AF4B015C0120E030E040EC5FE391
:10AF5000C301B2010E9494B1A50194010E9494B171
:10AF6000AB01BC0100E010E098018F2DE4DEFE0192
:10AF7000E95CFA4E2591359145915491C501B40192
:10AF80000E9494B14B015C0120E030E0A9010E94D5
:10AF900056AF8823C1F0B501A401705800E010E05D
:10AFA00098018F2DC8DE8F2D93DE2B013C01A5016A
:10AFB0009401C501B4010E947DAEAB01BC019301B7
:10AFC00082018F2DB8DE8F2D6BDFB5DAFE01E855DB
:10AFD000FA4FCE5ADD4F88819981AA81BB81808347
:10AFE0009183A283B383DF91CF911F910F91FF9043
:10AFF000BF90AF909F908F907F906F905F904F9099
:10B00000089580E1E0EFF5E0DF01982F1D929A9519
:10B01000E9F7E3ECF5E0DF01982F1D929A95E9F747
:10B02000ECEDF5E0DF011D928A95E9F71092D80565
:10B030001092D9051092DA051092DB058CE096E0AB
:10B040000E9434A81092AC061092AF061092AD0682
:10B050001092AE061092A90608954F925F926F92D9
:10B060007F928F929F92AF92BF92CF92DF92EF9298
:10B07000FF920F931F93CF93DF93CDB7DEB76897FF
:10B080000FB6F894DEBF0FBECDBF8C015B014A0145
:10B09000FC01EF5BFF4F60817181828193810E948F
:10B0A000F6AF6B017C01D5012D913D914D915C91E5
:10B0B0000E9494B10E9443AF0E94CAAF69877A8709
:10B0C0008B879C87F4012081318142815381C701A4
:10B0D000B6010E9494B10E9443AF0E94CAAF6D872F
:10B0E0007E878F87988B29853A854B855C852837A5
:10B0F00031054105510540F488E790E0A0E0B0E05B
:10B1000089879A87AB87BC872D853E854F8558896F
:10B11000283731054105510540F488E790E0A0E06B
:10B12000B0E08D879E87AF87B88B9801235B3F4F38
:10B13000D9018D919D910D90BC91A02D89839A8309
:10B14000AB83BC83BC01CD010E94F8AF2B013C0155
:10B1500069857A858B859C850E94F6AF698B7A8B91
:10B160008B8B9C8B20E030E0A901C301B2010E94CF
:10B1700056AF882329F1A7019601C701B6010E94A5
:10B1800094B14B015C0129893A894B895C89CA01D8
:10B19000B9010E9494B19B01AC01C501B4010E94A8
:10B1A0007CAE4B015C01A3019201C301B2010E947C
:10B1B0007DAE9B01AC01C501B4010E945DAF03C02F
:10B1C00060E070E0CB010E9443AF0E94CAAF6D8384
:10B1D0007E838F83988769817A818B819C8190950A
:10B1E0008095709561957F4F8F4F9F4F0E94F8AF6C
:10B1F0004B015C016D857E858F8598890E94F6AF35
:10B2000069837A838B839C8320E030E0A901C501A8
:10B21000B4010E9456AF882349F129813A814B81BC
:10B220005C81CA01B9010E9494B16D8B7E8B8F8BBA
:10B23000988FA7019601C701B6010E9494B19B01A6
:10B24000AC016D897E898F89988D0E947CAE6B01DF
:10B250007C01A5019401C501B4010E947DAE9B0152
:10B26000AC01C701B6010E945DAF03C060E070E0B1
:10B27000CB010E9433B0F80185A096A0A7A0B0A48E
:10B28000750164012D813E814F815885C21AD30A10
:10B29000E40AF50A0E94CAAFC61AD70AE80AF90AF0
:10B2A000F7FE73C020E030E0A901C301B2010E94A3
:10B2B00056AF882309F443C0A3019201C301B20130
:10B2C0000E947DAE6B017C01C501B4010E94F6AF06
:10B2D0009B01AC01C701B6010E9494B16B017C01D6
:10B2E00029893A894B895C89CA01B9010E9494B1C4
:10B2F0009B01AC01C701B6010E947CAE6B017C01D1
:10B3000029813A814B815C81CA01B9010E9494B1C3
:10B310009B01AC01C701B6010E947DAE6B017C01AF
:10B3200020E030E040E850E4C301B2010E9494B153
:10B330009B01AC01C701B6010E945DAF03C060E094
:10B3400070E0CB010E9443AF7B016C0120E030E054
:10B35000A9010E9459B1181624F0E12CF12CC12C3E
:10B36000D12CB701C6010E94CAAF6D837E838F8343
:10B37000988786169706A806B90620F48D829E82C5
:10B38000AF82B886C12CD12C76018D819E81AF8190
:10B39000B885F80181A792A7A3A7B4A7C80ED91EA4
:10B3A000EA1EFB1EC5A6D6A6E7A6F0AAEB5BFF4FDA
:10B3B00029853A854B855C8520833183428353837D
:10B3C00034968D859E85AF85B88980839183A283CD
:10B3D000B38368960FB6F894DEBF0FBECDBFDF9182
:10B3E000CF911F910F91FF90EF90DF90CF90BF9082
:10B3F000AF909F908F907F906F905F904F90089547
:10B400002F923F924F925F926F927F928F929F9274
:10B41000AF92BF92CF92DF92EF92FF920F931F9362
:10B42000CF93DF93009709F471C08B01EC01D984AD
:10B43000CA847B846C848D809E80AF80B8842D2DDF
:10B440003C2D472D562DC501B4010E9456AF8111E8
:10B4500008C00115110509F459C0F801808180FF69
:10B4600055C0888181FD34C00115110531F0F80106
:10B47000258036804780508408C08BE0282E87EDD9
:10B48000382E83E2482E8BE3582E89899A89AB891E
:10B49000BC89BC01CD0190589B01AC010E947DAEDE
:10B4A0002D853E854F8558890E9494B19B01AC0142
:10B4B000C201B1010E947CAE7B018C019B01AC01F9
:10B4C0006D2D7C2D872D962D0E9456AF87FF04C0D1
:10B4D000ED2CFC2C072D162D9701A801C501B401F8
:10B4E0000E9456AF882391F0888181608883CE01C5
:10B4F0000E940638882321F088818E7F888306C0C9
:10B50000A701B8014D835E836F837887DF91CF9168
:10B510001F910F91FF90EF90DF90CF90BF90AF9071
:10B520009F908F907F906F905F904F903F902F9063
:10B530000895FF920F931F93CF93DF93C091AF06AF
:10B54000C150CF70D091AD068091AF06D817E9F009
:10B5500060E070E086E5F82ECD17B9F0FC9E800122
:10B5600011240055194FF801808183FD03C0C801E3
:10B5700047DFB801C150CF708091AD06D81761F395
:10B58000CD1719F0DF5FDF70F7CFDF91CF911F91FB
:10B590000F91FF9008954F925F926F927F928F92DA
:10B5A0009F92AF92BF92FF920F931F93CF93DF931F
:10B5B000009709F459C0F42EEB018C01FC01808145
:10B5C00081FD3CC045805680678070848D809E8060
:10B5D000AF80B884A5019401C301B2010E9456AFA7
:10B5E00087FF2CC0F80181899289A389B489BC01A5
:10B5F000CD0190589B01AC010E947DAEF8012585DC
:10B600003685478550890E9494B19B01AC01C301E6
:10B61000B2010E947CAE2B013C01A50194010E9465
:10B6200056AF87FF0BC0888181608883CE010E945E
:10B630000638882391F088818E7F888329853A8512
:10B640004B855C856D817E818F8198850E9456AF88
:10B6500081110AC0F092AD0607C04D825E826F82F2
:10B660007886F092AD06EACFDF91CF911F910F91CE
:10B67000FF90BF90AF909F908F907F906F905F9062
:10B680004F900895CF92DF92EF92FF920F931F9306
:10B69000CF93DF931091AD06C0E0D0E086E5C82ED1
:10B6A0008091AF06181709F1C19EB0011124CB019A
:10B6B0008055994F7C01FC01808183FD0AC00E2DCD
:10B6C000DF2C209769F0CE010E940638882341F0D4
:10B6D00002C00C2FDD2E1F5F1F70C02FDD2DE0CFAD
:10B6E000412FB701CE0157DFF6CFDF91CF911F91E8
:10B6F0000F91FF90EF90DF90CF9008952F923F929F
:10B700004F925F926F927F928F929F92AF92BF9271
:10B71000CF92DF92EF92FF920F931F93CF93DF931D
:10B72000CDB7DEB72E970FB6F894DEBF0FBECDBFF4
:10B730002091AC0629873091AF063B8796E58B8533
:10B74000E9858E1759F08B8581508F70989FF00195
:10B750001124E055F94F208123FD0DC0812C912C3F
:10B76000A12CB12C1A861C861D861E86212C312CFC
:10B7700000E010E01AC08B87E2CFF6E52985F29F42
:10B78000C0011124FC01E055F94F1F01808183FFA6
:10B7900011C0FA84EC84DD84CE8489858F5F8F703C
:10B7A0008987FA86EC86DD86CE86F9852B85F213AD
:10B7B000E4CF93C065817681878190850E9401B234
:10B7C000F62EE72ED82EC92E0115110509F47FC0DB
:10B7D000F801808180FD04C0F101808180FF77C085
:10B7E000F801808181608083C8010E940638811140
:10B7F0006AC0F80161817281838194810E9401B2E3
:10B800002B013C019B01AC0160E070E080E89FE30C
:10B810000E945DAF4B015C019B01AC016F2D7E2D41
:10B820008D2D9C2D0E9494B169837A838B839C8398
:10B83000A50194016A857C858D859E850E9494B1C1
:10B840006D837E838F839887AE014F5F5F4FBE010C
:10B850006B5F7F4FC80101DCF80186A9882399F14D
:10B860002091D3053091D4054091D5055091D6054E
:10B87000FD9660817181828193810E9494B12091B3
:10B8800081063091820640918306509184060E9481
:10B8900094B14B015C019B01AC01C301B2010E9458
:10B8A00094B10E94CAAFF80172AF61AFA5019401D3
:10B8B0006F2D7E2D8D2D9C2D0E9494B10E94CAAFBC
:10B8C000F80174AF63AFF80180818E7F80838F2C85
:10B8D0009E2CAD2CBC2C810160CF2114310409F4C5
:10B8E00073C0F101808181608083C8010E940638A5
:10B8F000811166C0F10161817281838194810E940E
:10B9000001B26B017C019B01AC0160E070E080E85A
:10B910009FE30E945DAF2B013C012DEC3CEC4CE41D
:10B920005DE30E9494B169837A838B839C83A30136
:10B930009201B401C5010E9494B16D837E838F830F
:10B940009887AE014F5F5F4FBE016B5F7F4FC101B4
:10B9500084DBF10186A9882399F12091D3053091E8
:10B96000D4054091D5055091D605FD966081718131
:10B97000828193810E9494B1209181063091820648
:10B9800040918306509184060E9494B14B015C0162
:10B990009B01AC01C701B6010E9494B10E94CAAFDD
:10B9A000F10172AF61AF2DEC3CEC4CE45DE3C501FD
:10B9B000B4010E9494B10E94CAAFF10174AF63AFA9
:10B9C000F10180818E7F80832E960FB6F894DEBFC2
:10B9D0000FBECDBFDF91CF911F910F91FF90EF90E0
:10B9E000DF90CF90BF90AF909F908F907F906F909F
:10B9F0005F904F903F902F9008958091AF06909167
:10BA0000AD0681508F70891711F093DD3BDE76CE45
:10BA1000AF92BF92CF92DF92EF92FF920F931F935C
:10BA2000CF939091AF068091AC06981791F0E0917A
:10BA3000AC0686E5E89FF0011124EF5FF84FC08166
:10BA40008091AC069091AF06891729F08F5F8F70B7
:10BA5000F9CFC091EF04CC2339F10E94EF1100918E
:10BA6000BF051091C0052091C1053091C205DC01D0
:10BA7000CB01011511052105310571F48C599F4F3A
:10BA8000AF4FBF4F8093BF059093C005A093C105F2
:10BA9000B093C205CFEF21C0801B910BA20BB30B5B
:10BAA000B7FF1BC0CFEF19C01092BF051092C005A1
:10BAB0001092C1051092C20560E070E020E04FEFE7
:10BAC00050E088E0CF911F910F91FF90EF90DF90B1
:10BAD000CF90BF90AF900C94F5196C2F70E080E080
:10BAE00090E01F921F921F922FEF2F9326E4A22E19
:10BAF000B12CC12CD12CE12CF12C8701EA9421E04E
:10BB000030E040E050E00E94D0150F900F900F9071
:10BB10000F90D4CFCF92DF92EF92FF920F931F93AB
:10BB2000CF93DF93CDB7DEB728970FB6F894DEBF7B
:10BB30000FBECDBF20913006222309F44AC06A010E
:10BB40008B017C0120E030E040E450E4FC016081A6
:10BB50007181828193810E947DAE6D837E838F830C
:10BB600098872DEC3CEC46E353E4F8016081718149
:10BB7000828193810E947CAE69837A838B839C83CC
:10BB80009601AE014F5F5F4FBE016B5F7F4F8CE050
:10BB900096E00E946CA720E030E040E450E46D8124
:10BBA0007E818F8198850E947CAEF70160837183CE
:10BBB000828393832DEC3CEC46E353E469817A81E4
:10BBC0008B819C810E947DAEF801608371838283AA
:10BBD000938328960FB6F894DEBF0FBECDBFDF91DA
:10BBE000CF911F910F91FF90EF90DF90CF9008952C
:10BBF0000F931F93CF93DF93CDB7DEB7AC970FB6FC
:10BC0000F894DEBF0FBECDBF20913006222309F489
:10BC100050C08C016CE076E0CE0101960E94EFA846
:10BC200020E030E040E450E4F801608171818281DD
:10BC300093810E947DAE69A77AA78BA79CA72DEC64
:10BC40003CEC46E353E4F801648175818681978179
:10BC50000E947CAE6DA37EA38FA398A79801285F56
:10BC60003F4FAE014B5D5F4FBE01675D7F4FCE0121
:10BC700001960E946CA720E030E040E450E469A502
:10BC80007AA58BA59CA50E947CAEF8016083718388
:10BC9000828393832DEC3CEC46E353E46DA17EA1BB
:10BCA0008FA198A50E947DAEF80164837583868379
:10BCB0009783AC960FB6F894DEBF0FBECDBFDF9171
:10BCC000CF911F910F91089580916F0081FB99276B
:10BCD00090F981FF05C080916F008D7F80936F0088
:10BCE0008091AC068093AF068093AD068093AE063C
:10BCF00084E68093A90628EE33E03093AB062093C8
:10BD0000AA06992329F080916F00826080936F00CA
:10BD100081E080937E0508950C94353ECF93C82F23
:10BD20000E945E3E0E94F8AF24E0C29FF001112401
:10BD3000EF5BF94F20813181428153810E9494B1A0
:10BD4000CF9108959091AF068091AC06981719F0A5
:10BD50000E94E4ADF7CF8091AA069091AB06892BA3
:10BD6000B9F70C94D8ACCF93C82F0E94173E0E940D
:10BD7000F8AF24E0C29FF0011124EF5BF94F20815E
:10BD80003181428153810E9494B1CF910895909165
:10BD9000AF068091AC06981719F00E94E4ADF7CF7A
:10BDA0008091AA069091AB06892BB9F708952F923E
:10BDB0003F924F925F926F927F928F929F92AF923B
:10BDC000BF92CF92DF92EF92FF920F931F93CF9388
:10BDD000DF93CDB7DEB7CE56D1090FB6F894DEBFEC
:10BDE0000FBECDBF1C01AB966FAFAB976E965FAF2A
:10BDF0004EAF6E9768963FAF2EAF68976596EFAEE1
:10BE000065972C96FFAE2C9769960FAF6997619650
:10BE10001FAF61971C2D2E96BFAEAEAE2E97FA01C6
:10BE200080819181A281B3814091F0055091F1050B
:10BE30006091F2057091F305841B950BA60BB70B6F
:10BE400089A79AA7ABA7BCA784819581A681B78152
:10BE50004091F4055091F5056091F6057091F70554
:10BE6000841B950BA60BB70B8DA39EA3AFA3B8A7FE
:10BE700080859185A285B3854091F8055091F9059B
:10BE80006091FA057091FB05841B950BA60BB70B0F
:10BE900089A39AA3ABA3BCA3C484D584E684F78406
:10BEA0008091FC059091FD05A091FE05B091FF05E4
:10BEB000A7019601281B390B4A0B5B0B2BAB3CAB44
:10BEC0004DAB5EAB232B242B252B09F496C0609140
:10BED000F4047091F5048091F6049091F704209198
:10BEE000C90421112BC00E94C5AF20911F023091BF
:10BEF00020026217730714F5C092FC05D092FD056D
:10BF0000E092FE05F092FF056896EEADFFAD6897F2
:10BF100084859585A685B7858093CF059093D005B8
:10BF2000A093D105B093D2050E94851682E995E1D0
:10BF30000E9477161BAA1CAA1DAA1EAA6BA97CA97F
:10BF40008DA99EA90E94F8AF24E0129FF001112450
:10BF5000EE59FD4F20813181428153810E9494B17D
:10BF60006B017C0120E030E0A9010E9459B187FFFC
:10BF700004C0F7FAF094F7F8F09420E030E048E4D9
:10BF800053E46091810670918206809183069091BE
:10BF900084060E9494B19B01AC01C701B6010E94C6
:10BFA00059B1181654F56E96EEADFFAD6E978485B7
:10BFB0009585A685B7858093FC059093FD05A09394
:10BFC000FE05B093FF056896EEADFFAD68978485DA
:10BFD0009585A685B7858093CF059093D005A093CE
:10BFE000D105B093D2050E94851683E795E10E94A2
:10BFF00077161BAA1CAA1DAA1EAA49A45AA46BA4A0
:10C000007CA4D301C2018827B7FD83959927AA276D
:10C01000BB27082F8DA09EA0AFA0B8A4B7FC0260DC
:10C02000C9A0DAA0EBA0FCA0F7FC04602BA93CA9F6
:10C030004DA95EA957FD08606BA97CA98DA99EA991
:10C040000E94F8AF34E0139FF0011124EE59FD4F28
:10C0500020813181428153810E9494B16FA778ABD6
:10C0600089AB9AAB20E030E0A9010E9459B187FF6B
:10C0700006C06FA578A989A99AA9905804C06FA590
:10C0800078A989A99AA920E030E040E05FE30E9406
:10C090007DAE0E94CAAF2B966CAF7DAF8EAF9FAFC7
:10C0A0002B97D1011C92D5960C934FAA58AE69AE2E
:10C0B0007AAE77FE0BC022273327A9012419350950
:10C0C000460957092FAB38AF49AF5AAF8FA998AD82
:10C0D000A9ADBAADF101858B968BA78BB08F239656
:10C0E0008CAE9DAEAEAEBFAE2397B7FE0DC022277D
:10C0F0003327A901281939094A095B0923962CAF6E
:10C100003DAF4EAF5FAF239723968CAD9DADAEADE7
:10C11000BFAD2397F101818F928FA38FB48F2796A4
:10C12000CCAEDDAEEEAEFFAE2797F7FE0DC02227F8
:10C130003327A9012C193D094E095F0927962CAF19
:10C140003DAF4EAF5FAF279727968CAD9DADAEAD9F
:10C15000BFAD2797F101858F968FA78FB0A3C3013D
:10C16000B2010E94F8AF2091410630914206409101
:10C170004306509144060E9494B16BAF7CAF8DAFE3
:10C180009EAF698B7A8B8B8B9C8BC501B4010E940F
:10C19000F8AF2091450630914606409147065091F0
:10C1A00048060E9494B12B013C016D8B7E8B8F8BD6
:10C1B000988FC701B6010E94F8AF209149063091CF
:10C1C0004A0640914B0650914C060E9494B14B0197
:10C1D0005C01698F7A8F8B8F9C8F20914D063091F7
:10C1E0004E0640914F06509150066FA578A989A937
:10C1F0009AA90E9494B16B017C016D8F7E8F8F8F05
:10C2000098A32FA938AD49AD5AAD26303105410567
:10C21000510554F523968CAD9DADAEADBFAD2397C2
:10C220000697A105B10504F527962CAD3DAD4EADA1
:10C230005FAD27972630310541055105ACF420E06C
:10C2400030E0A901C701B6010E9459B187FF04C0BF
:10C25000F7FAF094F7F8F094D1011D96CD92DD92A3
:10C26000ED92FC92509752C02E96EEADFFAD2E97F8
:10C27000C080D180E280F38020E030E0A901C701D6
:10C28000B6010E9456AF882341F0D1011D96CD9290
:10C29000DD92ED92FC9250972BC02BAD3CAD4DAD95
:10C2A0005EADCA01B9010E9494B16B017C01A3018A
:10C2B0009201C301B2010E9494B19B01AC01C7017C
:10C2C000B6010E947DAE6B017C01A5019401C50100
:10C2D000B4010E9494B19B01AC01C701B6010E9458
:10C2E0007DAE0E9401B2F101658776878787908BCA
:10C2F00071019E012F5D3F4FAE014B5D5F4FBE014F
:10C30000675D7F4F86E694E00E94FA1D2B96CCACC9
:10C31000DDACEEACFFAC2B97D1019196CD92DD92C6
:10C32000ED92FC92949755964D915D916D917C9113
:10C3300058975D96CD90DD90ED90FC909097599632
:10C340008D919D910D90BC91A02D8C159D05AE05F4
:10C35000BF0510F4D701C60184179507A607B707D4
:10C3600010F4DB01CA012B96CCACDDACEEACFFAC1B
:10C370002B978C159D05AE05BF0510F4D701C6019E
:10C38000F10185A396A3A7A3B0A70697A105B105C0
:10C39000B0F18091EF04EF5AFF4F8083452B462B7D
:10C3A000472B09F01798F101818D928DA38DB48DE3
:10C3B000892B8A2B8B2B09F01698F101858D968D90
:10C3C000A78DB0A1892B8A2B8B2B09F015982B9662
:10C3D000CCACDDACEEACFFAC2B97CD28CE28CF2873
:10C3E000D1F08091D705882319F081508093D7052B
:10C3F000111108C0149880E28093D70503C080E033
:10C400000C94406AE090A106F090A2060091A30669
:10C410001091A40608C0E090A506F090A606009131
:10C42000A7061091A8069701A80165966FAD6597BC
:10C430002C967FAD2C9769968FAD699761969FADCD
:10C4400061970E9456AF87FD02C00C94326AD101F9
:10C450001D962D913D914D915C9150976C962CAF0E
:10C460003DAF4EAF5FAF6C9760E070E080E89FE358
:10C470000E945DAF60966CAF7DAF8EAF9FAF60974F
:10C480009B01AC01B701C8010E9494B14B015C0152
:10C490008091AF069091AE06891B8F702C968FAF5E
:10C4A0002C97A501940160E074E284E799E40E946E
:10C4B0005DAF0E9464B16B017C012C968FAD2C970F
:10C4C00082508630C0F58091710690917206A091DD
:10C4D0007306B0917406C816D906EA06FB0658F52D
:10C4E0008C199D09AE09BF09BC01CD01660F771FEC
:10C4F000881F991F2C96BFAD2C970B2F10E020E0C2
:10C5000030E0A90198010E9494B2CA01B9010E94C9
:10C51000F6AF0E9464B16C0D7D1D8E1D9F1D0E94A3
:10C52000F6AF9B01AC0160E074E284E799E40E94FD
:10C530005DAF4B015C01A50194016C966CAD7DADC6
:10C540008EAD9FAD6C970E9494B19B01AC010E948F
:10C5500094B1A2966CAF7DAF8EAF9FAFA297F10161
:10C560006183728383839483C5A0D6A0E7A0F0A4DF
:10C570002396CCAEDDAEEEAEFFAE2397C701B6017B
:10C580000E94F6AF27966CAF7DAF8EAF9FAF279717
:10C59000A50194010E9494B10E9443AF0E94CAAFCA
:10C5A000A6966CAF7DAF8EAF9FAFA697F101EF5B04
:10C5B000FF4F6083718382839383FE017196FCAF8A
:10C5C000EBAF9E012F5F3F4F66963FAF2EAF669752
:10C5D00045E856E0A8965FAF4EAFA897CE0181968A
:10C5E0009EA78DA762963FAF2EAF62971FA61FAA88
:10C5F00000E81FE3ABADBCAD6D917D918D919D9138
:10C60000BCAFABAFA50194010E9494B16B017C015A
:10C610006296EEADFFAD62976193719381939193B2
:10C620006296FFAFEEAF629720E030E0A9010E9472
:10C6300059B187FF04C0F7FAF094F7F8F094A89680
:10C64000AEADBFADA8974D905D906D907D90A896D2
:10C65000BFAFAEAFA897A3019201C701B6010E9478
:10C6600059B11816A4F4A7019601C301B2010E94A2
:10C670005DAF6B017C019B01AC016FA57FA9C80177
:10C680000E9459B118161CF4CFA6DFAA8701CBACC3
:10C69000DCACEDA4FEA4CE14DF0409F0ABCF20E0A7
:10C6A00030E040E85FE36FA57FA9C8010E9456AF64
:10C6B00087FF4BC06E0121E1C20ED11C6696EEAC25
:10C6C000FFAC66972FA53FA9A801D7016D917D9179
:10C6D0008D919C910E9494B1F70161937193819324
:10C6E00091937F01EC15FD0569F77101F1E4EF0EFF
:10C6F000F11CA6966CAD7DAD8EAD9FADA6970E9448
:10C70000F6AF2FA53FA9A8010E9494B10E94CAAF1D
:10C71000D7016D937D938D939C9313972FA53FA97C
:10C72000A8016FA57FA9C8010E9494B19B01AC012B
:10C73000A2966CAD7DAD8EAD9FADA2970E9494B1D7
:10C74000F101618372838383948360962CAD3DAD48
:10C750004EAD5FAD609727966CAD7DAD8EAD9FAD54
:10C7600027970E9494B16BAF7CAF8DAF9EAFD10184
:10C7700055968D909D90AD90BC9058975D96CD90BC
:10C78000DD90ED90FC909097CFA6D8AAE9AAFAAADE
:10C790005996CD90DD90ED90FC905C97CFAAD8AEE5
:10C7A000E9AEFAAE81149104A104B10401F5CD28DB
:10C7B000CE28CF28E1F4CFA4D8A8E9A8FAA8CD289C
:10C7C000CE28CF28A1F42091990630919A06409165
:10C7D0009B0650919C060E9494B10E9443AF0E9418
:10C7E000CAAF2B013C01D101D6961C9208C32B96EF
:10C7F000CCACDDACEEACFFAC2B97CD28CE28CF284F
:10C8000049F06091950670919606809197069091F7
:10C81000980608C060919D0670919E0680919F06C3
:10C820009091A0062BAD3CAD4DAD5EAD0E9494B194
:10C830000E9443AF0E94CAAF2B013C012B96CCACA7
:10C84000DDACEEACFFAC2B97CD28CE28CF28C9F0BD
:10C8500020E030E0A9016091D3057091D40580916A
:10C86000D5059091D6050E9456AF882351F081E0FE
:10C87000CBA8DCA8EDA8FEA81C141D041E041F04F0
:10C880000CF080E0D101D6968C93882309F4CAC0BD
:10C890002091C3053091C4054091C5055091C6054E
:10C8A0006896EEADFFAD689760817181828193815A
:10C8B0000E947CAE6BAB7CAB8DAB9EAB2091C70571
:10C8C0003091C8054091C9055091CA056896AEAD32
:10C8D000BFAD689714966D917D918D919C9117973E
:10C8E0000E947CAE2B966CAF7DAF8EAF9FAF2B9727
:10C8F0002091CB053091CC054091CD055091CE05CE
:10C900006896EEADFFAD68976085718582859385E9
:10C910000E947CAE6B017C012BA93CA94DA95EA9AC
:10C92000CA01B9010E9494B16BAB7CAB8DAB9EABDD
:10C930002B962CAD3DAD4EAD5FAD2B97CA01B90125
:10C940000E9494B19B01AC016BA97CA98DA99EA901
:10C950000E947DAE6BAB7CAB8DAB9EABA70196010D
:10C96000C701B6010E9494B19B01AC016BA97CA9DF
:10C970008DA99EA90E947DAE0E9401B26B017C012F
:10C980002091CF053091D0054091D1055091D2052D
:10C990006896AEADBFAD68971C966D917D918D91F7
:10C9A0009C911F970E947CAEA70196010E945DAFEB
:10C9B0006B017C01F101FD96608371838283938317
:10C9C00020E030E040E450E40E9459B118161CF415
:10C9D000F10116AA27C02091D3053091D4054091CA
:10C9E000D5055091D605C701B6010E9494B19B01AF
:10C9F000AC0160913D0670913E0680913F0690919A
:10CA000040060E945DAF2BAD3CAD4DAD5EAD0E94CA
:10CA100094B10E94CAAF641575058605970510F498
:10CA20002B013C018091EC059091ED05A091EE0564
:10CA3000B091EF05F101C1A0D2A0E3A0F4A0CBAA70
:10CA4000DCAAEDAAFEAA2396CCACDDACEEACFFAC22
:10CA500023978C159D05AE05BF0508F4D1C0811440
:10CA60009104A104B10431F1209151063091520694
:10CA70004091530650915406241535054605570537
:10CA8000C8F4C701B6010E945EB26B017C01A3012C
:10CA90009201C501B4010E945EB2C616D706E8062F
:10CAA000F90640F4C701B601A50194010E9494B2B1
:10CAB00029013A01CFA8D8ACE9ACFAACCD28CE28F0
:10CAC000CF2871F1209155063091560640915706B6
:10CAD00050915806241535054605570508F5239647
:10CAE0006CAD7DAD8EAD9FAD23970E945EB26B01A4
:10CAF0007C01A30192016FA978AD89AD9AAD0E9426
:10CB00005EB2C616D706E806F90650F4C701B601AC
:10CB10002FA938AD49AD5AAD0E9494B229013A010E
:10CB2000CFA4D8A8E9A8FAA8CD28CE28CF2871F19B
:10CB30002091590630915A0640915B0650915C064F
:10CB4000241535054605570508F523966CAD7DADD2
:10CB50008EAD9FAD23970E945EB26B017C01A30155
:10CB600092016FA578A989A99AA90E945EB2C616FA
:10CB7000D706E806F90650F4C701B6012FA538A973
:10CB800049A95AA90E9494B229013A01CBA8DCA86C
:10CB9000EDA8FEA8CD28CE28CF2809F430C12091D9
:10CBA0005D0630915E0640915F0650916006241547
:10CBB00035054605570508F022C123966CAD7DADBD
:10CBC0008EAD9FAD23970E945EB26B017C01A301E5
:10CBD00092016BA97CA98DA99EA90E945EB2C6167E
:10CBE000D706E806F90608F00AC1C701B6012BA965
:10CBF0003CA94DA95EA90E9494B229013A01FFC047
:10CC000081149104A104B104B9F1609151067091AD
:10CC10005206809153069091540664157505860559
:10CC2000970550F50E94F6AF27962CAD3DAD4EAD61
:10CC30005FAD27970E9494B16B017C01C501B401DF
:10CC40000E94F6AF4B015C01C301B2010E94F6AF36
:10CC5000A50194010E9494B1A70196010E9459B1C7
:10CC6000181654F4A5019401C701B6010E945DAFE6
:10CC70000E94CAAF2B013C01CFA8D8ACE9ACFAACFA
:10CC8000CD28CE28CF28C9F160915506709156065F
:10CC9000809157069091580664157505860597058D
:10CCA00060F50E94F6AF27962CAD3DAD4EAD5FAD61
:10CCB00027970E9494B16B017C016FA978AD89AD73
:10CCC0009AAD0E94F6AF4B015C01C301B2010E9414
:10CCD000F6AFA50194010E9494B1A70196010E94AC
:10CCE00059B1181654F4A5019401C701B6010E9468
:10CCF0005DAF0E94CAAF2B013C01CFA4D8A8E9A820
:10CD0000FAA8CD28CE28CF28C9F160915906709194
:10CD10005A0680915B0690915C0664157505860540
:10CD2000970560F50E94F6AF27962CAD3DAD4EAD50
:10CD30005FAD27970E9494B16B017C016FA578A924
:10CD400089A99AA90E94F6AF4B015C01C301B20107
:10CD50000E94F6AFA50194010E9494B1A70196012B
:10CD60000E9459B1181654F4A5019401C701B601E7
:10CD70000E945DAF0E94CAAF2B013C01CBA8DCA88A
:10CD8000EDA8FEA8CD28CE28CF28C9F160915D0678
:10CD900070915E0680915F0690916006641575053E
:10CDA0008605970560F50E94F6AF27962CAD3DAD40
:10CDB0004EAD5FAD27970E9494B16B017C016BA9CA
:10CDC0007CA98DA99EA90E94F6AF4B015C01C3010D
:10CDD000B2010E94F6AFA50194010E9494B1A7018F
:10CDE00096010E9459B1181654F4A5019401C70187
:10CDF000B6010E945DAF0E94CAAF2B013C01F10158
:10CE0000E35BFF4F4082518262827382C301B201B1
:10CE10000E94F6AF6B017C012BAD3CAD4DAD5EAD1C
:10CE20000E945DAF64966CAF7DAF8EAF9FAF64978D
:10CE3000D10151966D937D938D939C9354972DEBD7
:10CE400037E346E051E4C701B6010E9494B10E9465
:10CE5000CAAFF10161AB72AB83AB94AB86A98823F7
:10CE600081F1FD9620813181428153816091D3050A
:10CE70007091D4058091D5059091D6050E9494B10A
:10CE800064962CAD3DAD4EAD5FAD64970E9494B1FC
:10CE9000209181063091820640918306509184064C
:10CEA0000E9494B19B01AC0160E074E284EF99E4CC
:10CEB0000E945DAF0E94CAAFD101D8967C936E9359
:10CEC000D797D1011196CD90DD90ED90FC901497FD
:10CED000A296CCAEDDAEEEAEFFAEA297C701B60114
:10CEE0000E9401B26FAB28967FAF28978FAF249630
:10CEF0009FAF2497E1E3F6E0A496FFAFEEAFA497CF
:10CF00003E01F1E16F0E711C21E336E02E963FAF3A
:10CF10002EAF2E9766964EAC5FAC66976BAB7FA735
:10CF2000182F092F1BAED201CD90DD90ED90FD9012
:10CF30002D0120E030E0A901C701B6010E9459B1DE
:10CF400087FF04C0F7FAF094F7F8F0942E96EEAD50
:10CF5000FFAD2E9781909190A190B1902E96FFAF4A
:10CF6000EEAF2E97A5019401C701B6010E9459B1F9
:10CF700018160CF043C0FBADFF2349F1A501940145
:10CF80006FA928967FAD28978FAD24969FAD2497E3
:10CF90000E9494B14B015C012BA93FA5412F502F5A
:10CFA000C701B6010E9494B1A50194010E9459B134
:10CFB000181614F5A7019601C501B4010E945DAFD2
:10CFC0006BAB7FA7182F092F21E02BAF17C0A7014C
:10CFD0009601C501B4010E945DAF9B01AC016BA934
:10CFE0007FA5812F902F0E9494B16BAB7FA7182F44
:10CFF000092F31E03BAF02C041E04BAF461457046C
:10D0000009F091CFCBA8AC96CFAEAC97DFA4AD968C
:10D01000DFAEAD97AE961FAFAE97AF960FAFAF979F
:10D020002C96EFAC2C97EE2009F475C1C090D80572
:10D03000D090D905E090DA05F090DB052DEB37E3D1
:10D0400046E855E3C701B6010E9456AF87FD63C1AC
:10D05000C701B6010E9401B26B017C019B01AC01CA
:10D060006FA928967FAD28978FAD24969FAD249702
:10D070000E9456AF87FD08C0CFAA2896DFAE28973A
:10D08000EFAE2496FFAE24979601A7016FA92896CC
:10D090007FAD28978FAD24969FAD24970E945DAFFA
:10D0A000AA966CAF7DAF8EAF9FAFAA972CED35E0FF
:10D0B0002E963FAF2EAF2E97C12CD12C80E8E82EB4
:10D0C0008FE3F82ECBAEDCAEEDAEFEAE2C961FAEEF
:10D0D0002C972E96AEADBFAD2E976D917D918D9113
:10D0E0009D912E96BFAFAEAF2E97AA962CAD3DADBB
:10D0F0004EAD5FADAA970E9494B16B017C0166961C
:10D10000EEADFFAD669781909190A190B19066963B
:10D11000FFAFEEAF66972C96FFAD2C97FF2391F0F3
:10D120002BAD3CAD4DAD5EAD0E9494B16B017C0169
:10D130002BAD3CAD4DAD5EADC501B4010E9494B1C7
:10D140004B015C01A5019401C701B6010E9459B1D0
:10D1500020E030E0A90118164CF5C501B4010E9489
:10D1600059B118164CF020E030E0A901C701B60112
:10D170000E9456AF87FF09C0A5019401C701B601FF
:10D180000E947CAE2B013C0139C02401350177FAA5
:10D19000709477F87094A3019201C701B6010E94C0
:10D1A00059B118165CF52601370128C0C501B40134
:10D1B0000E9456AF87FD09C020E030E0A901C701F9
:10D1C000B6010E9459B118164CF4A7019601C50189
:10D1D000B4010E947CAE2B013C0110C02601370136
:10D1E00077FA709477F87094A5019401C301B201A5
:10D1F0000E9459B1181614F024013501A496AEAD61
:10D20000BFADA497CD90DD90ED90FD90A496BFAFFB
:10D21000AEAFA497A7019601C301B2010E9459B114
:10D220001816CCF4A3019201C701B6010E945DAFAC
:10D230009B01AC016BAD7CAD8DAD9EAD0E9494B1F8
:10D240006BAF7CAF8DAF9EAF2C96BFAD2C97BF5F01
:10D250002C96BFAF2C972E96EEADFFAD2E97EC5EC1
:10D26000F54009F036CF2C96CFAC2C97CC20B1F0FE
:10D270002BAD3CAD4DAD5EAD6FA928967FAD289727
:10D280008FAD24969FAD24970E9494B16FAB2896E2
:10D290007FAF28978FAF24969FAF249724EA30E77B
:10D2A0004DE75FE36FA928967FAD28978FAD249651
:10D2B0009FAD24970E9494B16B017C019B01AC014E
:10D2C0006091BB057091BC058091BD059091BE0534
:10D2D0000E9459B11816ACF4A70196016BA97FA55D
:10D2E000812F902F0E9459B11816ACF0FFA8FBAA0D
:10D2F0002896CFAC2897CFA61FAD24960FAD2497C4
:10D300000AC0DFA8DBAA2896EFAC2897EFA61FADCE
:10D3100024960FAD2497AC968FADAC97AD969FAD8C
:10D32000AD97AE96AFADAE97AF96BFADAF978093CA
:10D33000BB059093BC05A093BD05B093BE052BA97A
:10D340003FA5412F502F6BA97FA5812F902F0E94C1
:10D3500094B17B018C01CB01D801F10181879287C7
:10D36000A387B48764966CAD7DAD8EAD9FAD649799
:10D3700090589B01AC010E947DAE6C962CAD3DADEA
:10D380004EAD5FAD6C970E9494B19B01AC016BE018
:10D3900077ED83E29BE30E947CAE5B016C01AB9670
:10D3A000FFADAB97FF2361F09B01AC01B701C80152
:10D3B0000E9456AF87FD09C09A2D8B2D860107C0AC
:10D3C0009BE087ED03E21BE302C09E2D8F2D492FCA
:10D3D000582FB801D10115964D935D936D937C93B1
:10D3E00018971C919501A601A2966CAD7DAD8EADEE
:10D3F0009FADA2970E9456AF181614F481E001C0A9
:10D4000083E0182BF101108380E1FE013196ACED31
:10D41000B5E001900D928A95E1F7F1018181928149
:10D42000A381B4818093D8059093D905A093DA05A0
:10D43000B093DB0580E16E96EEADFFAD6E97A0EF89
:10D44000B5E001900D928A95E1F780E16896EEAD26
:10D45000FFAD6897A3ECB5E001900D928A95E1F7D6
:10D4600081E00EC06596EFAC65972C96FFAC2C97CB
:10D4700069960FAD699761961FAD61970C9427620D
:10D48000C259DF4F0FB6F894DEBF0FBECDBFDF919C
:10D49000CF911F910F91FF90EF90DF90CF90BF90B1
:10D4A000AF909F908F907F906F905F904F903F9044
:10D4B0002F9008956F927F928F929F92AF92BF921A
:10D4C000CF92DF92EF92FF920F931F93CF93DF9350
:10D4D00000D01F92CDB7DEB74C013B018091AA0668
:10D4E0009091AB06892BD9F59091AF068091AC064F
:10D4F000981B9F709F3059F429833A834B835C8338
:10D500000E94E4AD5C814B813A812981EDCFD090BE
:10D51000AF068091AF0666E5869FC00111245701D2
:10D52000C02E79018A019301A40160E08055994FD2
:10D530000E94D75E8823A9F02091AF069091AC0697
:10D54000291303C094E69093A90691E09D0D9F7066
:10D550009093AF0689830E94FD5C898103C080E0BF
:10D5600001C081E00F900F900F900F90DF91CF914D
:10D570001F910F91FF90EF90DF90CF90BF90AF90F1
:10D580009F908F907F906F9008958091AF069091BB
:10D59000AC06891B8F708F3019F40E94E4ADF5CF73
:10D5A0008091AF068F5F8F70E091AF0696E59E9FEA
:10D5B000F0011124E055F94FDF011D929A95E9F72A
:10D5C00098E090834091F0055091F1056091F2054B
:10D5D0007091F305458B568B678B708F4091F405E6
:10D5E0005091F5056091F6057091F705418F528FC6
:10D5F000638F748F4091F8055091F9056091FA0599
:10D600007091FB05458F568F678F70A34091FC0585
:10D610005091FD056091FE057091FF0541A352A355
:10D6200063A374A32091AF069091AC06291303C0A5
:10D6300094E69093A9068093AF060C94E7342F925A
:10D640003F924F925F926F927F928F929F92AF9292
:10D65000BF92CF92DF92EF92FF920F931F93CF93DF
:10D66000DF93CDB7DEB7A9970FB6F894DEBF0FBE34
:10D67000CDBFF801A091AA06B091AB06AB2B09F083
:10D68000A7C016010E2DF8A7EFA33EA32DA36A0194
:10D690007B01FC014080518062807380209175067F
:10D6A000309176064091770650917806C301B20119
:10D6B0000E9494B10E9464B1698B7A8B8B8B9C8B96
:10D6C000D7018D909D90AD90BC90209179063091BE
:10D6D0007A0640917B0650917C06C501B4010E94F8
:10D6E00094B10E9464B16D8B7E8B8F8B988FD60125
:10D6F0002D913D914D915C9129A33AA34BA35CA33D
:10D7000020917D0630917E0640917F0650918006E3
:10D7100069A17AA18BA19CA10E9494B10E9464B1DD
:10D72000698F7A8F8B8F9C8FEDA1FEA1C080D180F5
:10D73000E280F38020918106309182064091830639
:10D7400050918406C701B6010E9494B10E9464B151
:10D750006D8F7E8F8F8F98A349825A826B827C82D5
:10D760008D829E82AF82B88629A13AA14BA15CA18D
:10D7700029873A874B875C87CD86DE86EF86F88AD5
:10D780002091A70323FF10C06093FC057093FD0553
:10D790008093FE059093FF05C092CF05D092D005EF
:10D7A000E092D105F092D205AFA1B8A52D913D919F
:10D7B0004D915C917101BE016F5F7F4FCE0141962B
:10D7C00079DE882331F089A70E94E73489A501C05A
:10D7D00080E0A9960FB6F894DEBF0FBECDBFDF91F3
:10D7E000CF911F910F91FF90EF90DF90CF90BF905E
:10D7F000AF909F908F907F906F905F904F903F90F1
:10D800002F900895AF92BF92CF92DF92EF920F9335
:10D810001F93CF93DF93CDB7DEB764970FB6F8941D
:10D82000DEBF0FBECDBFA98ABA8ACB8ADC8AFC01D3
:10D8300080819181A281B38189839A83AB83BC83E8
:10D84000FB0180819181A281B3818D839E83AF830F
:10D85000B887FA0180819181A281B38189879A87F3
:10D86000AB87BC87F90180819181A281B3818D87CB
:10D870009E87AF87B88BAE01475F5F4FBE016B5F7E
:10D880007F4FCE0101960E948A5DCE0141966C01C8
:10D890009E01235F3F4FAE01475F5F4FBE016B5F4D
:10D8A0007F4F4097CCDE64960FB6F894DEBF0FBE74
:10D8B000CDBFDF91CF911F910F91EF90DF90CF906F
:10D8C000BF90AF9008958F929F92AF92BF92EF92C8
:10D8D000FF920F931F93CF93DF937B018A01E9019E
:10D8E000FC0180809180A280B380209175063091E8
:10D8F00076064091770650917806C501B4010E94E2
:10D9000094B10E9464B16093F0057093F105809327
:10D91000F2059093F3052091790630917A064091B3
:10D920007B0650917C06F701608171818281938131
:10D930000E9494B10E9464B16093F4057093F50560
:10D940008093F6059093F70520917D0630917E0631
:10D9500040917F0650918006F8016081718182813B
:10D9600093810E9494B10E9464B16093F805709312
:10D97000F9058093FA059093FB052091810630917B
:10D9800082064091830650918406688179818A815C
:10D990009B810E9494B10E9464B16093FC057093D6
:10D9A000FD058093FE059093FF058092C30590923C
:10D9B000C405A092C505B092C605F701808191818A
:10D9C000A281B3818093C7059093C805A093C90530
:10D9D000B093CA05F80180819181A281B3818093BF
:10D9E000CB059093CC05A093CD05B093CE0588814F
:10D9F0009981AA81BB818093CF059093D005A09394
:10DA0000D105B093D2059091AF068091AC069817DE
:10DA100059F0DF91CF911F910F91FF90EF90BF9040
:10DA2000AF909F908F90B1CD0E94C75E80916F00A4
:10DA300081FBCC27C0F981FF05C080916F008D7FED
:10DA400080936F002CEF35E048EF55E064EF75E010
:10DA500080EF95E00E941A38CC2329F080916F0066
:10DA6000826080936F00DF91CF911F910F91FF90A3
:10DA7000EF90BF90AF909F908F900895CF93DF93DA
:10DA8000CDB7DEB760970FB6F894DEBF0FBECDBF3F
:10DA9000FC0180819181A281B38189839A83AB83C8
:10DAA000BC83FB0180819181A281B3818D839E83A0
:10DAB000AF83B887FA0180819181A281B381898780
:10DAC0009A87AB87BC87F90180819181A281B3815C
:10DAD0008D879E87AF87B88BAE01475F5F4FBE01D2
:10DAE0006B5F7F4FCE0101960E948A5D9E01235F8E
:10DAF0003F4FAE01475F5F4FBE016B5F7F4FCE016F
:10DB00000196E1DE60960FB6F894DEBF0FBECDBF82
:10DB1000DF91CF910895CF92DF92EF92FF92FC01B7
:10DB2000C080D180E280F38020918106309182060E
:10DB30004091830650918406C701B6010E9494B1BA
:10DB40000E9464B16093FC057093FD058093FE050F
:10DB50009093FF05C092CF05D092D005E092D105F9
:10DB6000F092D2059091AF068091AC06981729F0FB
:10DB7000FF90EF90DF90CF9008CD0E94C75E80911C
:10DB80006F0081FB992790F981FF05C080916F009C
:10DB90008D7F80936F004091FC055091FD05609151
:10DBA000FE057091FF054093210550932205609377
:10DBB000230570932405992329F080916F008260DA
:10DBC00080936F00FF90EF90DF90CF900895CF92F9
:10DBD000DF92EF92FF920F931F93CF93DF93C1E6F3
:10DBE000D6E001E516E0C12CD12C7601C3946991F1
:10DBF0007991899199910E94F6AF288939894A894A
:10DC00005B890E9494B10E94CAAFF801619371933D
:10DC1000819391938F01C616D706E806F90610F492
:10DC20006B017C01F6E0C137DF0709F76FEF7FEF8B
:10DC3000CB01A70196010E9494B22093EC0530938A
:10DC4000ED054093EE055093EF05DF91CF911F91C5
:10DC50000F91FF90EF90DF90CF9008950F931F9357
:10DC6000CF93DF9305E716E0C1E4D6E0F8012191F8
:10DC70003191419151918F0160E070E080E89FE324
:10DC80000E945DAF6993799389939993F6E0C135CA
:10DC9000DF0761F72EE532E04AE552E066E572E023
:10DCA00082E592E0EBDEDF91CF911F910F918FCF54
:10DCB00080E19CE00C94015881548A3108F041C005
:10DCC000A82FB0E04091390C50913A0C60913B0C78
:10DCD00070913C0C04C076956795579547958A9549
:10DCE000D2F740FF2EC0E091440CF091450CA15EAC
:10DCF000B34F8C918823E9F0E80FF11D808190EDFE
:10DD0000980F9A3098F08E3211F481810CC08D32C8
:10DD100011F08B3271F4818190ED980F9A3030F0D0
:10DD20008E3239F4828180538A3018F49E2F8F2FDF
:10DD300002C090E080E09093400C8093410C81E021
:10DD4000089580E00895B8DF882341F081E02091B4
:10DD5000400C3091410C232B09F480E008950F937F
:10DD60001F93CF938091400C9091410C009711F13B
:10DD7000FC018F01C1912C2F2F7DA9F0C53411F02A
:10DD8000C536B9F7F801108260E070E08091400C70
:10DD90009091410C0E94F9B2F801C083562F472F91
:10DDA000382F292F0BC060E070E0CF911F910F91A9
:10DDB0000C94F9B250E040E030E020E0652F742F81
:10DDC000832F922FCF911F910F9108958091400C36
:10DDD0009091410C009731F04AE050E060E070E033
:10DDE0000C945FB460E070E0CB010895CF9384E5BC
:10DDF000AADF882359F1EADF97FD24C0E7DF6F3FF0
:10DE000071058105910509F0FCF4E0DFC62F1616B7
:10DE1000FCF40E9485168DE40E94E11B6AE070E02C
:10DE200080913D0C90913E0C0E94D41C6C2FCC0F25
:10DE3000770B85E096E10E94A8168AE00E94E11B1C
:10DE40008FEF07C0C0E004C0CFEF02C080E001C088
:10DE50008C2FCF910895BF92CF92DF92EF92FF92D5
:10DE60000F931F93CF93DF9388EAE82E85E0F82E77
:10DE700002E512E096E1C92E9CE0D92ECBE4D3E076
:10DE8000BC2E84E0B80E89915EDF8823B1F067DF95
:10DE9000F6012081211104C02091B805222339F018
:10DEA000F80120813181428153810E947DAEF701CA
:10DEB00060837183828393830AC0F801808191819A
:10DEC000A281B381F70180839183A283B383F4E0BD
:10DED000EF0EF11C0C5F1F4F8FEFC81AD80ABC124F
:10DEE000D2CF86E430DF8823B9F039DF20E030E09C
:10DEF000A9010E9459B118167CF431DF20E030E00E
:10DF000040E752E40E945DAF60934E0270934F026F
:10DF10008093500290935102DF91CF911F910F9106
:10DF2000FF90EF90DF90CF90BF900895CF92DF9257
:10DF3000EF92FF926B017C010E94EF11C60ED71E7B
:10DF4000E81EF91E0E94EF11DC01CB018C199D091E
:10DF5000AE09BF09B7FF03C00E94E4ADF3CFFF9045
:10DF6000EF90DF90CF9008956F927F928F929F9263
:10DF7000AF92BF92CF92DF92EF92FF920F931F93D7
:10DF8000CF93DF93CDB7DEB73C01A090440CB090A7
:10DF9000450CCDB6DEB66AE070E0C3010E94CCB697
:10DFA0007C01009721F08C010619170904C0C301F8
:10DFB0000E94D7B68C01C80101962DB73EB7281B29
:10DFC000390B0FB6F8943EBF0FBE2DBF8DB79EB76D
:10DFD00001964C01A801B3010E94F8B6F401E00FCC
:10DFE000F11F1082C40148D581E034D0E114F1045E
:10DFF00051F037019FEF691A790A0FB6F894DEBE27
:10E000000FBECDBEC6CF0FB6F894DEBE0FBECDBEDE
:10E01000C501DF91CF911F910F91FF90EF90DF909D
:10E02000CF90BF90AF909F908F907F906F9024C5BE
:10E03000CF93C3E00E94178A882341F0C15019F0A2
:10E040000E94EBACF7CFCF910C9418AD8EEE95E11A
:10E05000CF918ACFCF93C82F41E04093150C909178
:10E060003F0C9D3409F45EC0943509F4F7C1973430
:10E0700009F0F8C120913D0C30913E0C2B31310557
:10E0800009F43EC0CCF42430310544F4223031058B
:10E0900064F537FDE7C10E94F799E7C12C303105DF
:10E0A00061F12531310509F4E0C12430310509F071
:10E0B000D9C10E94219AD9C12A35310551F154F4B0
:10E0C0002D31310521F1FCF02E31310509F0CAC1A5
:10E0D00051D2CBC12C35310511F1F4F0293A314040
:10E0E00009F0C0C10E94CD87C0C181E02230310556
:10E0F00009F080E00E945E9EB8C10E940B95B5C1F8
:10E100000E940F95B2C180E00E947E7EAEC190DF7A
:10E11000ACC11092B805A9C14093B805A6C10E9430
:10E12000997CA3C120913D0C30913E0C29373105DB
:10E1300009F45DC10CF083C02836310509F42AC109
:10E140000CF044C02C34310509F421C104F522310E
:10E15000310509F43EC164F437FD84C12230310534
:10E160000CF40DC12131310509F07CC1E9D77DC125
:10E170002A32310509F405C12B34310509F404C1F3
:10E180002F31310509F06EC10E94727B6EC12335BB
:10E19000310509F41BC16CF42135310509F411C1B5
:10E1A0000CF011C12D34310509F05CC10E94B07A28
:10E1B0005CC12535310509F40EC10CF40AC12C35BA
:10E1C000310509F04FC10E949E964FC1203731059D
:10E1D00009F44BC1CCF42C36310509F446C15CF48A
:10E1E0002A36310509F4E7C00CF0E8C00E94B9A452
:10E1F0001092150C41C12E36310509F4CEC00CF039
:10E20000CFC00E9432A431C12537310509F4E8C0DE
:10E210006CF42237310509F4E0C00CF4C3C0233795
:10E22000310509F01FC10E942B7C1FC12737310522
:10E2300009F4D8C00CF0D9C00E94DF7B16C12E357E
:10E2400081E0380709F408C10CF04BC0233D3105CB
:10E2500009F4D8C01CF5293C310509F4CAC07CF486
:10E260002B39310509F4A4C02E3B310509F49DC0BA
:10E270002C38310509F0F6C00E9489A3F6C02C3C69
:10E28000310509F4B9C02D3C310509F4B8C02B3C67
:10E29000310509F0E7C00E943898E7C02D3281E0CF
:10E2A000380709F4B6C07CF42D3D310509F4ACC043
:10E2B000223E310509F4ABC02C3D310509F0D2C036
:10E2C0000E944D96D2C02F3281E0380709F4A7C0D2
:10E2D0000CF4A2C02033314009F0C4C00E94DB9589
:10E2E000C4C0243F81E0380709F4A8C014F52239DE
:10E2F00081E0380709F49AC06CF4203981E03807CE
:10E3000009F490C00CF090C02F35314009F0AAC03C
:10E31000ABD5ABC0243A81E0380709F489C0293A6B
:10E3200081E0380709F487C02A39314009F09AC0E2
:10E330009CC0283F81E0380709F486C04CF4263F92
:10E3400081E0380709F47CC00CF07CC010D58DC08A
:10E35000243883E0380709F479C034F42335334096
:10E3600009F080C040D281C02B3883E0380709F41F
:10E3700070C0273E334009F075C0E2D776C0ACD2FA
:10E3800074C00E944D7A71C00E94AC7A6EC00E9427
:10E39000AE7A6BC00E940FA468C00E947F7C65C0EB
:10E3A00055D763C00E949D7B60C00E94A2A35DC040
:10E3B0000E94C8A35AC00E9488A457C00E94B2A459
:10E3C00054C0ADD752C00E94F0994FC00E94F3993B
:10E3D0004CC0B8D64AC063D648C00E94DB7B45C05B
:10E3E0007AD243C00E94D37B40C0D0D73EC0D1D7A1
:10E3F0003CC00E94099839C00E945D9836C00E94B6
:10E40000D39833C0CBD731C00E9480952EC00AD696
:10E410002CC00E94599929C00E94729726C00E9460
:10E42000D4A223C0B9D721C09BD01FC09ED01DC08D
:10E430000E94FD881AC00E94287D17C096D415C07E
:10E4400098D413C098D411C0BBD40FC00E94939429
:10E450000CC00E945B9509C0D2D407C080913D0CCE
:10E4600069D603C08EE19CE072D41092150CC111E4
:10E4700003C0CF910C94EFA0CF910895CF93DF9379
:10E48000C091C10E80E6C89FE0011124C052D34F55
:10E490008091A70380FF05C00E948516CE010E94CF
:10E4A000381CCE01E9D280E0DF91CF91D3CDCF925D
:10E4B000DF92EF92FF920F931F930E94EF116B0177
:10E4C0007C018091E10E81112FC080916802882328
:10E4D00059F18091150C882339F14091110C50911C
:10E4E000120C6091130C7091140C97018601041B9F
:10E4F000150B260B370B37FD2CC0833079F03CF41D
:10E50000813094F00E9485168CED95E10BC084302B
:10E5100059F40E9485168DEA95E104C00E94851683
:10E5200085EC95E10E9477162091680230E0A8EE14
:10E53000B3E00E94DAB2DC01CB018C0D9D1DAE1D53
:10E54000BF1D8093110C9093120CA093130CB093E9
:10E55000140C1F910F91FF90EF90DF90CF900895D2
:10E5600081E00E948F4F0C94735280E00E948F4F85
:10E570000C9473528F929F92AF92BF92CF92DF9280
:10E58000EF92FF920F931F93CF93DF93CDB7DEB738
:10E5900028970FB6F894DEBF0FBECDBFC0905202D1
:10E5A000D0905302E0905402F090550288E5CBDB06
:10E5B000811108C020E030E0A901C701B6010E9426
:10E5C0007DAE01C0CCDB6D837E838F839887C09046
:10E5D0005602D0905702E0905802F090590289E517
:10E5E000B2DB811108C020E030E0A901C701B6010B
:10E5F0000E947DAE01C0B3DB6B017C0169837A832D
:10E600008B839C838D809E80AF80B8842CE933E31C
:10E6100043E651EC0E9459B187FDD2C024ED3CEC99
:10E6200046E353E4C701B6010E9456AF18160CF436
:10E63000C7C023EA31E040E450ECC501B4010E94B8
:10E6400059B187FDBDC027E030E042E253E4C50187
:10E65000B4010E9456AF18160CF4B2C027E030E0A7
:10E6600041E253E4C501B4010E9456AF18160CF400
:10E67000A7C027E030E041E253E4C701B6010E94A1
:10E6800056AF18160CF49CC080E00E94D51D0E9465
:10E69000735485E458DB182F8823B1F08091400C27
:10E6A0009091410C892B09F489C090DB97FD0FC034
:10E6B0008DDB6F3F71058105910509F04CF486DB18
:10E6C00061117CC040E005C085E4F6DA77C010E057
:10E6D000412F01E021E0BE016F5F7F4FCE01059623
:10E6E0000E9430506B017C019B01AC010E9442B240
:10E6F00081115FC08D809E80AF80B88420E030E0C3
:10E70000A901C501B4010E9456AF87FD05C027E1EC
:10E7100037EB41E558E304C027E137EB41E558EB1F
:10E72000C501B4010E947DAEAB01BC0182E296E15D
:10E730000E94C21689809A80AB80BC8020E030E0C5
:10E74000A901C501B4010E9456AF87FD05C027E1AC
:10E7500037EB41E558E304C027E137EB41E558EBDF
:10E76000C501B4010E947DAEAB01BC018DE196E113
:10E770000E94C21620E030E0A901C701B6010E9444
:10E7800056AF87FD05C027E137EB41E558E304C0EC
:10E7900027E137EB41E558EBC701B6010E947DAE9A
:10E7A000AB01BC0188E196E10E94C2168AE00E949A
:10E7B000E11B0E9492540E94735202C041E089CF33
:10E7C00028960FB6F894DEBF0FBECDBFDF91CF9174
:10E7D0001F910F91FF90EF90DF90CF90BF90AF907F
:10E7E0009F908F900895EF92FF920F931F93CF9376
:10E7F000DF938AE561DA882309F456C08091400CE2
:10E800009091410C009709F44FC0FC017F01C19128
:10E810002C2F2F7D89F0C53411F0C536B9F7F701DB
:10E82000108260E070E08091400C9091410C0E9459
:10E83000F9B2F701C08304C060E070E00E94F9B251
:10E840008B01D82FC92F20E030E040E050EC0E942F
:10E8500059B187FD1DC020E030E040EA50E4B80126
:10E860008D2F9C2F0E9456AF181694F0C801AD2F23
:10E87000BC2F8093920590939305A0939405B09339
:10E880009505DF91CF911F910F91FF90EF90089523
:10E890000E9488168BE396E1DF91CF911F910F9133
:10E8A000FF90EF900C9477160E9485164091920588
:10E8B0005091930560919405709195058AE296E1D7
:10E8C0000E94C2168AE0DF91CF911F910F91FF90B5
:10E8D000EF900C94E11B0895CF92DF92EF92FF929C
:10E8E0000F931F93CF93DF93C091420CD091430CB1
:10E8F00080E529DA8823D1F08091400C9091410C79
:10E90000009749F04AE050E060E070E00E9487B56F
:10E910006B017C0103C0C12CD12C760111E0C11424
:10E92000D104E104F10431F410E004C010E0C12C82
:10E93000D12C760183E507DA882309F486C080911B
:10E94000400C9091410C009701F1FC017F01019175
:10E95000202F2F7D89F0053411F00536B9F7F70126
:10E96000108260E070E08091400C9091410C0E9418
:10E97000F9B2F701008304C060E070E00E94F9B2D0
:10E98000B62FA72FF82FE92F04C0B0E0A0E0F0E0E9
:10E99000E0E020E030E04AE754E46B2F7A2F8F2F3D
:10E9A0009E2F0E9494B10E94CAAF6B017C0111118D
:10E9B00009C0672B682B692B29F4209719F08881EF
:10E9C000811102C010E001C011E00E94C75E112356
:10E9D00029F00E948516CE010E94381C83E08093A6
:10E9E000150C81E08093E20EC114D104E104F1041E
:10E9F00029F10E94EF11C60ED71EE81EF91E0E94D3
:10EA0000EF11DC01CB018C199D09AE09BF09B7FDDF
:10EA10000EC01092E20E81E08093150CDF91CF9131
:10EA20001F910F91FF90EF90DF90CF90089580910C
:10EA3000E20E882371F30E94E4ADE1CF8091E20EF3
:10EA4000882339F30E94E4ADF9CF1111BBCFB5CFC4
:10EA50001092430C1092420C8FE380933F0C109263
:10EA60003E0C10923D0C1092390C10923A0C109200
:10EA70003B0C10923C0C08953F924F925F926F9224
:10EA80007F928F929F92AF92BF92CF92DF92EF923E
:10EA9000FF920F931F93CF93DF931F921F92CDB7D7
:10EAA000DEB789839A83D4DF8981282F9A81392F11
:10EAB000F90180812F5F3F4F8032D1F38E34B1F462
:10EAC000818190ED980F9A3020F08D3211F08B32C9
:10EAD00069F43296DF0131962C9120532A30D0F31D
:10EAE000CD01FC01019620812032D9F3F093450C31
:10EAF000E093440C8F010F5F1F4F30806AE270E09B
:10EB0000C8010E942EB7009731F0FC013197808137
:10EB10008032E1F311828DE4381631F0E4E53E16DF
:10EB200019F0F7E43F12FFC0F80180810F5F1F4F1B
:10EB30008032D1F380538A3008F0F5C030923F0C18
:10EB400010923E0C10923D0C4AE020913D0C309109
:10EB50003E0C429FC001439F900D112490933E0CA8
:10EB600080933D0C3196DF0111972C91022E000C01
:10EB7000330B20533109280F391F30933E0C20935B
:10EB80003D0C808180538A3000F3DF0131968C91F7
:10EB90008032D9F38DE438121AC02E31310591F04C
:10EBA0003CF42731310571F02C31310581F40AC074
:10EBB0002537310564F02737310524F0203AE3E0AA
:10EBC0003E0729F4B093430CA093420CACC01092C2
:10EBD000430C1092420C5091440CC12CD12C760164
:10EBE000C394FD0131964C91442309F49CC04132F9
:10EBF000A9F48DE4381212C02032310579F4F09373
:10EC0000430CE093420C63E270E0CF010E942EB708
:10EC1000009709F488C0FC01108285C041544A3134
:10EC200008F055C0BF01FB0180816F5F7F4F8032CC
:10EC3000D1F390ED980F9A3008F18E3211F4818162
:10EC40000CC08D3211F08B3259F4818190ED980F08
:10EC50009A30A0F08E3221F4828180538A3070F095
:10EC60008091420C9091430C892B09F059C0CF013F
:10EC700001979093430C8093420C52C0CF01A42F74
:10EC8000B0E04601570104C0880C991CAA1CBB1CAB
:10EC90004A95D2F74090390C50903A0C60903B0C5A
:10ECA00070903C0C84289528A628B7288092390CAF
:10ECB00090923A0CA0923B0CB0923C0C009711F051
:10ECC000851B01C080E0A15EB34F8C930AC0809188
:10ECD000420C9091430C892B21F4B093430CA093E8
:10ECE000420C808181548A3130F4DF017ACF80ED8B
:10ECF000890F8A3040F44E2F6F2F91919111F7CFE9
:10ED0000842F962F07C083ED890F8230A0F39B32AA
:10ED100091F3F6CFFC01019640814032D9F3E5CF63
:10ED200080E090E0ACCF0F900F90DF91CF911F91DA
:10ED30000F91FF90EF90DF90CF90BF90AF909F909A
:10ED40008F907F906F905F904F903F9008950E94BA
:10ED500085166091440C7091450C89E596E10E94FE
:10ED60008B1686E596E10C9477160C9430410C9442
:10ED7000804F0C942445CF9383E50E945C6EC82F8E
:10ED8000882331F08091400C9091410C892B41F403
:10ED900083E50E945C6EC1E08C2FCF910C948D4670
:10EDA00015D897FD0BC012D86F3F710581059105ED
:10EDB00009F094F70BD8C1E06111EECFC0E0ECCFC1
:10EDC0000E94794F882331F00E9485168CE696E1E7
:10EDD0000C94771608950E94E66E97FD0CC00E9471
:10EDE000E66E6F3F71058105910509F034F40E94CC
:10EDF000E66E862F089580E008958FEF08950F93B3
:10EE00001F93CF9383E50E945C6E811104C00FE4D1
:10EE100013E0C0E00DC0C0E0DEDF682F8C2F0E9441
:10EE2000A83FCF5FC530C1F7F2CFCF5FC43069F0E4
:10EE3000F80181918F010E945C6E8823B1F3CBDFD2
:10EE4000682F8C2F0E94A83FF0CF82E40E945C6E56
:10EE5000882329F0C0DF682F84E00E94A83FCF916B
:10EE60001F910F910C9455400F931F93CF9383E5FF
:10EE70000E94A36E882309F465C0ADDF823029F1BA
:10EE8000833009F43FC0813009F05CC00FE413E027
:10EE9000C0E0F80181918F010E94A36E882339F0B0
:10EEA0009ADF2FEF4FEF682F8C2F0E94513FCF5FDB
:10EEB000C43079F782E40E94A36E882309F442C02B
:10EEC0008ADF2FEF4FEF682F3AC00FE413E0C0E066
:10EED000F80181918F010E94A36E882339F07BDFB6
:10EEE0002FEF482F6FEF8C2F0E94513FCF5FC43020
:10EEF00079F782E40E94A36E882321F16CDF2FEF63
:10EF0000482F1CC00FE413E0C0E0F80181918F018D
:10EF10000E94A36E882339F05EDF282F4FEF6FEF3A
:10EF20008C2F0E94513FCF5FC43079F782E40E945A
:10EF3000A36E882339F04FDF282F4FEF6FEF84E067
:10EF40000E94513FCF911F910F910C945540CF9348
:10EF5000DF931F921F92CDB7DEB769837A830E9439
:10EF60005C6E69817A81882361F08091400C909178
:10EF7000410C009731F04AE050E060E070E00E9400
:10EF80005FB4972F862F0F900F90DF91CF91089548
:10EF9000CF93DF93EC0181E00E941F168AE090E09E
:10EFA0000E945912CC30D105C9F05CF4CA30D105A9
:10EFB00039F1CB30D10541F5C3B1C5FBCC27C0F940
:10EFC0001CC0C831D105A9F0CE31D10561F0C731DF
:10EFD000D105D1F4C0B1C695C1700FC0C3B1C6FB95
:10EFE000CC27C0F90AC0C6B1C095CC1FCC27CC1F16
:10EFF00012C0C0B1C2FBCC27C0F981E0C8270BC04A
:10F00000C3B1C295C170F9CF8C2F0E944E14C1E0DC
:10F01000892B09F4C0E080E00E941F168C2FDF913D
:10F02000CF9108950F931F93CF93DF9380E50E94B4
:10F030005C6E882379F160E070E080E588DF082F5E
:10F040006FEF7FEF83E583DFEC010196039710F507
:10F0500007FD20C00E94C75E002E000C110BCF3FA1
:10F060008FEFD80729F0219751F4C1E0D0E009C013
:10F07000C8018EDFC1E08C27C82FD0E002C0C0E0FD
:10F08000D0E0C80185DF90E08C179D0719F00E9441
:10F09000E4ADF7CFDF91CF911F910F9108950F93BA
:10F0A0001F93CF9383E50E945C6E882309F43EC0D2
:10F0B0008091400C9091410C009701F1FC018F016F
:10F0C000C1912C2F2F7D89F0C53411F0C536B9F7C9
:10F0D000F801108260E070E08091400C9091410C4A
:10F0E0000E94F9B2F801C08304C060E070E00E94A1
:10F0F000F9B2B62FA72FF82FE92F04C0B0E0A0E097
:10F10000F0E0E0E020E030E04AE754E46B2F7A2FB3
:10F110008F2F9E2F0E9494B10E94CAAF6093DD0E84
:10F120007093DE0E8093DF0E9093E00ECF911F91CF
:10F130000F91089520E040E050E0BA010C9496341D
:10F140000C94D1AC0F931F93CF9383E50E945C6E18
:10F15000882391F18091400C9091410C009761F1CE
:10F16000FC018F01C1912C2F2F7D89F0C53411F046
:10F17000C536B9F7F801108260E070E08091400C6C
:10F180009091410C0E94F9B2F801C08304C060E084
:10F1900070E00E94F9B220E030E04AE754E40E94B7
:10F1A00094B10E94CAAF6093690270936A0280931F
:10F1B0006B0290936C0246C088E50E945C6E8111E0
:10F1C00014C089E50E945C6E81110FC08AE50E941F
:10F1D0005C6E81110AC085E40E945C6E811105C0DD
:10F1E000CF911F910F910C94A25E0E94C75E88E59B
:10F1F0000E945C6E882331F0179A8091B9058E7F4A
:10F200008093B90589E50E945C6E882331F0169AD7
:10F210008091B9058D7F8093B9058AE50E945C6E67
:10F22000882331F0159A8091B9058B7F8093B905B9
:10F2300085E40E945C6E882329F0CF911F910F9185
:10F240000C94D6ACCF911F910F910895FF920F931C
:10F250001F93CF93DF9383E50E945C6E8823F1F0C8
:10F2600083E50E945C6E811102C060E015C0809150
:10F27000400C9091410C892BC1F30E94E66E97FDE2
:10F28000F4CF0E94E66E6F3F71058105910511F084
:10F290000CF043C00E94E66E6093A7030E9485169F
:10F2A0008BEA96E10E9477168091A703882349F1A3
:10F2B00001EA16E1C0E0D0E020E08091A70390E0F1
:10F2C000A0E0B0E00C2E04C0B695A7959795879561
:10F2D0000A94D2F780FF0EC0FF24F394F20E22238B
:10F2E00019F08CE20E94E11BF801859194910E9433
:10F2F00077162F2D21960E5F1F4FC530D105E9F6E9
:10F3000004C08DE996E10E9477168AE0DF91CF91E3
:10F310001F910F91FF900C94E11B6FEFBDCF0E94E6
:10F3200043260E9421AA0E94A25E60E070E080E075
:10F330000E94B72068EE73E080E090E00C943516F0
:10F3400081E080936E0283E50E945C6E882331F039
:10F350008091400C9091410C892B39F483E50E94F7
:10F360005C6E811112C00C944EA10E94E66E97FD56
:10F37000FACF0E94E66E6F3F71058105910509F095
:10F3800024F40E94E66E662371F3089581E00C94E4
:10F390002D3380E00C942D330C94C75ECF930E94E4
:10F3A000851682ED96E10E94771683E50E945C6ED9
:10F3B000C82F8823D1F08091400C9091410C892B6B
:10F3C00091F00E94E66E97FD0DC00E94E66E6F3FC1
:10F3D00071058105910509F034F40E94E66EC1E0E3
:10F3E000611101C0C0E0C0934702809147020E94B2
:10F3F000FC168AEC96E10E94771640912F025091FC
:10F400003002609131027091320288EC96E10E94E4
:10F41000C2164091370250913802609139027091C2
:10F420003A0285EC96E10E94C21640913F0250914B
:10F430004002609141027091420282EC96E10E948A
:10F44000C2168AEB96E10E947716409133025091E2
:10F450003402609135027091360288EB96E10E9489
:10F46000C21640913B0250913C0260913D02709166
:10F470003E0285EB96E10E94C216409143025091F4
:10F480004402609145027091460282EB96E10E942F
:10F49000C2168AE0CF910C94E11B0F931F93CF9378
:10F4A000DF9383E50E94A36E882309F450C093DCA8
:10F4B000182F80E50E94A36E81110AC081E011110E
:10F4C00001C080E0DF91CF911F910F910C941F1626
:10F4D00080E50E94A36E882331F00E94E66EEB0166
:10F4E00077FD35C002C0CDE0D0E00C2F89E40E944A
:10F4F000A36E882351F08091400C9091410C892B90
:10F5000049F069DC811106C017C089E40E945C6E75
:10F51000882391F061E08C2F0E94E313612F8C2FE0
:10F520000E941F14612F70E08C2F0E94C6120830B9
:10F5300071F41093EF040BC0802F0E949AAC8823C3
:10F5400049F3DF91CF911F910F910C94C2ACDF91E1
:10F55000CF911F910F9108950C949AAA0C9436AAFA
:10F560000C9421AA4F925F926F927F92AF92BF92BA
:10F57000CF92DF92EF92FF92CF93DF93EB01FC01EA
:10F5800060817181828193812CE3C22ED12CE12C88
:10F59000F12CA70196010E9494B2B62EA72ECA01A3
:10F5A000B901A70196010E9494B26B017C01CA01C6
:10F5B000B90128E130E040E050E00E9494B22B0114
:10F5C0003C01C9016DE671E00E946DB261157105E3
:10F5D000D9F0AF92BF92DF92CF925F924F929F93FA
:10F5E0008F937F936F938AE097E19F938F93DF933D
:10F5F000CF930E9459B78DB79EB70E960FB6F89469
:10F600009EBF0FBE8DBF61C00097C9F0AF92BF9281
:10F61000DF92CF925F924F929F938F938AEF96E102
:10F620009F938F93DF93CF930E9459B7EDB7FEB7A7
:10F630003C960FB6F894FEBF0FBEEDBF46C0411416
:10F64000510461047104B9F0AF92BF92DF92CF927E
:10F650005F924F928EEE96E19F938F93DF93CF93BD
:10F660000E9459B78DB79EB70A960FB6F8949EBF01
:10F670000FBE8DBF2AC0C114D104E104F104A9F06A
:10F68000AF92BF92DF92CF9286EE96E19F938F93D7
:10F69000DF93CF930E9459B7EDB7FEB738960FB6F8
:10F6A000F894FEBF0FBEEDBF10C0AF92BF9282EEC6
:10F6B00096E19F938F93DF93CF930E9459B70F905A
:10F6C0000F900F900F900F900F90DF91CF91FF90C0
:10F6D000EF90DF90CF90BF90AF907F906F905F9052
:10F6E0004F900895CF93DF93CDB7DEB769970FB6EC
:10F6F000F894DEBF0FBECDBF0E9466AA6E8B7F8BD3
:10F70000888F998FBE016F5F7F4FCE0146962ADFAB
:10F710000E948516BE016F5F7F4F8EE197E10E94C8
:10F720008B168AE00E94E11B69960FB6F894DEBF43
:10F730000FBECDBFDF91CF91089583E50E945C6E2F
:10F74000882331F08091400C9091410C892B71F409
:10F750000E9485164091680250E060E070E08BE204
:10F7600097E10E94EC168AE00C94E11B0E94E66E81
:10F7700097FD17C00E94E66E6F3F710581059105E8
:10F7800009F01CF40E94E66E01C06FEF862F90E036
:10F79000CD971CF46093680208958CE3809368020F
:10F7A000089560E0F3CF81E00E941F160E94943319
:10F7B00080E00C941F160E94C75E0C9473521F9336
:10F7C000CF93DF93C091420CD091430C83E010E0C3
:10F7D00040E08150C9F09881292F2B7F2134C9F74F
:10F7E00029812133B1F7913421F0953419F441E0A6
:10F7F00001C011E09E012E5F3F4FE9012F5F3F4F97
:10F8000098819032D1F3E5CF41110E9485161123E2
:10F8100021F082E397E10E947716CE01DF91CF912C
:10F820001F910C94381C0F931F93CF938C01C62FFC
:10F8300086E397E10E947716C8010E9477168AE353
:10F840000E94E11B6AE070E08C2F90E0CF911F9145
:10F850000F910C94DA1C8FE598E10E94771660E016
:10F860008FE498E1E0DF60E08AE398E1DCDF61E0CB
:10F8700083E398E1D8DF60E088E298E1D4DF61E0DB
:10F8800088E198E1D0DF60E08FE098E1CCDF61E0D3
:10F8900085E098E1C8DF61E08BEF97E1C4DF61E0CC
:10F8A00083EF97E1C0DF61E085EE97E1BCDF60E0C8
:10F8B00087ED97E1B8DF60E088EC97E1B4DF60E0C6
:10F8C0008AEB97E1B0DF60E084EA97E1ACDF61E0CA
:10F8D00083E997E1A8DF60E084E897E1A4DF60E0D6
:10F8E0008FE697E1A0DF61E08CE597E19CDF60E0C7
:10F8F0008FE497E198DF60E08BE397E194CF8EE4AB
:10F900000E945C6E8823A1F08091400C9091410C84
:10F91000009771F04AE050E060E070E00E945FB450
:10F920006093C30E7093C40E8093C50E9093C60E61
:10F9300008954F925F926F927F929F92AF92BF9283
:10F94000CF92DF92EF92FF920F931F93CF93DF93AB
:10F9500083E5E82E83E0F82E02E512E0B12C912C2D
:10F96000A12CF70181917F010E945C6E882309F42C
:10F9700050C08091400C9091410C009709F449C00F
:10F98000FC013F01C1912C2F2F7D89F0C53411F06E
:10F99000C536B9F7F301108260E070E08091400C49
:10F9A0009091410C0E94F9B2F301C08304C060E061
:10F9B00070E00E94F9B26B01D82FC92FF8012081A5
:10F9C0003181428153810E947CAE2B013C012DEBA1
:10F9D00037E346E855EB0E9459B187FD0AC02DEB8D
:10F9E00037E346E855E3C301B2010E9456AF18164B
:10F9F00084F4F3E0BF1619F09924939402C0AA246A
:10FA0000A394A6016D2F7C2FF8014083518362835C
:10FA10007383B3940C5F1F4FF4E0BF12A2CF992001
:10FA200019F00E949B5203C0A1100E94A552DF91C1
:10FA3000CF911F910F91FF90EF90DF90CF90BF90EB
:10FA4000AF909F907F906F905F904F900C94735207
:10FA5000BF92CF92DF92EF92FF920F931F93CF93BB
:10FA6000DF9337E5E32E33E0F32E07E614E067017A
:10FA7000C0E0D0E0BB24B394F60181916F010E94F5
:10FA80005C6E882359F10E94C75E8091400C909172
:10FA9000410C892B19F00E94AF6E18C0F8016081EB
:10FAA000662389F070E080E090E00E94F8AF9B014F
:10FAB000AC01FE01E659FB4F608171818281938127
:10FAC0000E945DAF03C060E070E0CB01FE01E95829
:10FAD000FB4F6083718382839383B12C24960F5FE5
:10FAE0001F4FCC30D10541F686E40E945C6E88231E
:10FAF00081F10E94C75E0E94AF6E8B01D82FC92F83
:10FB000020E030E040E85FE30E9459B118167CF035
:10FB100020E030E0A901B8018D2F9C2F0E9456AF44
:10FB200087FF09C000E010E0D0E0C0E004C000E0C2
:10FB300010E0D0E8CFE320E030E04FE753E4B80135
:10FB40008D2F9C2F0E9494B10E94CAAF60937604BF
:10FB5000B12C83E50E945C6E882369F00E94C75E29
:10FB60000E94AF6E60931002709311028093120294
:10FB700090931302B9C0BB2009F4B6C086E29AE1A3
:10FB80000E94771680917604811104C083E29AE185
:10FB90000E9477168AE19AE10E9477168091760496
:10FBA000F4E68F9FC001112481589F4F6FEF70E0E2
:10FBB0000E9481B270E080E090E00E94F6AF20E009
:10FBC00030E048EC52E40E945DAFAB01BC0186EF2F
:10FBD00099E10E94C21689ED99E10E94771687EBA0
:10FBE00099E10E94771607E714E0C7E5D3E023E028
:10FBF000D22EDE0C80E20E94E11B89910E94E11B63
:10FC0000F80161917191819191918F0142E050E0F1
:10FC10000E945F1D8AE00E94E11BDC12EBCF409145
:10FC2000100250911102609112027091130283E947
:10FC300099E10E94C2168AE00E94E11B81E799E1E6
:10FC40000E94771680916704882349F00AE614E041
:10FC5000C7E6D4E0CE0193E0D92ED80E31C0809112
:10FC600068048111F3CF809169048111EFCF8DE594
:10FC700099E10E9477162CC080E20E94E11BF701F7
:10FC800080810E94E11B68816623F1F070E080E0D2
:10FC900090E00E94F8AF9B01AC01F8016081718196
:10FCA000828193810E945DAF42E050E00E945F1D1F
:10FCB0002196FFEFEF1AFF0A0C5F1F4FDC1641F091
:10FCC00088818823A9F3D8CF60E070E0CB01ECCF26
:10FCD0008AE0DF91CF911F910F91FF90EF90DF901D
:10FCE000CF90BF900C94E11BDF91CF911F910F91AA
:10FCF000FF90EF90DF90CF90BF9008952F923F92AA
:10FD00004F925F926F927F928F929F92AF92BF922B
:10FD1000CF92DF92EF92FF920F931F93CF93DF93D7
:10FD2000CDB7DEB768970FB6F894DEBF0FBECDBF74
:10FD3000F82E81E00E941F168FE40E94A36E882394
:10FD4000B9F08091400C9091410C892BB1F00E9448
:10FD5000E66E97FD18C00E94E66E6F3F7105810543
:10FD6000910509F054F40E94E66E611106C00BC0C3
:10FD70008FE40E945C6E882331F09091BA059770F1
:10FD8000973009F4DDC10E94C75E209130062F8BA9
:10FD900080E00E94D51D0E94735481E00E94403390
:10FDA00088E50E945C6E082F89E50E945C6E182F22
:10FDB0008AE50E945C6EF1100AC0011305C00817A5
:10FDC00031F0102F202E01C0202E382E05C011E05A
:10FDD000222423943324339480E1E2E5F2E0A8EA7C
:10FDE000B5E001900D928A95E1F7332019F082E099
:10FDF0000E94795782E50E94A36E882371F1809159
:10FE0000400C9091410C009709F458C0FC016F011F
:10FE10000191202F2F7D89F0053411F00536B9F7B7
:10FE2000D6011C9260E070E08091400C9091410CF2
:10FE30000E94F9B2F601008304C060E070E00E9405
:10FE4000F9B2D62EE72EF82E092F20E030E0A901D6
:10FE50000E9456AF882391F105C0D12CE12C30E8E7
:10FE6000F32E00E4211003C0112309F409C18D2DE4
:10FE70009E2DAF2DB02F8093B0059093B105A09328
:10FE8000B205B093B30520915A0230915B024091C4
:10FE90005C0250915D026D2D7E2D8F2D902F0E9462
:10FEA00059B118165CF419821A821B821C82BE0199
:10FEB0006F5F7F4F80EB95E00E943454222009F45D
:10FEC00093C1112309F4D4C0109256021092570224
:10FED000109258021092590210925202109253023C
:10FEE00010925402109255020E949B52E4E3F5E1F5
:10FEF0002491288FE3E4F5E185909590A590B49046
:10FF0000E7E4F5E1C590D590E590F490A70196015E
:10FF1000C501B4010E9459B118162CF4A501940131
:10FF2000C701B60104C0A7019601C501B4010E9432
:10FF30005DAF2B013C01ECE2F5E185919591A59136
:10FF4000B4918D879E87AF87B88BE8E2F5E1859104
:10FF50009591A591B491898B9A8BAB8BBC8B2D8598
:10FF60003E854F855889BC01CD010E9456AF87FD63
:10FF700008C00D859E859D8BAF85AE8BB889BD87EA
:10FF800007C00989EA89ED8BFB89FE8B2C892D87B7
:10FF9000A3019201C301B2010E9494B120E030E0BC
:10FFA00040E85FE30E947DAE0E9401B29B01AC017C
:10FFB000602F7D898E899D850E9494B169877A879B
:10FFC0008B879C87E5E3F5E1049120E030E040EC8D
:10FFD0005FE3C701B6010E9494B16B017C01602F01
:10FFE000000F770B880B990B0E94F8AF9B01AC01B7
:10FFF000C701B6010E9494B169837A838B839C8385
:020000021000EC
:1000000020E030E040EC5FE3C501B4010E9494B110
:100010006B017C01A88D6A2FAA0F770B880B990BB7
:100020000E94F8AF9B01AC01C701B6010E9494B1D8
:100030006D837E838F839887AE01475F5F4FBE01DC
:100040006F5F7F4FCE0105960E9452540E94073386
:1000500010925602109257021092580210925902B2
:1000600010925202109253021092540210925502B2
:1000700080E00E9479571123D1F081E00E947957E6
:100080000E949B5280E00E944033211004C0812CCA
:10009000912C540106C0812C912C20EAA22E20EC38
:1000A000B22E111198C0C12CD12C76019AC00E9499
:1000B0009B5280E00E944033812C912C90EAA92E23
:1000C00090ECB92EC12CD12C7601332009F454C008
:1000D00019821A821B821C8220E030E040E050E44A
:1000E00060915A0270915B0280915C0290915D0276
:1000F0000E947CAE6D837E838F839887BE016F5F85
:100100007F4FCE0105960E94345420E030E0A901D3
:10011000C501B4010E9456AF81112EC020E030E02D
:10012000A901C701B6010E9456AF811125C00E94E6
:1001300002338F890E94D51D0E9492540E947352EF
:1001400080E00E941F1668960FB6F894DEBF0FBEBF
:10015000CDBFDF91CF911F910F91FF90EF90DF9076
:10016000CF90BF90AF909F908F907F906F905F9057
:100170004F903F902F90089519821A821B821C8203
:10018000A701960160915602709157028091580222
:10019000909159020E947CAE6D837E838F839887F5
:1001A000A501940160915202709153028091540212
:1001B000909155020E947CAE69877A878B879C87D5
:1001C000AE014F5F5F4FBE016B5F7F4FCE0109965F
:1001D0000E945254ACCFC12CD12C80EAE82E80E48E
:1001E000F82E311075CF91CF111147CF0E949B523D
:1001F00080E00E944033812C912C540175016401F0
:10020000F0CF80E1E2E5F2E0A8EAB5E001900D92DE
:100210008A95E1F708952F923F924F925F926F92E5
:100220007F928F929F92AF92BF92CF92DF92EF9286
:10023000FF920F931F93CF93DF93CDB7DEB72C9729
:100240000FB6F894DEBF0FBECDBF270138012C8753
:10025000488759876A877B878F83D3DF8F812C8577
:10026000488559856A857B858F3F51F094E0899F49
:10027000F0011124E855FA4F408351836283738360
:100280002F3F51F084E0289FF0011124E855FA4FE8
:1002900040825182628273829FEFC91651F084E0DE
:1002A000C89EF0011124E855FA4F80829182A28203
:1002B000B3824090A8055090A9056090AA0570905F
:1002C000AB0520E030E042E253E4C301B2010E94FA
:1002D00056AF87FF11C020E030E040E450ECC3018E
:1002E000B2010E9459B118166CF0412C512C70E4E7
:1002F000672E70EC772E06C0412C512C62E2662EE0
:1003000063E4762E4092A8055092A9056092AA0552
:100310007092AB058090AC059090AD05A090AE05B5
:10032000B090AF052DEC3CEC46E353E4B401C501BD
:100330000E9456AF87FF13C023E333E343E651EC3B
:10034000B401C5010E9459B1181694F093E39D833E
:1003500083E38E8343E6242E51EC352E0CC09DECB6
:100360009D838CEC8E8326E3222E33E4332E03C050
:100370008D829E8215018D819E81D1018093AC0575
:100380009093AD05A093AE05B093AF058090B005F6
:100390009090B105A090B205B090B30520E030E098
:1003A0004FE153E4C501B4010E9456AF87FF10C06E
:1003B00020E030E040E050ECC501B4010E9459B1AA
:1003C000181664F0812C912CA12C90ECB92E06C04B
:1003D000812C912C8FE1A82E83E4B82E8092B00559
:1003E0009092B105A092B205B092B30580E090E082
:1003F000A8E4B2E489839A83AB83BC83CE010196DF
:100400006C01850174012D813E81A101C301B201FE
:100410000E9480532C960FB6F894DEBF0FBECDBF5E
:10042000DF91CF911F910F91FF90EF90DF90CF90D0
:10043000BF90AF909F908F907F906F905F904F9004
:100440003F902F9008958F929F92AF92BF92CF923C
:10045000DF92EF92FF920F931F93CF93DF93EC0104
:100460006A017B0120E030E040E45FE36885798544
:100470008A859B850E947DAEA70196010E947DAE74
:10048000AB01BC01812C912C5401CC24CA94850170
:1004900074012FEF82E0BFDEEC80FD800E811F81B2
:1004A000488159816A817B8121E080E0B4DEDF915F
:1004B000CF911F910F91FF90EF90DF90CF90BF9061
:1004C000AF909F908F9008952F923F924F925F929E
:1004D0006F927F928F929F92AF92BF92CF92DF9254
:1004E000EF92FF920F931F93CF93DF93CDB7DEB7B9
:1004F0002E970FB6F894DEBF0FBECDBF89878B0154
:100500004A87222359F0812C912C90E8A92E9EE352
:10051000B92E80E090E0A0EAB1E40CC08AE0882E19
:1005200087ED982E83E2A82E8CE3B82E80E090E031
:10053000A0E8BFE389839A83AB83BC83211105C004
:1005400080E090E0A0EAB0E404C080E090E0A8E49D
:10055000B2E48D839E83AF83B88753DE412C512C48
:100560003201B985A4E0BA9FC0011124FC01E8550D
:10057000FA4F1F01C801110FAA0BBB0B8B879C8779
:10058000AD87BE872D813E814F815885C301B20161
:100590000E9456AF87FF3FC06B857C858D859E8509
:1005A0000E94F8AFA50194010E9494B19B01AC0197
:1005B000D1016D917D918D919C910E947DAEF10153
:1005C0006083718382839383E090B005F090B105DE
:1005D0000091B2051091B3052091AC053091AD05A5
:1005E0004091AE055091AF056091A8057091A905A5
:1005F0008091AA059091AB05DE0111966D010E94D4
:1006000080530E94C75E83B182958170B1E08B27D1
:10061000EA858E1324C0398524E0329FF00111242D
:10062000E855FA4F60817181828193812E960FB6D1
:10063000F894DEBF0FBECDBFDF91CF911F910F9118
:10064000FF90EF90DF90CF90BF90AF909F908F90F2
:100650007F906F905F904F903F902F900895A501ED
:100660009401C301B2010E947DAE2B013C018ACFEF
:100670004F925F926F927F928F929F92AF92BF92B2
:10068000CF92DF92EF92FF920F931F93CF93DF935E
:10069000CDB7DEB728970FB6F894DEBF0FBECDBF3B
:1006A000B82E6B01A42E4901C801B701FF24F394B1
:1006B00020E030E040EA50E40E9456AF8111F12C76
:1006C000A0DD84E0B89E80011124F801E855FA4FBE
:1006D00080819181A281B3818D839E83AF83B8870E
:1006E0002F2D4A2DB6018B2DEFDE2B013C018114FD
:1006F000910411F1F11020C041E04A2566277727C7
:100700006C197D0920E08B2DDFDEA30192010E9490
:100710007CAE6B017C0120E030E0A9010E9459B160
:1007200087FF04C0F7FAF094F7F8F094D401CD9263
:10073000DD92ED92FC921397F801E855FA4F8D8106
:100740009E81AF81B88580839183A283B38380E04B
:1007500090E0A8E4B2E489839A83AB83BC83E09001
:10076000B005F090B1050091B2051091B30520914C
:10077000AC053091AD054091AE055091AF0560914B
:10078000A8057091A9058091AA059091AB05DE019D
:1007900011966D010E948053C301B20128960FB6D5
:1007A000F894DEBF0FBECDBFDF91CF911F910F91A7
:1007B000FF90EF90DF90CF90BF90AF909F908F9081
:1007C0007F906F905F904F9008952F923F924F923D
:1007D0005F926F927F928F929F92AF92BF92CF92D1
:1007E000DF92EF92FF920F931F93CF93DF93CDB7DA
:1007F000DEB769970FB6F894DEBF0FBECDBF3C01E0
:100800004C8B5D8B6E8B7F8B2D878CE0EFE0F3E064
:10081000DE01119601900D928A95E1F74C895D8970
:100820006E897F89C3010FDE2D852230D1F060F4FF
:100830002223F1F0213009F073C1212C312C60E822
:10084000462E6FEB562E46C03D853330C9F134300D
:1008500009F066C1212C312C70E8472E7FEB572E12
:1008600036C0212C312CF0E84F2EFFE35F2E2FC035
:100870009301205E3F4FEC88FD880E891F8941E07F
:100880006FEF7FEF82E0F4DE6B017C0120E030E06F
:1008900040E05FE369857A858B859C850E9494B1F1
:1008A0009B01AC01C701B6010E947CAEF3016087D9
:1008B000718782879387C486D586E686F78630C19E
:1008C000212C312CE0E84E2EEFE35E2E03C0DD2418
:1008D000D39401C0D12C2D2D30E03F872E870023EB
:1008E00009F463C0C901880F991F880F991F73010C
:1008F000E80EF91EE1E0F0E0EC0FFD1FE80FF91F34
:1009000020E030E040E05FE360817181828193818B
:100910000E9494B1F701E05CFF4F20813181428158
:1009200053810E947CAE9B01AC01C201B101905881
:100930000E9494B1F70120813181428153810E944C
:100940007DAEAB01BC01812C912C5401CC24CA9406
:10095000850174012FEF8D2D5EDCEC88FD880E89FA
:100960001F899301205E3F4F41E06FEF7FEF82E0F0
:100970007FDE4B015C01F30164877587868797876B
:1009800020E030E040E05FE369857A858B859C85D7
:100990000E9494B19B01AC01C501B4010E947CAEE0
:1009A000F30160877187828793878E859F85880F83
:1009B000991F880F991F9301280F391F3F872E8792
:1009C000E1E0F0E0EC0FFD1FE80FF91F20E030E060
:1009D00040E05FE360817181828193810E9494B1E4
:1009E000688B798B8A8B9B8B52014101B7FAB0944B
:1009F000B7F8B0948E859F85805C9F4F998F888FC4
:100A000020E030E040E05FE3FC01608171818281A1
:100A100093810E9494B19B01AC01688979898A898C
:100A20009B890E947DAE2C893D894E895F890E94F9
:100A30007DAE9B01AC01C501B4010E9494B1EE856D
:100A4000FF8520813181428153810E947DAEAB01BF
:100A5000BC01812C912C5401CC24CA9485017401D1
:100A60002FEF8D2DD8DB23E333E343E35FE3F30183
:100A700064857585868597850E947CAEAB01BC0137
:100A80002FEF82E0C8DBFD85AF2EB12C450128E0B9
:100A9000820E911C880C991C880C991C860C971C42
:100AA000C201B1010E94C5AFEC88FD880E891F8983
:100AB000940141E08D2DDCDD6B017C0120E030E014
:100AC00040E05FE3E88DF98D6081718182819381DF
:100AD0000E9494B19B01AC01688979898A899B89BC
:100AE0000E947DAE9B01AC01C201B1010E9494B194
:100AF0009B01AC01C701B6010E947DAEEE85FF856A
:100B00006083718382839383F5013396EE0FFF1F19
:100B1000EE0FFF1FE60DF71DC082D182E282F38245
:100B200069960FB6F894DEBF0FBECDBFDF91CF91AF
:100B30001F910F91FF90EF90DF90CF90BF90AF90FB
:100B40009F908F907F906F905F904F903F902F90ED
:100B50000895CF92DF92EF92FF920F93CF93DF939E
:100B6000EC016A017B0100E020E02FDE22E0B7010A
:100B7000A601CE012ADE23E0B701A601CE0125DEC3
:100B8000B701A601CE015FDC1CAA1DAA1EAA1FAADE
:100B900018AE19AE1AAE1BAE288539854A855B851D
:100BA00060E070E0CB010E947CAE6CAF7DAF8EAF99
:100BB0009FAFDF91CF910F91FF90EF90DF90CF909B
:100BC00008958F929F92AF92BF92FF920F931F93BF
:100BD000CF93DF93EC01F09076048FEF809376044F
:100BE0008090100290901102A0901202B090130217
:100BF000109210021092110210921202109213021F
:100C0000CE01A7DF0E94C75E02E512E02CAD3DAD2C
:100C10004EAD5FADF80160857185828593850E9438
:100C20007DAEF80160877187828793871886198661
:100C30001A861B861CAE1DAE1EAE1FAE0E949B52B6
:100C40008092100290921102A0921202B0921302AE
:100C5000F0927604DF91CF911F910F91FF90BF909A
:100C6000AF909F908F9008952F923F924F925F92F6
:100C70006F927F928F929F92AF92BF92CF92DF92AC
:100C8000EF92FF920F931F93CF93DF9300D01F92A9
:100C9000CDB7DEB75C01D0907604109276048091D7
:100CA000100290911102A0911202B0911302898357
:100CB0009A83AB83BC83109210021092110210929F
:100CC000120210921302C50144DFE7E7F4E0D501F8
:100CD0009C964D915D916D917C919F97408351833E
:100CE0006283738398964D915D916D917C919B97F2
:100CF000448355836683778390964D915D916D9182
:100D00007C91939740875187628773878FEF809399
:100D10007604109210021092110210921202109298
:100D2000130282E5282E82E0382E20E030E040E4F5
:100D300050E4F10160857185828593850E947DAEC6
:100D40004B015C0120E030E040E450E4D101149616
:100D50006D917D918D919C9117970E947DAE2B0195
:100D60003C0120E030E040E450E4F1016081718119
:100D7000828193810E947DAEAB01BC0192E0C92EBD
:100D80008301720121E080E046DA20E030E040E4B7
:100D900050E4D10118966D917D918D919C911B9796
:100DA0000E947CAE4B015C0120E030E040E450E466
:100DB000F10164817581868197810E947CAE2B014F
:100DC0003C0120E030E040E450E4D1016D917D91A0
:100DD0008D919C910E947CAEAB01BC01830172019C
:100DE00021E080E018DA89819A81AB81BC8180930F
:100DF000100290931102A0931202B0931302D092AA
:100E000076040F900F900F900F90DF91CF911F916C
:100E10000F91FF90EF90DF90CF90BF90AF909F9099
:100E20008F907F906F905F904F903F902F9008959C
:100E3000CF92DF92EF92FF92CF93C09176042FEF83
:100E400020937604C0901002D0901102E09012021C
:100E5000F0901302109210021092110210921202DE
:100E600010921302AEDEC0921002D0921102E092F4
:100E70001202F0921302C0937604CF91FF90EF908C
:100E8000DF90CF9008959C018CE0EBE1F3E0D90175
:100E900001900D928A95E1F798E0E7E2F3E0D9013D
:100EA000A05CBF4F01900D929A95E1F708954F9283
:100EB0005F926F927F928F929F92AF92BF92CF92EA
:100EC000DF92EF92FF920F931F93CF93DF93CDB7F3
:100ED000DEB7C854D1090FB6F894DEBF0FBECDBF40
:100EE000CE010196D0DFD09076048FEF8093760408
:100EF0004090100250901102609012027090130204
:100F0000109210021092110210921202109213020B
:100F100040E050E060EA70E4CE01019689DF40E0F5
:100F200050E060E87FE3CE0101969EDE40E050E0B5
:100F300060E87FE3CE0101967BDF812C912C540188
:100F4000CC24CA94850174012FEF40E050E066E1A3
:100F500073E480E060D940921002509211026092D6
:100F6000120270921302D0927604C85BDF4F0FB664
:100F7000F894DEBF0FBECDBFDF91CF911F910F91CF
:100F8000FF90EF90DF90CF90BF90AF909F908F90A9
:100F90007F906F905F904F9008959F92AF92BF9215
:100FA000CF92DF92EF92FF920F931F93CF93DF9335
:100FB000CDB7DEB7C854D1090FB6F894DEBF0FBE67
:100FC000CDBF81E00E941F16009147021092470298
:100FD0009090300680E00E94D51D41E061E081E004
:100FE0000E9423568111EEC0CE0101964CDF85E5AB
:100FF0000E945C6E882341F12091400C3091410C9D
:101000002115310509F1F9015F011191812F8F7DC2
:1010100099F0153411F01536B9F7F501108260E03A
:1010200070E08091400C9091410C0E94F9B26B01EC
:101030007C01F50110830EC060E070E0C9010E94E0
:10104000F9B26B017C0106C0C12CD12C80E8E82EDE
:101050008FE3F82E82E40E945C6E882331F0B701A2
:10106000A601CE01019600DEADC084E50E945C6E53
:10107000882391F08091400C9091410C009731F0C1
:101080004AE050E060E070E00E945FB4B701A60162
:10109000CE01019696DD96C086E50E945C6E88239F
:1010A00009F48FC0B701A601CE01019652DD8AE096
:1010B0000E94E11B8DEB9AE10E9477164D855E85BB
:1010C0006F85788985EB9AE10E94C2168AE00E94BA
:1010D000E11B498D5A8D6B8D7C8D8CEA9AE10E94C3
:1010E000C2168AE00E94E11B4D895E896F89788D66
:1010F00082EA9AE10E94C2168AE00E94E11B8AE01D
:101100000E94E11B89E99AE10E94771649855A8578
:101110006B857C8586E99AE10E94C2168AE00E946E
:10112000E11B8AE00E94E11B8BE89AE10E9477169E
:101130004DA55EA56FA578A982E89AE10E94C21626
:101140008AE00E94E11B49A55AA56BA57CA588E70A
:101150009AE10E94C2168AE00E94E11B49A15AA1AD
:101160006BA17CA180E79AE10E94C2168AE00E94EE
:10117000E11B8AE00E94E11B82E59AE10E9477165A
:101180008AE00E94E11B84E50E94E11B6AE070E0B6
:1011900080E090E00E94D41C8EE39AE10E947716D2
:1011A00021964CAD5DAD6EAD7FAD21978BE39AE19D
:1011B0000E94C2168AE00E94E11B8AE00E94E11BA5
:1011C00001C075DE892D0E94D51D0093470280E085
:1011D0000E941F16C85BDF4F0FB6F894DEBF0FBE2C
:1011E000CDBFDF91CF911F910F91FF90EF90DF90D6
:1011F000CF90BF90AF909F9008951F93CF93DF93B0
:10120000CDB7DEB72C970FB6F894DEBF0FBECDBFBB
:1012100083E50E945C6E8823B9F08091400C909128
:10122000410C892BC9F00E94E66E97FD10C00E9408
:10123000E66E6F3F71058105910509F06CF40E941F
:10124000E66E611109C003C01091300606C080E04F
:101250000E94D51D10E001C011E0809152029091D2
:101260005302A0915402B091550289839A83AB83B3
:10127000BC838091560290915702A0915802B09180
:1012800059028D839E83AF83B88780915A029091D3
:101290005B02A0915C02B0915D0289879A87AB875F
:1012A000BC8786E50E945C6E882331F062EF7AE1AC
:1012B0008CE096E00E944CA9812F0E94D51D11233D
:1012C00051F080913006811106C00E94881683ED8E
:1012D0009AE10E9477160E94851685EC9AE10E9499
:1012E0007716809130060E9404174CE050E062E5CA
:1012F00072E0CE0101960E9421B7892B59F02C96FD
:101300000FB6F894DEBF0FBECDBFDF91CF911F9116
:101310000C9473522C960FB6F894DEBF0FBECDBF5F
:10132000DF91CF911F9108958F929F92AF92BF92BC
:10133000CF92DF92EF92FF92CF934B015C01690154
:101340007A012CE933E343E651ECC701B6010E9470
:1013500059B187FD33C024ED3CEC46E353E4C701AB
:10136000B6010E9456AF18164CF123EA31E040E472
:1013700050ECC501B4010E9459B187FD1FC027E0A0
:1013800030E042E253E4C501B4010E9456AF1816A2
:10139000ACF027E030E041E253E4C501B4010E9423
:1013A00056AF18165CF0C1E027E030E041E253E4AC
:1013B000C701B6010E9456AF18160CF4C0E08C2F7E
:1013C000CF91FF90EF90DF90CF90BF90AF909F9024
:1013D0008F900895CF93DF93D82FC62F0E94A36ECE
:1013E0008823D1F08091400C9091410C892B11F40D
:1013F00081E01AC00E94E66E97FD15C00E94E66E5D
:101400006F3F71058105910509F094F70E94E66E22
:1014100081E0611109C007C08D2F0E945C6E8111AF
:10142000E7CF8C2F01C080E0DF91CF9108952F92FC
:101430003F924F925F926F927F928F929F92AF9264
:10144000BF92CF92DF92EF92FF920F931F93CF93B1
:10145000DF93CDB7DEB7CB51D1400FB6F894DEBFE6
:101460000FBECDBF81E00E941F1641E061E081E028
:101470000E94235681111AC080913006882329F0DA
:1014800060E08FE4A7DF811111C0FE0131968CE38B
:10149000DF011D928A95E9F7309030068AE40E94B8
:1014A0005C6EB82E882329F00E94F41DB12C0C9498
:1014B000669460E070E086E50E94A777C351DF4F35
:1014C00099838883CD5ED040059718F085ED9CE127
:1014D00073C160E084E47EDFC950DF4F8883C75F5B
:1014E000D040C351DF4F28813981CD5ED0402330B9
:1014F00031054CF460E084E56DDFC450DF4F888334
:10150000CC5FD04006C031E0C450DF4F3883CC5FA1
:10151000D04062E070E088E50E94A777182F62E073
:1015200070E089E50E94A777082F80E50E94A36EEE
:10153000811103C0612F802F03C00E94E66E862FA9
:10154000623019F08CEA9CE137C1823019F083E8EF
:101550009CE132C183E50E94A36E882319F00E94AA
:10156000AF6E04C060E070E88BEB95E420E030E003
:1015700040E752E40E945DAF6093480270934902D5
:1015800080934A0290934B0288E40E945C6E882309
:1015900009F46EC00E94AF6E0E94C5AF2B013C01E2
:1015A000CB01820177FF02C00F5F1F4F1595079592
:1015B000119501951109035B1F4F0E3F4FEF140763
:1015C00014F40DEF1FEF6801C40CD51C51EAC516C9
:1015D000D1041CF051EAC52ED12CB20197FF02C0F4
:1015E0006F5F7F4F75956795072E000C880B990BE1
:1015F0000E94F8AF9B01AC0160E070E08BE992E4DF
:101600000E947CAE962EA72E7C0123E333E343E6B3
:1016100051EC0E9459B118162CF053E343E333E622
:1016200021EC04C0592D4A2D3E2D2F2D652F742FEE
:10163000832F922F0E94C5AF4B01640D751D072E9D
:10164000000C880B990B0E94F8AF2B013C0120E0A5
:1016500030E041E253E40E9456AF87FD06C0412CC2
:10166000512C31E2632E33E4732EC301B20131C039
:101670008CE40E94A36E882331F00E94AF6E0E941A
:10168000C5AF8B0102C00DEF1FEF82E50E94A36E74
:10169000882331F00E94AF6E0E94C5AF6B0103C07A
:1016A00021EAC22ED12C86E40E94A36E882331F059
:1016B0000E94AF6E0E94C5AF4B0104C092EF892E0D
:1016C00099249A9482E40E94A36E882331F00E94A8
:1016D000AF6E0E94C5AF7B0103C081EAE82EF12CFA
:1016E000B401092C000C880B990B0E94F8AFC25072
:1016F000DF4F688379838A839B83CE5FD040B801B4
:10170000012E000C880B990B0E94F8AFCE5FDE4FC4
:10171000688379838A839B83C250D140C250DF4F54
:10172000288139814A815B81CE5FD040FDDD8823ED
:1017300009F440C0B7010F2C000C880B990B0E94D4
:10174000F8AF9B01AC01B6010D2C000C880B990B76
:10175000C85EDE4F2883C851D140C75EDE4F388354
:10176000C951D140C65EDE4F4883CA51D140C55EE3
:10177000DE4F5883CB51D1400E94F8AFC85EDE4F98
:101780002881C851D140C75EDE4F3881C951D14050
:10179000C65EDE4F4881CA51D140C55EDE4F5881DA
:1017A000CB51D140C1DDCA50DF4F8883C65FD040E6
:1017B000811106C087E69CE10E9477160C9466941E
:1017C000B601601B710B072E000C880B990B0E9451
:1017D000F8AFC85FDE4F688379838A839B83C850E4
:1017E000D140B70168197909072E000C880B990BB5
:1017F0000E94F8AFC45FDE4F688379838A839B833E
:10180000CC50D140C351DF4FE881F981CD5ED0404B
:10181000EF2B91F081E59CE10E947716C950DF4FD4
:101820008881C75FD040882321F087E49CE10E9433
:1018300077168AE00E94E11B0E94C75E80E00E944A
:10184000D51D81E00E948F4F882329F0832D0E94AF
:10185000D51D0C9466940E94735460E085E4BADD53
:10186000811107C092E0C350DF4F9883CD5FD04015
:1018700006C0A1E0C350DF4FA883CD5FD040C15167
:10188000DF4F19821882CF5ED040C752DF4F1882D7
:1018900019821A821B82C95DD040C850DF4F18825E
:1018A00019821A821B82C85FD040C751DF4F18824D
:1018B000C95ED040EFEFFFEFC352DF4FF983E883FB
:1018C000CD5DD040FFEFCB50DF4FF883C55FD040F8
:1018D0002FEFCD50DF4F2883C35FD04031E0CB5294
:1018E000DF4F3883C55DD040C352DF4F8881998177
:1018F000CD5DD0400196880F991F880F991FEDE3A9
:10190000F0E0EC0FFD1FE80FF91FCB51DF4FF9831B
:10191000E883C55ED0409C0124503109C05FDE4F92
:1019200039832883C051D1408CE0C352DF4FA88156
:10193000B981CD5DD0408A9FA0018B9F500D1124AD
:10194000CA5FDE4F59834883C650D140CF51DF4F25
:1019500019821882C15ED040C151DF4F2881398180
:10196000CF5ED040032E000C440B550BCE5EDE4FF5
:10197000288339834A835B83C251D140C151DF4FF1
:1019800048815981CF5ED040440F551FCA5EDE4F5B
:1019900059834883C651D140CB52DF4F5881C55D32
:1019A000D040CD50DF4F8881C35FD040581709F435
:1019B00097C2CE5EDE4F688179818A819B81C25158
:1019C000D1400E94F8AF9B01AC01C85FDE4F688137
:1019D00079818A819B81C850D1400E9494B19B013A
:1019E000AC01CE5FDE4F688179818A819B81C250D4
:1019F000D1400E947DAE4B015C01CB52DF4F58813C
:101A0000C55DD040652F550F770B880B990B0E9451
:101A1000F8AF9B01AC01C45FDE4F688179818A8198
:101A20009B81CC50D1400E9494B19B01AC01C2502B
:101A3000DF4F688179818A819B81CE5FD0400E948F
:101A40007DAE6B017C0120E030E0A901C501B4014D
:101A50000E9456AF87FD05C020E030E040E05FE324
:101A600003C020E030E0A901C501B4010E947DAEB1
:101A70000E9433B0C355DF4F688379838A839B8389
:101A8000CD5AD04020E030E0A901C701B6010E9444
:101A900056AF87FD05C020E030E040E05FE303C0C3
:101AA00020E030E0A901C701B6010E947DAE0E948E
:101AB00033B0C755DF4F688379838A839B83C95AC4
:101AC000D040C352DF4F88819981CD5DD0400196CF
:101AD000C352DF4F99838883CD5DD040CA5EDE4F0D
:101AE000E881F981C651D140CB52DF4F9881C55D65
:101AF000D040E90FF11D97FDFA95EE0FFF1FA1EA07
:101B0000B0E0AC0FBD1FEA0FFB1FC352DF4F2881AF
:101B10003981CD5DD0403183208301E0C351DF4F57
:101B20002881CD5ED040C350DF4F4881CD5FD0408B
:101B3000BE0167557F4FCE0183559F4F0E943050A5
:101B4000C752DF4F688379838A839B83C95DD04006
:101B50009B01AC010E9442B2882321F0832D0E9498
:101B6000D51DD5C1C752DF4F288139814A815B819C
:101B7000C95DD040C850DF4F688179818A819B81DF
:101B8000C85FD0400E947DAEC850DF4F6883798324
:101B90008A839B83C85FD040CF51DF4FE881F981B2
:101BA000C15ED040C05FDE4F48815981C051D140F5
:101BB000E40FF51F8DE690E08C0F9D1FE80FF91FD5
:101BC000C752DF4F288139814A815B81C95DD0408E
:101BD0002483358346835783C355DF4F488059801C
:101BE0006A807B80CD5AD040CB51DF4FA881B9812C
:101BF000C55ED0404D925D926D927D92CB51DF4F8C
:101C0000B983A883C55ED040CF51DF4FE881F98109
